:020000040800F2
:100000000000012059750008EF330008F1330008A3
:10001000F3330008F5330008F73300080000000050
:10002000000000000000000000000000F93300089C
:10003000FB33000800000000FD330008FF33000818
:10004000A9750008A975000801340008A975000801
:10005000A9750008A97500080D3400081D340008B2
:10006000A97500082D340008A9750008353400086A
:10007000413400084D340008A9750008A97500082E
:10008000593400085D340008A9750008A9750008F6
:1000900000000000A975000869340008A97500086F
:1000A000A9750008A9750008A9750008A9750008B8
:1000B000A9750008A9750008A9750008A9750008A8
:1000C000A9750008A97500086D340008A975000815
:1000D000A975000879340008A9750008A9750008F9
:1000E000A9750008A975000885340008A9750008DD
:1000F000A97500080000000000000000A9750008B4
:10010000A9750008A975000891340008A9750008B0
:10011000A9750008A9750008A9750008A975000847
:10012000A9750008A9750008A9750008A975000837
:08013000A9750008A97500087B
:1001400010B5054C237833B9044B13B10448AFF311
:1001500000800123237010BDC807002000000000AC
:10016000541B030808B5034B1BB103490348AFF305
:10017000008008BD00000000CC070020541B0308CD
:1001800014214160704714207047406A7047000096
:1001900081010008870100088B010008A101000807
:1001A00010B5044604F1100000F05CFCC4F8F8003F
:1001B0000148C4F87C0110BD90010008F8B5E6B014
:1001C00004460D4616461F460A4906A800F0CAFE18
:1001D00070996F9A05910492009733466E996D9AC3
:1001E000039102922A466C990191214600F060F831
:1001F00067B0F0BD9C010008F8B5E6B004460D46B6
:1002000016461F46094906A800F0ACFE6F996E9A83
:100210000491039200976D996C9A02910192334672
:100220002A46214600F087F867B0F0BD9C0100081F
:1002300038B500281CBF01680029184A23D1184B83
:100240001C684FF6F0710C404CF24025AC421FBFC9
:100250001B6819404CF27024A14212D1114D29683B
:1002600079B911490B68C3F30B03B3F58A6F1FBF4C
:100270000968C1F30B0140F28343994204BF012195
:10028000117028B905E0094B994204BF0121117092
:100290004068BDE8324002F073BC00BFE4070020B4
:1002A00000ED00E0002004E00010005C0000374892
:1002B0002DE9F04104460D46216816464A681F465E
:1002C00090478046B8F5403F2ED122680A9993683E
:1002D000204698478046B8F5403F25D12368089AC4
:1002E0000799D3F80CC02046E0478046B8F5403F58
:1002F0001AD12368069A39461F692046B8478046B6
:10030000B8F5403F10D1236829465D693246204642
:10031000A8478046B8F5403F06D123680B9A099953
:100320009D692046A847804621680A682046904774
:100330004046BDE8F0812DE9F04104460D462168B4
:1003400016464A681F4690478046B8F5403F2ED172
:1003500022680A999368204698478046B8F5403F3E
:1003600025D12368089A0799D3F80CC02046E047A6
:100370008046B8F5403F1AD12368069A39461F696E
:100380002046B8478046B8F5403F10D1236829463B
:100390005D6932462046A8478046B8F5403F06D101
:1003A00023680999DD6900222046A8478046216814
:1003B0000A68204690474046BDE8F0814FF440303F
:1003C00070470000F0B50C4685B0114600281A466B
:1003D0001CBF0568002D0B4B11D082B104B971B957
:1003E0000D9860B10F9E0E9F0A9B02900496039792
:1003F0000B980C9E009001962046A847034618468D
:1004000005B0F0BD020003002DE9F04F0646D0B064
:100410000868F56DD6F860E0726EB76EF36E00BADC
:1004200000906C46486800BA60600DF1400888682A
:1004300000BAA060C86800BAE060086900BA20612C
:10044000486900BA6061886900BAA061C86900BAE9
:10045000E061086A00BA2062486A00BA6062886A8D
:1004600000BAA062C86A00BAE062086B00BA2063F2
:10047000486B00BA6063886B00BAA063C86B00BAAF
:10048000E063402058F80C1C58F820CC58F838ACE1
:100490008CEA010158F840CC8AEA01018CEA010992
:1004A0004FEAF979401E48F8049BEBD187EA020035
:1004B00000EA0E00784010EBF5610098DFF824C4E4
:1004C00041186144C81882EABE032B404FEAF0612C
:1004D00053405918636859186144CF194FEAB5035E
:1004E00083EABE01014081EABE0111EBF765A16814
:1004F0004D196544A91883EAB0023A404FEAF16504
:100500005A405519E26855194FEAB70282EAB00716
:1005100065440F4005EBBE0E97EAB00717EBFE658A
:1005200027697D194FEAB10782EA0701654401EAAC
:100530000E01EB18514011EBF36561694D194FEA5B
:10054000BE0187EA010E65440EEA030E15EBB0000A
:100550008EEA070E0EEBF065D4F818E0754465449A
:10056000AA1881EAB30505404FEAF26E4D40AE4449
:10057000E569AE44E64477444FEAB00080EAB30E42
:100580000EEA020E8EEAB30E0EEBF765D4F820E009
:1005900075446544691880EAB2053D404FEAF16E42
:1005A0004540AE44656AAE44E6440EEBB3034FEA01
:1005B000B70787EAB20E0EEA010E8EEAB20E0EEB14
:1005C000F365D4F828E075446544281887EAB10536
:1005D0001D404FEAF06E7D40AE44E56AAE44E6440D
:1005E0000EEBB2024FEAB30383EAB10E0EEA000E3D
:1005F0008EEAB10E0EEBF265D4F830E07544654436
:10060000EF1983EAB00515404FEAF76E5D40AE443E
:10061000656BAE44E6440EEBB1014FEAB20282EAEA
:10062000B00E0EEA070E8EEAB00E0EEBF165D4F8AE
:1006300038E075446544EB1882EAB7050D404FEA8F
:10064000F36E5540AE44E56BAE44E6440EEBB000AD
:100650004FEAB10181EAB70E0EEA030E8EEAB70E39
:100660000EEBF065D4F840E07544654481EAB30EC2
:10067000AA180EEA000E4FEAF2658EEA010E7544E2
:10068000DDF844E04FEAB000754480EAB30E6544FB
:100690000EEA020E15EBB7078EEAB30E0EEBF76506
:1006A000DDF848E04FEAB202754480EA020E654484
:1006B0000EEA070E69188EEA000E0EEBF165DDF802
:1006C0004CE07544654405EBB3034FEAB70E1427BD
:1006D0000DF1500CDFF810528EEA010B82EA0B0B81
:1006E0000BEBF36A5CF804BBDA44AA44504483EA97
:1006F000B10B4FEAF06A8EEA0B0BDA445CF804BBEC
:10070000DA44AA44524480EAB30B4FEAF26A8BEA15
:10071000B10BDA445CF804BBDA444FEAB000AA44F7
:1007200080EA020BD6448BEAB30B0BEBFE6A5CF853
:1007300004BBDA444FEAB202AA4482EA0E0B0AEB87
:10074000B10180EA0B0B0BEBF16A5CF804BBDA44F5
:100750007F1DAA44282F0AEBB3034FEABE0EBBD37A
:100760003C2F61D3502F4DD204EB870CC7F15407B7
:100770005E4CA7FB04A504465D4FA8088EEA010A5B
:1007800082EA0A0A5CF804BB0AEBF3655D447D1952
:100790002C1983EAB10A4FEAF4658EEA0A0A554435
:1007A0005CF804AB5CF804BB55447D19AA1884EAD4
:1007B000B30A4FEAF2658AEAB10A55445D444FEA4A
:1007C000B4047D1984EA020AAE448AEAB30A0AEB49
:1007D000FE655CF804AB55444FEAB2027D1982EA2B
:1007E0000E0A15EBB10184EA0A0A5CF804BB0AEBB5
:1007F000F1655D447D1915EBB303401E4FEABE0E53
:10080000BCD12046F46D1B19F365336EC9183166EF
:10081000716E71447166B36ED218B266F16E401893
:10082000F06650B0BDE8F08F4EEA010B0EEA010A07
:100830000BEA020B4BEA0A0A0AEBF36554F827A00D
:10084000DFF8B0C0554443EAB10B654403EAB10A8E
:100850000BEA0E0B28184BEA0A0A7F1C0AEBF0651C
:1008600054F827A0554440EAB30B654400EAB30AA4
:100870000BEAB10BAA184BEA0A0A7F1C0AEBF265D5
:1008800054F827A055444FEAB00040EA020B6544F3
:1008900000EA020A0BEAB30BAE444BEA0A0A7F1CD9
:1008A0000AEBFE6554F827A055444FEAB20242EA2B
:1008B0000E0B654402EA0E0A0BEA000B15EBB101C0
:1008C0004BEA0A0A7F1C0AEBF16554F827A055444D
:1008D0007F1C65443C2F05EBB3034FEABE0EA3D348
:1008E00040E700BF9979825AA1EBD96ECDCCCCCC30
:1008F000D6C162CADCBC1B8F00B581B00168074A53
:10090000914200D110B9064801B000BD7C212DF004
:10091000D2FE4FF4003001B000BD00BF040A000851
:10092000030002002DE9F0410B4A92E8F85188B02B
:10093000694681E8F8510268084B9A4200D118B91B
:10094000074808B0BDE8F0811422083000F04FFBE2
:1009500008B0BDE8F08100BFE4090008040A0008FF
:1009600003000200152904D20268044B9A4200D108
:1009700008B903487047083000F048BB040A000873
:100980000300020010B481B013460268074CA24273
:1009900000D118B901B010BC0548704701B000F192
:1009A000240210BC083000F035BB00BF040A000868
:1009B0000300020010B481B013460268074CA24243
:1009C00000D118B901B010BC054870470A4601B003
:1009D00000F1240110BC083000F070BB040A0008CC
:1009E000030002000123456789ABCDEFFEDCBA9816
:1009F00076543210F0E1D2C3000000000000000085
:100A000000000000F9080008250900086509000831
:100A100085090008B509000809040008810F0008CD
:100A2000CD0F0008890F0008F0B5A3B004460B48AD
:100A300002900D4616461F46094B0822402104A885
:100A400000F0D1FA28980190009733462A462146B3
:100A500002A800F01BF823B0F0BD00BF040A000894
:100A6000180A000810B5040008BF002408D0054883
:100A7000054B20600822402104F1080000F0B3FA81
:100A8000204610BD040A0008180A00082DE9F041AC
:100A900004460E46216817464A681D469047804620
:100AA000B8F5003F19D12268069993682046984707
:100AB0008046B8F5003F10D123683146DE683A46DB
:100AC0002046B0478046B8F5003F06D12368079A14
:100AD00029461D692046A847804621680A682046A5
:100AE00090474046BDE8F08110B500F033FA4FF46E
:100AF000403400280EBF034C4FF4C0712DF0DBFDD5
:100B0000204610BD0200030010B5044600F022FA92
:100B100008B9054810BD0021A160D0F87C211168FA
:100B200088474FF4403010BD0200030070B5044602
:100B30000D4600F00FFA064E40B1D0F87C01416836
:100B40008847A84224BF65604FF44036304670BDE8
:100B5000020003002DE9FF4715000C4600D02CB120
:100B6000064600F0F7F95FEA000801D16448C3E0E7
:100B7000D8F8F80001684A689047B0F5003F17D1EF
:100B8000D8F87C118A68404690478146B9F1810FB8
:100B900080F09E80A94508F1FC0A17D2D8F8F80029
:100BA0000368D3F80CC02A462146E047B0F5003F61
:100BB00040F08E80D8F8F8000368D3F810C06A4679
:100BC0005146E047B0F5003F76D10AE0002004E04E
:100BD000215C0AF800100098401C00900098A84280
:100BE000F6D34FF0000C4749474A484B01AC0098F8
:100BF000844558D2D3E9007001ADC5E90070107882
:100C000000281ABF042086464FF0000E085854F8FA
:100C10000E5028443E4D05600127D0F800E0876063
:100C2000019D4F681AF80C007D408EEA050585F09D
:100C3000040E65680F687D4085F0FC05754485F0FD
:100C4000A30568400AF80C000CF1010CCFE7D3E9CA
:100C5000004501A8C0E9004510782E4D002814BFBA
:100C60004FF0040E4FF0000E01A8744651F80EE04C
:100C70000459A6440127CEF80050DEF80040CEF813
:100C800008704D68019F40687D406C400D68684069
:100C900084F0040480F0FC00041984F057040AF87E
:100CA0000C400CF1010CCC45D1D3D8F8F800016808
:100CB0004A689047B0F5003F0AD1D8F8F8000368B9
:100CC000D3F80C804A465146C047B0F5003F01D0EA
:100CD000114811E0002006E05AF8201081F06A3136
:100CE0004AF82010401CB0EB990FF5D3B06840F0E3
:100CF0000100B0604FF4403004B0BDE8F08700BFA1
:100D0000020003008C5C0308E40700202C0F00089D
:100D1000ADBE4ED70DBE75A10100030038B50C461F
:100D2000017A1546CA0702D500F014F908B9084837
:100D300032BDD0F8F80003682146DC682A46A04797
:100D4000B0F5003F01D0034832BD4FF4403032BD12
:100D500002000300010003002DE9F84191B00546AF
:100D60000E461746402101A82DF0A5FC297AC80798
:100D700004D5284600F0EEF8040002D1DFF8A48084
:100D80004BE0D4F8F800DFF8A0800368D3F810C077
:100D90006A4601A9E047B0F5003F3ED1D4F8F8001B
:100DA00001684A689047B0F5003F36D1D4F87C110D
:100DB0008A6820469047D4F8F830024618461B68E7
:100DC000D3F80CC004F1FC01E047B0F5003F24D19A
:100DD000D4F87C0141688847D4F8F83002461846B8
:100DE0001B68D3F80CC001A9E047B0F5003F14D14F
:100DF000D4F8F8000268696893689847B0F5003F36
:100E00000BD1D4F8F80003681C693A463146A04774
:100E1000B0F5003F08BF4FF44038404612B0BDE87F
:100E2000F08100BF02000300010003002DE9F8413A
:100E3000A5B0074688461646402115A82DF03BFC74
:100E400000220492402105A82DF035FC387AC10714
:100E50005ED5384600F07EF8050059D0D5F8F80088
:100E60002D4C0368D3F810C06A4605A9E047B0F5D9
:100E7000003F3CD1D5F8F80001684A689047B0F5CA
:100E8000003F34D1D5F87C118A6828469047D5F8C0
:100E9000F830024618461B68D3F80CC005F1FC0177
:100EA000E047B0F5003F22D1D5F87C014168884782
:100EB000D5F8F830024618461B68D3F80CC005A9CF
:100EC000E047B0F5003F12D1D5F8F8000268796824
:100ED00093689847B0F5003F09D1D5F8F80003684A
:100EE0001D6904AA15A9A847B0F5003F01D0204606
:100EF0000FE00A4B0A490B4A0396029101924046C1
:100F00001C68049B009415AA796800F0E5F900E0DC
:100F1000054826B0BDE8F08101000300945C030899
:100F2000936E030026C703000200030004B0010112
:100F300000170145E90A0008090B00082D0B0008FD
:100F4000BD030008550B00081D0D0008590D0008D1
:100F50002D0E00080168024A914218BF0020704718
:100F6000340F000810B5040008BF002404D0034863
:100F70002060204609688847204610BD340F0008CD
:100F800020225C302DF093BBF0B58468A3080022CA
:100F900004F0030407E000F15C0555F8226035BA5F
:100FA00041F82250521C9A42F5D300220BE000F186
:100FB0005C0502EB830755F82360D500C5F11805E1
:100FC000EE40CE55521CA242F1D3F0BD30B5C468FC
:100FD00003690022E31AD5188C5C0544521C082AC8
:100FE0002C77F8D330BD0360C1600261704738B51B
:100FF000044615460022626023685A689047002024
:101000006061A061A5604FF4003032BD81604FF493
:10101000003070472DE9F84304462079D4F80C805D
:10102000450748BF244845D466691D46A8F101001C
:1010300000EAD60306EBC506B6EBC50F666102D221
:10104000A669761CA6611746A66906EB5576A661C9
:101050000E46E918884225D2A8EB03094A463146D4
:10106000F8182DF024FB2268136839460FE0424639
:1010700038462DF01CFB23681A68394620469047F5
:1010800007E0311811F00300F1D1226813682046FF
:101090009847484600EB0809A9F10101A942F0D39D
:1010A000002300E000202A1A3118F8182DF0FFFA6A
:1010B0004FF40030BDE8F283040002002DE9FC4F3C
:1010C000024685B0D0681369DFF86CC1DFF86C8127
:1010D000A0EB030A506840F004005060002703A80A
:1010E00002900DF10C0ED8E9003403A8544DC0E96C
:1010F00000342878534D00280CBF00230423994660
:101100005CF803305EF80940234401261D601C682A
:101110009E60DCF80430039DDCF80090DEF804608B
:101120005D406540484C654089EA0606474C66408C
:101130007519474C6540D8E9006B03AC0028C4E939
:10114000006B0EBF002404200424029E5CF8000003
:10115000345920183F4C04600126046886600398C7
:10116000029E43406340384C7068634089EA000047
:10117000364C6040034438484340280018BF0120E3
:101180005B1E9B41042F2CBFC0B2D80F02F1140389
:1011900053F8200007F00303C3F10303DB00D8403A
:1011A0000DF807007F1C082F9DD315460C466A6971
:1011B000AB69E868D20842EA4372401E00EA0207BF
:1011C000002302409B420AD8524508D28020E055B5
:1011D0007F1C574516D2AAEB0701E01910E08020CA
:1011E000E05500E0E355E8687F1C8742FAD32A689F
:1011F000136828469847BAF1000F03D0514620469D
:101200002DF059FA2A68069E059F9368694628467C
:1012100098472A68D2F8009021462846C8472B688C
:10122000DA683946284690470EB1A86830604FF416
:10123000003007B0BDE8F08F8C5C03085C1200083A
:10124000E40700205FC5109304850012FC68017A52
:10125000C0F524FF24AF33D426AF698B04B001015D
:1012600000170145F8B501240094002300240DE087
:10127000009D065D0F5D7E40F643761CF60F86F0FE
:10128000010635400095641C009DEB189442EFD395
:101290001846F2BDF8B5002301240094002A11E09D
:1012A000009C85188F1815F8016C17F8015C6E40CA
:1012B000F643761CF60F86F0010634400094009C3D
:1012C000E318521EECD11846F2BD0000651200086A
:1012D00095120008010000002DE9F84F1D46DDF8C9
:1012E00028900B9F0D9C4FF0FF3300930E469246C3
:1012F000D9F800B0804632465146D847834664B399
:10130000D9F8043032465146404698476FEA0B02FE
:10131000521C42EA0B0200996FEAD2735B1C19401F
:10132000C2430091521C024300996FEAD2735B1CC6
:101330001940009186F05531484087EA000181F05C
:101340005531216080F05531C943491C0843009A4A
:101350006FEAD070401C82430092D9F8080001283F
:1013600009D17540E943491C0D4300986FEAD572D5
:10137000521C90430AE0F11C85EA9102D243521CB0
:10138000154300986FEAD5735B1C984386F0AA3624
:10139000009086EA0B0686F0AA33F243DB430C98F2
:1013A000C2F3C0725B1C42EAD3720099D243521C52
:1013B00091430091774000998843009987F0AA37BC
:1013C0000F403843BDE8F28F00000000000000002D
:1013D00001F0FF01102A2BDB10F0070F08D010F8E6
:1013E000013B013A8B422DD010F0070F42B3F6D1EA
:1013F000F0B441EA012141EA014122F007047FF003
:1014000000070023F0E80256083C85EA010586EA59
:10141000010685FA47F5A3FA87F586FA47F6A5FA95
:1014200087F68EB9EED1F0BC01F0FF0102F00702A1
:1014300032B110F8013B013A83EA010313B1F8D14C
:101440000020704701387047002D06BF354603382D
:10145000073815F0010F07D1013015F4807F02BF66
:10146000013015F4C03F0130F0BC0138704700BFB7
:10147000034613F8012B002AFBD1181A01387047D4
:1014800081F0004102E000BF83F0004330B54FEA35
:1014900041044FEA430594EA050F08BF90EA020FA2
:1014A0001FBF54EA000C55EA020C7FEA645C7FEA35
:1014B000655C00F0E2804FEA5454D4EB5555B8BF58
:1014C0006D420CDD2C4480EA020281EA030382EAC9
:1014D000000083EA010180EA020281EA0303362D5B
:1014E00088BF30BD11F0004F4FEA01314FF4801C2E
:1014F0004CEA113102D0404261EB410113F0004F40
:101500004FEA03334CEA133302D0524263EB4303F6
:1015100094EA050F00F0A780A4F10104D5F1200E94
:101520000DDB02FA0EFC22FA05F2801841F10001EF
:1015300003FA0EF2801843FA05F359410EE0A5F1C3
:1015400020050EF1200E012A03FA0EFC28BF4CF0F4
:10155000020C43FA05F3C01851EBE37101F00045AA
:1015600007D54FF0000EDCF1000C7EEB00006EEBB7
:101570000101B1F5801F1BD3B1F5001F0CD3490841
:101580005FEA30004FEA3C0C04F101044FEA445298
:1015900012F5800F80F09A80BCF1004F08BF5FEA1F
:1015A000500C50F1000041EB045141EA050130BDFF
:1015B0005FEA4C0C404141EB0101013C28BFB1F511
:1015C000801FE9D291F0000F04BF01460020B1FA5C
:1015D00081F308BF2033A3F10B03B3F120020CDA2F
:1015E0000C3208DD02F1140CC2F10C0201FA0CF00D
:1015F00021FA02F10CE002F11402D8BFC2F1200C72
:1016000001FA02F120FA0CFCDCBF41EA0C01904027
:10161000E41AA2BF01EB0451294330BD6FEA040470
:101620001F3C1CDA0C340EDC04F11404C4F120025B
:1016300020FA04F001FA02F340EA030021FA04F36D
:1016400045EA030130BDC4F10C04C4F1200220FAC4
:1016500002F001FA04F340EA0300294630BD21FA02
:1016600004F0294630BD94F0000F83F4801306BFC8
:1016700081F480110134013D4EE77FEA645C18BFBC
:101680007FEA655C29D094EA050F08BF90EA020F53
:1016900005D054EA000C04BF1946104630BD91EA4B
:1016A000030F1EBF0021002030BD5FEA545C05D14E
:1016B0004000494128BF41F0004130BD14F580048D
:1016C0003CBF01F5801130BD01F0004545F0FE4101
:1016D00041F470014FF0000030BD7FEA645C1ABF36
:1016E000194610467FEA655C1CBF0B46024650EA6D
:1016F000013406BF52EA033591EA030F41F4002199
:1017000030BD00BF90F0000F04BF0021704730B51E
:101710004FF4806404F132044FF000054FF00001F3
:1017200050E700BF90F0000F04BF0021704730B5B4
:101730004FF4806404F1320410F0004548BF404289
:101740004FF000013EE700BF42004FEAE2014FEADE
:1017500031014FEA02701FBF12F07F4393F07F4FB9
:1017600081F06051704732F07F4208BF704793F0BC
:101770007F4F04BF41F40021704730B54FF46074CF
:1017800001F0004521F000411CE700BF50EA0102D2
:1017900008BF704730B54FF000050AE050EA01027B
:1017A00008BF704730B511F0004502D5404261EBEB
:1017B00041014FF4806404F132045FEA915C3FF42C
:1017C000D8AE4FF003025FEADC0C18BF03325FEAC9
:1017D000DC0C18BF033202EBDC02C2F1200300FA7A
:1017E00003FC20FA02F001FA03FE40EA0E0021FA9F
:1017F00002F11444BDE600BF70B54FF0FF0C4CF48D
:10180000E06C1CEA11541DBF1CEA135594EA0C0F3E
:1018100095EA0C0F00F0DEF82C4481EA030621EA79
:101820004C5123EA4C5350EA013518BF52EA0335B4
:1018300041F4801143F4801338D0A0FB02CE4FF066
:101840000005E1FB02E506F00042E0FB03E54FF096
:101850000006E1FB03569CF0000F18BF4EF0010E8E
:10186000A4F1FF04B6F5007F64F5407404D25FEA8A
:101870004E0E6D4146EB060642EAC62141EA55513D
:101880004FEAC52040EA5E504FEACE2EB4F1FD0C7F
:1018900088BFBCF5E06F1ED8BEF1004F08BF5FEAFD
:1018A000500E50F1000041EB045170BD06F00046AF
:1018B00046EA010140EA020081EA0301B4EB5C045C
:1018C000C2BFD4EB0C0541EA045170BD41F4801154
:1018D0004FF0000E013C00F3AB8014F1360FDEBF79
:1018E000002001F0004170BDC4F10004203C35DA55
:1018F0000C341BDC04F11404C4F1200500FA05F3D8
:1019000020FA04F001FA05F240EA020001F0004278
:1019100021F0004110EBD37021FA04F642EB0601EE
:101920005EEA430E08BF20EAD37070BDC4F10C0418
:10193000C4F1200500FA04F320FA05F001FA04F2DC
:1019400040EA020001F0004110EBD37041F10001C8
:101950005EEA430E08BF20EAD37070BDC4F12005D3
:1019600000FA05F24EEA020E20FA04F301FA05F23B
:1019700043EA020321FA04F001F0004121FA04F2E3
:1019800020EA020000EBD3705EEA430E08BF20EAB3
:10199000D37070BD94F0000F0FD101F000464000ED
:1019A00041EB010111F4801F08BF013CF7D041EA6F
:1019B000060195F0000F18BF704703F00046520073
:1019C00043EB030313F4801F08BF013DF7D043EA44
:1019D0000603704794EA0C0F0CEA135518BF95EAFA
:1019E0000C0F0CD050EA410618BF52EA4306D1D181
:1019F00081EA030101F000414FF0000070BD50EAA0
:101A0000410606BF1046194652EA430619D094EA29
:101A10000C0F02D150EA013613D195EA0C0F05D113
:101A200052EA03361CBF104619460AD181EA030167
:101A300001F0004141F0FE4141F470014FF000001F
:101A400070BD41F0FE4141F4780170BD70B54FF0BA
:101A5000FF0C4CF4E06C1CEA11541DBF1CEA13553A
:101A600094EA0C0F95EA0C0F00F0A7F8A4EB05041C
:101A700081EA030E52EA03354FEA013100F0888013
:101A80004FEA03334FF0805545EA131343EA1263DC
:101A90004FEA022245EA111545EA10654FEA002691
:101AA0000EF000419D4208BF964244F1FD0404F54A
:101AB000407402D25B084FEA3202B61A65EB0305A6
:101AC0005B084FEA32024FF480104FF4002CB6EB63
:101AD000020E75EB030E22BFB61A754640EA0C00E3
:101AE0005B084FEA3202B6EB020E75EB030E22BF23
:101AF000B61A754640EA5C005B084FEA3202B6EB64
:101B0000020E75EB030E22BFB61A754640EA9C0022
:101B10005B084FEA3202B6EB020E75EB030E22BFF2
:101B2000B61A754640EADC0055EA060E18D04FEAB0
:101B3000051545EA16754FEA06164FEAC30343EA50
:101B400052734FEAC2025FEA1C1CC0D111F4801F1D
:101B50000BD141EA00014FF000004FF0004CB6E716
:101B600011F4801F04BF01430020B4F1FD0C88BFB5
:101B7000BCF5E06F3FF6AFAEB5EB030C04BFB6EBC0
:101B8000020C5FEA500C50F1000041EB045170BDB3
:101B90000EF0004E4EEA113114EB5C04C2BFD4EBE0
:101BA0000C0541EA045170BD41F480114FF0000E64
:101BB000013C90E645EA060E8DE60CEA135594EAE0
:101BC0000C0F08BF95EA0C0F3FF43BAF94EA0C0FE3
:101BD0000AD150EA01347FF434AF95EA0C0F7FF458
:101BE00025AF104619462CE795EA0C0F06D152EAAC
:101BF00003353FF4FDAE1046194622E750EA410690
:101C000018BF52EA43067FF4C5AE50EA41047FF4A0
:101C10000DAF52EA43057FF4EBAE12E74FF0FF3C05
:101C200006E000BF4FF0010C02E000BF4FF0010CD6
:101C30004DF804CD4FEA410C7FEA6C5C4FEA430C4F
:101C400018BF7FEA6C5C1BD001B050EA410C0CBF9E
:101C500052EA430C91EA030F02BF90EA020F002000
:101C6000704710F1000F91EA030F58BF994208BF67
:101C700090422CBFD8176FEAE37040F00100704724
:101C80004FEA410C7FEA6C5C02D150EA013C07D17B
:101C90004FEA430C7FEA6C5CD6D152EA033CD3D0C6
:101CA0005DF8040B704700BF8446104662468C46C0
:101CB0001946634600E000BF01B5FFF7B7FF0028F3
:101CC00048BF10F1000F01BD4DF808EDFFF7F4FF1C
:101CD0000CBF012000205DF808FB00BF4DF808EDA7
:101CE000FFF7EAFF34BF012000205DF808FB00BFCA
:101CF0004DF808EDFFF7E0FF94BF012000205DF8EC
:101D000008FB00BF4DF808EDFFF7CEFF94BF0120A0
:101D100000205DF808FB00BF4DF808EDFFF7C4FF99
:101D200034BF012000205DF808FB00BF4FEA410CE2
:101D30007FEA6C5C02D150EA013C0AD14FEA430CC5
:101D40007FEA6C5C02D152EA033C02D14FF0000002
:101D500070474FF0010070474FEA410212F5001240
:101D600015D211D56FF47873B3EB625212D94FEAE2
:101D7000C12343F0004343EA505311F0004F23FACC
:101D800002F018BF404270474FF00000704750EA21
:101D9000013005D111F0004008BF6FF000407047DE
:101DA0004FF00000704700BF4FEA4102B2F1E0433C
:101DB00024BFB3F5001CDCF1FE5C0DD901F0004C32
:101DC0004FEAC0024CEA5070B2F1004F40EB830082
:101DD00008BF20F00100704711F0804F21D113F1AE
:101DE0003872BCBF01F00040704741F480114FEAE7
:101DF0005252C2F11802C2F1200C10FA0CF320FA70
:101E000002F018BF40F001004FEAC1234FEAD3238C
:101E100003FA0CFC40EA0C0023FA02F34FEA4303F6
:101E2000CCE77FEA625307D150EA01331EBF4FF07F
:101E3000FE4040F44000704701F0004040F0FE409A
:101E400040F40000704700BF80F0004002E000BF97
:101E500081F0004142001FBF5FEA410392EA030F95
:101E60007FEA226C7FEA236C6AD04FEA1262D2EBDF
:101E70001363C1BFD218414048404140B8BF5B42E4
:101E8000192B88BF704710F0004F40F4000020F07D
:101E90007F4018BF404211F0004F41F4000121F093
:101EA0007F4118BF494292EA030F3FD0A2F10102DD
:101EB00041FA03FC10EB0C00C3F1200301FA03F11B
:101EC00000F0004302D5494260EB4000B0F5000F3E
:101ED00013D3B0F1807F06D340084FEA310102F1FD
:101EE0000102FE2A51D2B1F1004F40EBC25008BFAF
:101EF00020F0010040EA03007047490040EB000079
:101F0000013A28BFB0F5000FEDD2B0FA80FCACF179
:101F1000080CB2EB0C0200FA0CF0AABF00EBC250A6
:101F200052421843BCBFD0401843704792F0000F94
:101F300081F4000106BF80F400000132013BB5E7E7
:101F40004FEA41037FEA226C18BF7FEA236C21D05D
:101F500092EA030F04D092F0000F08BF08467047C2
:101F600090EA010F1CBF0020704712F07F4F04D190
:101F7000400028BF40F00040704712F100723CBFA3
:101F800000F50000704700F0004343F0FE4040F4CD
:101F9000000070477FEA226216BF08467FEA23638B
:101FA0000146420206BF5FEA412390EA010F40F476
:101FB000800070474FF0000304E000BF10F00043C2
:101FC00048BF40425FEA000C08BF704743F09643A9
:101FD00001464FF000001CE050EA010208BF7047C4
:101FE0004FF000030AE000BF50EA010208BF70474B
:101FF00011F0004302D5404261EB41015FEA010C60
:1020000002BF84460146002043F0B64308BFA3F157
:102010008053A3F50003BCFA8CF2083AA3EBC25339
:1020200010DB01FA02FC634400FA02FCC2F1200258
:10203000BCF1004F20FA02F243EB020008BF20F08F
:102040000100704702F1200201FA02FCC2F12002F5
:1020500050EA4C0021FA02F243EB020008BF20EAEA
:10206000DC7070474FF0FF0C1CEAD0521EBF1CEA18
:10207000D15392EA0C0F93EA0C0F6FD01A4480EA06
:10208000010C400218BF5FEA41211ED04FF00063EF
:1020900043EA501043EA5111A0FB01310CF000401B
:1020A000B1F5000F3EBF490041EAD3715B0040EA41
:1020B000010062F17F02FD2A1DD8B3F1004F40EB11
:1020C000C25008BF20F00100704790F0000F0CF0E4
:1020D000004C08BF49024CEA502040EA51207F3AA8
:1020E000C2BFD2F1FF0340EAC250704740F4000083
:1020F0004FF00003013A5DDC12F1190FDCBF00F074
:1021000000407047C2F10002410021FA02F1C2F121
:10211000200200FA02FC5FEA310040F1000053EABD
:102120004C0308BF20EADC70704792F0000F00F00B
:10213000004C02BF400010F4000F013AF9D040EA11
:102140000C0093F0000F01F0004C02BF490011F4A5
:10215000000F013BF9D041EA0C018FE70CEAD153A3
:1021600092EA0C0F18BF93EA0C0F0AD030F0004C23
:1021700018BF31F0004CD8D180EA010000F00040D7
:10218000704790F0000F17BF90F0004F084691F095
:10219000000F91F0004F14D092EA0C0F01D14202CF
:1021A0000FD193EA0C0F03D14B0218BF084608D198
:1021B00080EA010000F0004040F0FE4040F40000E2
:1021C000704740F0FE4040F4400070474FF0FF0C75
:1021D0001CEAD0521EBF1CEAD15392EA0C0F93EABC
:1021E0000C0F69D0A2EB030280EA010C49024FEA0E
:1021F000402037D04FF0805343EA111143EA1013C7
:102200000CF000408B4238BF5B0042F17D024FF47E
:10221000000C8B4224BF5B1A40EA0C00B3EB510F59
:1022200024BFA3EB510340EA5C00B3EB910F24BF42
:10223000A3EB910340EA9C00B3EBD10F24BFA3EBC7
:10224000D10340EADC001B0118BF5FEA1C1CE0D18F
:10225000FD2A3FF650AF8B4240EBC25008BF20F042
:10226000010070470CF0004C4CEA50207F32C2BF96
:10227000D2F1FF0340EAC250704740F400004FF033
:102280000003013A37E792F0000F00F0004C02BF64
:10229000400010F4000F013AF9D040EA0C0093F02E
:1022A000000F01F0004C02BF490011F4000F013B88
:1022B000F9D041EA0C0195E70CEAD15392EA0C0FF0
:1022C00008D142027FF47DAF93EA0C0F7FF470AF28
:1022D000084676E793EA0C0F04D14B023FF44CAF6B
:1022E00008466EE730F0004C18BF31F0004CCAD100
:1022F00030F000427FF45CAF31F000437FF43CAF3C
:102300005FE700BF4FF0FF3C06E000BF4FF0010C5D
:1023100002E000BF4FF0010C4DF804CD4FEA40023F
:102320004FEA41037FEA226C18BF7FEA236C11D089
:1023300001B052EA530C18BF90EA010F58BFB2EB3C
:10234000030088BFC81738BF6FEAE17018BF40F0BC
:10235000010070477FEA226C02D15FEA402C05D170
:102360007FEA236CE4D15FEA412CE1D05DF8040BF5
:10237000704700BF844608466146FFE70FB5FFF788
:10238000C9FF002848BF10F1000F0FBD4DF808ED40
:10239000FFF7F4FF0CBF012000205DF808FB00BF31
:1023A0004DF808EDFFF7EAFF34BF012000205DF88B
:1023B00008FB00BF4DF808EDFFF7E0FF94BF0120D8
:1023C00000205DF808FB00BF4DF808EDFFF7D2FFD5
:1023D00094BF012000205DF808FB00BF4DF808ED18
:1023E000FFF7C8FF34BF012000205DF808FB00BFE5
:1023F0004FEA40024FEA41037FEA226C02D15FEAD2
:10240000402C08D17FEA236C02D15FEA412C02D133
:102410004FF0000070474FF0010070474FEA400254
:10242000B2F1FE4F0FD34FF09E03B3EB12620DD902
:102430004FEA002343F0004310F0004F23FA02F06C
:1024400018BF404270474FF00000704712F1610F13
:1024500001D1420205D110F0004008BF6FF00040EA
:1024600070474FF00000704742000ED2B2F1FE4FAD
:102470000BD34FF09E03B3EB126209D44FEA002353
:1024800043F0004323FA02F070474FF0000070471A
:1024900012F1610F01D1420202D14FF0FF307047BB
:1024A0004FF00000704700BF53B94AB9002908BF78
:1024B00000281CBF4FF0FF314FF0FF3000F06AB929
:1024C000ADF1080C6DE904CE00F006F8DDF804E08B
:1024D000DDE9022304B070472DE9F047089D0C4662
:1024E000002B4ED194468C458646B2FA82F262D9D0
:1024F0004AB1C2F12003914020FA03F30CFA02FC26
:10250000194300FA02FE4FEA1C471FFA8CF6B1FB92
:10251000F7F44FEA1E4307FB141143EA014304FB9F
:1025200006F199420AD91CEB030304F1FF3080F055
:102530001281994240F20F81023C6344591A1FFAFA
:102540008EF3B1FBF7F007FB101143EA014300FBE8
:1025500006F69E420AD91CEB030300F1FF3180F01E
:10256000FC809E4240F2F980634402389B1B40EAA3
:10257000044000211DB1D3400022C5E90032BDE86E
:10258000F0878B4205D90DB1C5E90001002108464D
:10259000F5E7B3FA83F1002946D1A34202D3904272
:1025A000C0F0F080861A64EB03030120002DE6D012
:1025B000C5E90063E3E7002A40F09080A1EB0C043A
:1025C0004FEA1C481FFA8CF70121B4FBF8F64FEADA
:1025D0001E4308FB164443EA044307FB06F09842F7
:1025E00008D91CEB030306F1FF3402D2984200F233
:1025F000CD8026461C1A1FFA8EF3B4FBF8F008FBB8
:10260000104443EA044300FB07F79F4208D91CEB40
:10261000030300F1FF3402D29F4200F2B080204653
:10262000DB1B40EA0640A5E7C1F120068B4022FAF9
:1026300006F71F4320FA06FC04FA01F343EA0C03F1
:10264000F44000FA01F8380C4FEA1349B4FBF0FEED
:102650001FFA87FC00FB1E4449EA04440EFB0CF9F8
:10266000A14502FA01F20AD93C190EF1FF3A80F0B5
:102670008480A14540F28180AEF1020E3C44A4EB7F
:1026800009041FFA83F9B4FBF0F300FB134449EA91
:10269000044403FB0CFCA44507D93C1903F1FF30AB
:1026A00067D2A44565D9023B3C4443EA0E40A0FBF7
:1026B0000293A4EB0C049C42CE469C4651D34ED0D0
:1026C00055B1B8EB0E0364EB0C0404FA06F6CB40EC
:1026D0001E43CC40C5E90064002150E7C2F120034D
:1026E00020FA03F10CFA02FC24FA03F394400C43A1
:1026F0004FEA1C4800FA02FE1FFA8CF7B3FBF8F011
:1027000008FB1031230C43EA014300FB07F1994217
:1027100008D91CEB030300F1FF362CD299422AD9C9
:10272000023863445B1AA4B2B3FBF8F108FB11331F
:1027300044EA034401FB07F3A34208D91CEB040459
:1027400001F1FF3613D2A34211D902396444E41ACD
:1027500041EA004139E70446F0E6084606E7C84585
:10276000AED2B9EB020E63EB070C0138A8E7314695
:10277000EDE7034699E73046D4E7D6467FE7634462
:1027800002384DE70646234608460FE7023E6344FB
:1027900030E700BF704700BF00487047001BB74BD1
:1027A00070B50C4601F06EFA104E05460821304611
:1027B00005F0F6FF012804D001F064FA431BA342A0
:1027C00007D30821094805F0EBFF431E5842584142
:1027D00070BD72B60821304605F0E2FF012800D036
:1027E00030BF62B6BFF36F8FE0E700BF0004004860
:1027F00008B5002210214FF0904005F0D7FF0548A2
:102800000022202105F0D2FFBDE80840022001F09F
:1028100041BA00BF0004004810B50C4C0122102141
:10282000204605F0C3FF052001F034FA20460122BE
:10283000202105F0BBFF4FF090400122102105F050
:10284000B5FFBDE81040022001F024BA00040048A2
:1028500070B54FF090400C46164610210022144DE2
:1028600005F0A4FF00232B701248B3B22246214684
:1028700007F090F9D8B901F005FA41F2873604461D
:102880002B783BB1BDE87040012210214FF0904001
:1028900005F08CBF01F0F6F9031BB342F2D872B613
:1028A0002B7803B930BF62B6BFF36F8FE8E770BD16
:1028B000E507002048090020014B01221A707047EB
:1028C000E507002000487047985C030813B5114BDA
:1028D0000446186800909B88ADF804300120FFF78B
:1028E0009BFF062269460120FFF7B2FF0120FFF798
:1028F0007FFF9DF80430112B08D19DF80520122A86
:1029000004D101202370627002B010BD00231A466A
:102910001846F7E7701B03080CB4F0B5ADB032AB46
:1029200006AF53F8042B059305460E46384696210C
:102930002BF010FE9528C1BF42F62E63ADF8AA30E9
:102940002E23ADF8AC3000F037F83C24042D4FF4C2
:102950007A7E1449B0FBFEFCB0FBF1F14EF6602329
:10296000B0FBF3F3B3FBF4F204FB1232BCFBF4F361
:1029700004FB13C30EFB1C049ABF0B48405D3F20B1
:10298000CDE90040CDE9026708482BF063FD084B14
:102990001B6898682BF088FC2DB0BDE8F04002B0B1
:1029A000704700BF80EE3600F65C0308D45C030875
:1029B000F405002001F06EB901F064B91348144A1F
:1029C00008B54FF00043C0E9002304224261012210
:1029D0000023C2614FF480510722C0E90233C0E9ED
:1029E0000933C0E90C1203610383837680F8203039
:1029F00080F82C30826380F83C30C36404F028FEF9
:102A000018B1BDE8084000F099BB08BDE8070020F8
:102A1000002401400268084B9A4282B00AD14FF06C
:102A2000B0431A6E42F400721A661B6E03F4007310
:102A30000193019B02B07047002401400268054BDE
:102A40009A4201BF4FF0B042136E23F40073136635
:102A5000704700BF0024014030B585B00024054612
:102A6000CDE901440394FFF7A9FF144805F084F968
:102A700008B100F063FB1148039401A9CDE90154AA
:102A800004F044FF08B100F059FB0C4805F09EF833
:102A900008B100F053FB4FF0FF31084804F0D8FEB6
:102AA000064805F04BF9054804F02CFF044603489E
:102AB00005F0EEF8204605B030BD00BFE807002065
:102AC000014B024A1A607047E807002000240140C9
:102AD00008B50948FFF7C0FF68B1084BB3F8AA3042
:102AE0004FF6FF72934216BF40F6E442044B534345
:102AF000B3FBF0F398B208BD002000B40075FF1FCF
:102B0000D8084C0013B50023ADF80630FFF7E0FFFE
:102B100004461948FFF7A0FF184BB3F8C820B3F8D4
:102B2000A8108A4204FB00F018D040F6E443B0FB42
:102B3000F3F364205B1A4343521A93FBF2F31E3300
:102B40001BB2ADF80630BDF806305BB21B02ADF823
:102B50000630BDF8060000B202B010BD4FF47A7224
:102B600040F6FF73B0FBF3F35343A3F53923A3F50A
:102B70000C6340F6C412E0E7001000B00075FF1FC0
:102B80004FF0B04382B09A6A22F480529A629A6CF3
:102B900042F480529A649B6C03F480530193019B2E
:102BA000002002B070474FF0B04307B59A6C42F076
:102BB00004029A649A6C02F004020192019A9A6CDF
:102BC00042F001029A649B6C002203F0010311465B
:102BD00000930B20009B05F06DF90B2005F09CF98C
:102BE000002211460C2005F065F90C2005F094F93F
:102BF000002211460D2005F05DF90D2005F08CF93D
:102C0000002202210F2005F055F90F2005F084F96C
:102C100000221146102005F04DF9102005F07CF936
:102C200000221146112005F045F9112003B05DF88E
:102C300004EB05F071B9000008B505F0B1FB10B167
:102C40006FF0040008BD064B9A6942F040429A6159
:102C50004CF2FA321A6105F0B5FB0028F2D0EFE72A
:102C600000400058F0B585B000230D46009306469D
:102C7000A8B3FFF7E1FF044670BB05F091FB88BBEA
:102C80001A481B4A02230193D0F8E01506F1784355
:102C900002EA8121B3FBF1F701FB1733DB0A029350
:102CA000D0F8E00505F178410139314402EA80228B
:102CB000B1FBF2F002FB1011C3EBD12301336946E3
:102CC00001A8039305F0FEFB20B1022814BF6FF0AA
:102CD0000104012405F076FB204605B0F0BD6FF03D
:102CE0000504F9E76FF00404F6E700BF0070FF1F6A
:102CF00000FCFF03014B1860002070474C080020C7
:102D00002DE9F04FB0F1006F89B006460F469046AE
:102D1000C0F0C080DFF89091644DD9F8E03505EA45
:102D2000832303F10063013B984200F2B380002942
:102D300000F0B38040EA02035B0740F0AE80FFF78B
:102D40007BFF044690BB05F02BFB002840F0A880D9
:102D5000D9F8E015009705EA812106F17842B2FB27
:102D6000F1F301FB132208F17843013B3344B3FB39
:102D7000F1F001FB1033DB0A01334FEAD22AA3EB57
:102D8000D222012A039388BFC6F30A050AF58037C9
:102D9000C6F108038CBFC5F500654546FF02B34682
:102DA0000693039B9A4505D305F00CFB204609B01A
:102DB000BDE8F08FA6F10803069A1A4495421CD884
:102DC000009B04950193CDF814B04FF00009059BCA
:102DD00009EB0301049B99453DD3009BAB442B4475
:102DE000A8EB0505B5F5006F009328BF4FF400650B
:102DF0000AF1010A07F50067D3E753F8081F5A687C
:102E0000B2F1FF3F08BFB1F1FF3FD5D0284B1868A2
:102E100010B96FF00504C7E727B14FF400623946D7
:102E200011F05CFEDFF888900099D9F80030CBF300
:102E30000A001844AAB211F051FE4FF4006138465E
:102E4000FFF710FF00BBD9F8003001934FF4006387
:102E500005970493B9E7019B07914B440293012026
:102E6000D3E9002305F0E8FA88B90799019BD1E975
:102E7000000259F80310029B5B689A4208BF88421F
:102E800005D109F10809A2E76FF001048CE76FF0A2
:102E9000030489E74FF0FF3488E76FF0050485E706
:102EA0006FF0040482E700BF0070FF1F00FCFF0307
:102EB0004C080020B1F1006F70B510D30B4BD3F864
:102EC000E0650B4B03EA862303F10063013B994263
:102ED00005D838B192B211F001FE002070BD4FF05C
:102EE000FF30FBE76FF00500F8E700BF0070FF1F41
:102EF00000FCFF03B0F1006F10B40DD3084BD3F802
:102F0000E045084B03EA842303F10063013B984248
:102F100002D810BCFFF7A6BE4FF0FF3010BC7047C0
:102F20000070FF1F00FCFF034FF0B04382B0DA6C6B
:102F30000243DA64DB6C03400193019B02B07047EB
:102F40002DE9F04186B01422002101A82BF020FBCE
:102F50000220464EFFF7E8FF0420FFF7E5FF0120BF
:102F6000FFF7E2FF04213046002205F01FFC00229B
:102F700010214FF0904005F019FC04230024012596
:102F800002270DEB03013046CDE901354FF0100863
:102F9000CDE9034705F0E4FA01A93046CDE9018502
:102FA000CDE9037405F0DCFA202301A93046CDE910
:102FB0000135CDE9037405F0D3FA01A94FF0904033
:102FC000CDE90185CDE9034405F0CAFA08224FF4A2
:102FD000881301A93046CDE901234FF00308CDE95C
:102FE000034705F0BDFA4FF4441301A94FF0904098
:102FF000CDE90183CDE9035705F0B2FA4FF4405310
:1030000001A93046CDE90135CDE9034805F0A8FA1C
:103010004FF404134021CDE901131548039501A98C
:1030200005F09EFA22460F21062004F043FF0620F9
:1030300004F072FF22460F21072004F03BFF072017
:1030400004F06AFF22462146092004F033FF0920DC
:1030500004F062FF22462146092004F02BFF0920DC
:1030600004F05AFF06B0BDE8F08100BF000400483C
:103070000008004800B59BB04822002108A82BF0AA
:1030800087FA1822002102A82BF082FA05F0A8FB8B
:103090004FF0B0420120D2F8903023F01803C2F86C
:1030A0009030D2F8003423F4C06343F40073C2F8C4
:1030B0000034D2F8003403F4C0630193019B24234D
:1030C000089381230B930023CDE91003B02208A8B5
:1030D000CDE9122305F0FCFC08B172B6FEE74F23E0
:1030E000CDE90230CDE90400CDE90600022102A8B5
:1030F00005F088FF08B172B6FEE71BB05DF804FB6F
:1031000008B504F053FAFFF7B5FFFFF719FFFFF713
:103110004AFD01F03FF800F0EFFE00F089F80648A4
:103120000122042105F042FB02F070FC00F078FC63
:1031300002F073FCFCE700BF0004004872B6FEE733
:1031400000B58DB02C22002101A82BF021FA1748E0
:10315000174B03601F2383604FF080420023C0E9B8
:103160000433C0E9072383614FF48073436206F0A0
:10317000EFF908B1FFF7E2FF0C4806F015FB08B1C4
:10318000FFF7DCFF4FF00053002207930748089237
:103190004FF4807301A9029206920B9306F038FA5D
:1031A00008B1FFF7CBFF0DB05DF804FB500800201D
:1031B0000028004010B5044690B03822002102A833
:1031C0002BF0E6F92268194B9A422CD14FF4803348
:1031D000029302A84FF480730F9306F037F808B1FA
:1031E000FFF7ACFF4FF0B0430220D3F8902042F439
:1031F0000042C3F890209A6D42F480629A659B6DFC
:10320000002203F4806311460193019B04F052FEF7
:10321000022004F081FE00222A20114604F04AFE1A
:103220002A2004F079FE10B010BD00BF0028004035
:103230001148124A08B54FF48273C0E900230023F5
:103240004FF4E062C0E902324FF400712822C0E975
:1032500006120722C0E90433C0E90833C0E90B2392
:1032600083620823436306F00FFC18B1BDE80840F1
:10327000FFF764BF08BD00BF4809002000300140CF
:10328000F0B5054689B01422002103A82BF080F97F
:103290002A68374B9A4269D14FF0B04302261A6E22
:1032A00042F480521A661A6E02F480520292029A16
:1032B000DA6C42F00102DA64DA6C02F00102019287
:1032C000019ADA6C42F00202DA64DB6C03F002036A
:1032D00000930524009B0327D02303A94FF09040BF
:1032E000CDE90336CDE9067405F03AF92023CDE99E
:1032F00003364FF09040002603A90794CDE90567F7
:103300001C4C05F02DF91C4826620723C4E9000374
:1033100080232046C4E90266C4E90436C4E906668F
:1033200004F05AFE08B1FFF709FF144AAC65A56224
:10333000134C0823C4E900231021002380222046D7
:10334000C4E90213C4E90423C4E90633236204F088
:1033500043FE08B1FFF7F2FE002222206C65114601
:10336000A56204F0A7FD222004F0D6FD09B0F0BD4F
:1033700000300140E80800201C00024030000240FC
:10338000880800207047000008B504F025F9044BB8
:103390000120C3F88800BDE8084005F079BA00BFF5
:1033A0000004005808B504F01EF901F003F8FFF717
:1033B000C7FDFFF7F8FB00F09FFDBDE80840FFF7F1
:1033C00037BF08B504F00FF9FFF7BAFDFFF7EBFBC5
:1033D000BDE80840FFF72CBF08B504F0FDF8BDE8D4
:1033E00008400121002005F003BA70477047FEE74E
:1033F000FEE7FEE7FEE7FEE770477047704770475D
:10340000014806F0F7B900BF50080020024B012028
:10341000187005F0D9B900BF0A190020024B01222B
:1034200002201A7005F0D0B909190020082005F013
:10343000CBB90000014804F045BF00BFB40D002027
:10344000014804F03FBF00BFE8080020014804F035
:1034500039BF00BF8808002070470000014804F011
:1034600031BF00BF680E002070470000014806F021
:103470007FBD00BF48090020014807F037BF00BFEB
:10348000C80E0020014805F0E9BF00BF5008002029
:10349000014806F0FEBF00BFA00D00202DE9F0435B
:1034A00089B080460020109E0790894615461F4629
:1034B000FCF7BEFEF0B9104CCDE90090CDE9020456
:1034C00007AB0E480593142304933A464346294616
:1034D0000068FCF777FF2346324604F1140153F8E5
:1034E000044B42F8044B8B42F9D1079B337509B06A
:1034F000BDE8F0830120FAE7C2090020885C0308D8
:103500007FB5124C00253C2302A86375CDE9025516
:10351000257500F061FB042303AA009412210C48D6
:10352000FFF7BCFF0B49142220462BF021F806467A
:10353000B0FA80F040096075074B00902A46294692
:10354000022011F0C5F9304604B070BDAC0900206E
:10355000325D03088D1B0020145D030810B5074C75
:10356000074A0021204640F24B2307F035FD204654
:103570000021BDE8104007F041BC00BF140E002040
:10358000D6090020132BF0B52DD81825102415FBD3
:103590000343194D00244FF0800C4CFA04F6A3F1BC
:1035A0001007314205EB470714BF4FF0240E4FF0D0
:1035B000140EA7F806E0A3F10807304205EB470711
:1035C00014BF4FF0240E4FF0140E0134324205EBBD
:1035D0004306A7F806E00CBF14272427082CF78021
:1035E00003F10103D9D1054B1B781BB9BDE8F040AD
:1035F000FFF7B4BFF0BD00BFD6090020501900206E
:1036000010B500240022E3B2114610460134FFF742
:10361000B9FF142CF6D1BDE81040FFF79FBF0000A2
:10362000F8B504460D46FFF7EBFF0F4F002604EBFD
:1036300044040A2000F02EFB142E03D1BDE8F8400C
:10364000FFF78CBF3B19385D9A78597812FB05F269
:1036500011FB05F110FB05F0F3B2D2B2C9B2C0B252
:10366000FFF790FF0136E4E7070000202DE9F04165
:103670000646012090460F4600F00CFB1C4A102520
:103680004FF0800C2B4600244CFA04F1A3F11000FB
:103690000F4202EB400014BF4FF0240E4FF0140E07
:1036A000A0F806E0A3F108000E4202EB400014BFB0
:1036B0004FF0240E4FF0140E013418EA010F02EB04
:1036C0004301A0F806E00CBF14202420082CC88079
:1036D00003F10103D8D11835B5F5F87FD2D1054BE8
:1036E0001B781BB9BDE8F041FFF738BFBDE8F0819A
:1036F000D60900205019002003460846072B1CD885
:10370000DFE803F004070A0E12141719002211460D
:1037100000E00022104601E000221146FFF7A6BF9C
:103720000A4600210020F9E70022F7E70A460021B7
:10373000F0E70A46F6E70A46E9E77047024B1878D1
:10374000024B1978FFF7D8BF0500002000000020C9
:103750007FB502AC204611F01DFB94E80300824CBB
:10376000824D2378012B85E8030009D080490B782E
:1037700033B1804A13781BB17F4B1878052823D1C9
:103780007E4B1A686AB9296819607D491868086013
:103790007C490A601B68009311467B4B032011F0A3
:1037A00097F87A487A4D0378DBB20A2B32D8DFE8F3
:1037B00013F02C004D005100570060009700AA0044
:1037C000B600C300C300C3002078012806D10978E1
:1037D00021B9127812B91B78052BE2D0694B1A680F
:1037E000002ADED1296819606A49186808606349AF
:1037F0000A6018681B6809685B1ACDE90003114666
:10380000654B032011F064F8CBE7644B1B78DBB207
:10381000634A13700378634E012B06D0624C227802
:1038200002F0FF03002A00F08C805D4A0023137031
:103830002B703370FFF7E4FE5C4A002313705C4A80
:1038400013705C4B01221A7004B070BD544B0022FF
:103850001A70DFE7584A1278012A08BF0123D7E718
:10386000237813B94E4B0122F2E72378012BD1D1F3
:1038700046E0444B414A1B6812689B1A042BC9D985
:1038800023783C4A53B93A4B1B78012B06D1137865
:10389000012BD9B202D1424B1970BBE72378012B1F
:1038A00005D0334B1B7813B11378002BB2D13C4BAE
:1038B0000221197041490C78032C03D1042129708D
:1038C000197008E00C78012C01D10821F7E70C7879
:1038D000022CE1B2F3D01278002A9BD10822B7E77C
:1038E000237833B9344B1B78012BDAB201D12C4B3E
:1038F000AEE72378012B03D02F4B1B78002B89D107
:10390000274B0222A4E723781BB92D4B1B78002BF1
:10391000A8D02378012BF3D0294B1B78A6E7237876
:103920001BB9154B1B78042B9CD02378012BE7D0B7
:10393000114B1B78052B9AE70F4B1A78042AF8D104
:1039400090E7227812B9164B1B78DBB22B701D4B17
:1039500028781978FFF7D0FE237803B12B782B78DD
:10396000DBB2337068E700BFEB180020F0180020CE
:103970000A01002009010020E91800200419002094
:10398000FC18002000190020445D030806010020F7
:1039900005000020F8180020675D030804000020DF
:1039A000060000200100002050190020EE18002021
:1039B000ED180020481900208C1B0020720F0020F9
:1039C000EA18002000000020024803680021596323
:1039D00007F07CBB140E0020002270B50E4B114680
:1039E000022010F075FF01240A25294620461435CF
:1039F000FFF782FEEDB2322000F04CF96E2DF4D1CB
:103A00000134E4B2092CEFD10022BDE87040034B31
:103A10001146022010F05CBF9E5D0308D15D0308D3
:103A2000002210B51146164B022010F051FFFFF78F
:103A3000D3FF0022134B1146032010F049FF01244D
:103A4000204601341421E4B2FFF7EAFD082CF7D137
:103A5000FFF7D6FD00220C4B1146022010F038FF74
:103A60000A4B1B78012B05D1FFF7CAFDBDE81040BA
:103A7000FFF7C6BD14210120FFF73EFEF6E700BFA9
:103A8000075E0308325E03084C5E0308060100204F
:103A9000054808B50823036006F018FB18B1BDE817
:103AA0000840FFF74BBB08BDA00D00204FF0B0430E
:103AB00007B55A6E42F001025A665B6E002203F0AF
:103AC0000103019311463220019B04F0F3F93220E7
:103AD00003B05DF804EB04F01FBA00000CB407B5A6
:103AE000054A05AB1021019311F002FB03B05DF80C
:103AF00004EB02B0704700BF855E030830B585B0A7
:103B0000044602A80D4611F01FF9BDF90C30064A13
:103B100000931021029B2046FFF7E0FF2046FDF7AF
:103B2000A7FC288005B030BD855E03084FF0B04289
:103B300010B5936823F40043936011F08DF9104B96
:103B400001241C7000F0ACF810F058FE0D4810F085
:103B50006FFE0D4B4FF400421A61022010F06EFE12
:103B6000FEF7AEFF00F002F910F062FF214620469A
:103B700010F07EFF21462046BDE8104010F062BFE5
:103B8000AC0D0020FD3A00080040005810F086BF40
:103B900008B5FEF79DFF40F6B83398420CD8B0F553
:103BA000E16F0BD3FE23A0F5E16058434FF4966319
:103BB000B0FBF3F0C0B208BDFE20FCE70020FAE73E
:103BC0007FB5684600F0B6F80198FEF727FC00B212
:103BD00007B05DF804FB0000194A38B5D2F880350B
:103BE000591C044619D103F005FD054603F00EFDEE
:103BF000054403F005FD2B0EE3712B0CA3712B0A7A
:103C00006371030EE370C0F30742C0F3072325710D
:103C1000C0B2A2706370207038BD190AC37181717F
:103C2000190C1B0E41710371D2F88435C370D2F8A0
:103C30008405C0F30722C0F30743000EE9E700BF85
:103C40000070FF1F38B5094BD3F88035036001338E
:103C5000054609D103F0CEFC044603F0D1FC4440F4
:103C600003F0D4FC44402C6038BD00BF0070FF1F3F
:103C70000121022010F0E6BE0021022010F0E2BE79
:103C800000207047024B187808B100F0BFB97047A8
:103C9000AC0D002082B00190019802B000F052BA41
:103CA000F0B5224A224CD2F8903043F4804389B0D8
:103CB000C2F8903003F0B0FC03F0B6FC03F0BCFC9B
:103CC000012304930323069300254FF0B043059589
:103CD0000795DA6C42F00202DA64DA6C02F0020252
:103CE0000292029ADA6C42F00202DA64DB6C03F0B0
:103CF000020301934FF4805703A92046019B0397C9
:103D00004FF4005604F02CFC03A92046039604F05F
:103D100027FC2A463946204604F048FD2A4631460B
:103D2000204604F043FD09B0F0BD00BF0008005874
:103D30000004004810B50446FEF7E4FE074BA360FC
:103D400040F30F20FEF73AF9054B064A2360064B75
:103D50006060C4E90323002010BD00BF000048429A
:103D600000007A440D093E00AB03050000207047B7
:103D70000120704708B52AF06DFC162303604FF050
:103D8000FF3008BD08B52AF065FC16230360FEE786
:103D900070B50D4614460E46731B9C4201DC20464E
:103DA00070BDAFF3008006F8010BF5E730B51046A3
:103DB00000234FF06042834200DB30BDD2F8804EDA
:103DC000E50707D5D2F8004EE40703D5CC5C1568AB
:103DD00015B114700133EEE700BFF8E74FF0FF3084
:103DE00070474FF400534B6000207047012070472C
:103DF000002070470B4A116810B5034609B90A49FB
:103E00001160106809490A4C0344091B8B4206D90A
:103E10002AF020FC0C2303604FF0FF3010BD13602C
:103E2000FCE700BFB00D0020403B00200000012057
:103E30000008000037B5184B02689A42054628D1A1
:103E40004FF0B043154C1A6E42F400621A661B6EB6
:103E5000134A03F400630193019B1723C4E9002371
:103E6000102100238020C4E902134FF48073C4E9B9
:103E700004034FF4806C2023C4E906C320464FF4AA
:103E80000053236204F0A8F808B1FFF757F96C62F9
:103E9000A56203B030BD00BF002C0140B40D00206E
:103EA0000800024010B5044686B01422002101A883
:103EB0002AF06EFB22680F4B9A4218D14FF0B043A4
:103EC00001A9DA6C42F00102DA64DB6C03F0010351
:103ED00000930222009B4FF48073CDE901324FF032
:103EE00090400123CDE90332059304F039FB06B07D
:103EF00010BD00BF002C014010B58EB01022002173
:103F000003A82AF045FB00241C2221460DEB0200E9
:103F1000CDE9004402942AF03BFB1F481F4B84600C
:103F2000C0E900343B23C0E90334C0E9054406F08E
:103F300019FD08B1FFF702F94FF4805316480393B7
:103F400003A906F02DFE08B1FFF7F8F8124806F0B5
:103F500039FD08B1FFF7F2F800240F4802946946D2
:103F6000CDE9004407F0B4F808B1FFF7E7F86023A3
:103F700009480D94002207A9CDE90734CDE9094489
:103F8000CDE90B4406F086FD08B1FFF7D7F80248EB
:103F9000FFF788FF0EB010BD140E0020002C01406A
:103FA000014B1868704700BF600E00200320704767
:103FB00008B501464FF47A7200238002890DFEF79E
:103FC00073FA08BD4FF47A73A0FB0303800A40EA3A
:103FD00083507047034B98689A689042FBD1C04366
:103FE000704700BF0028004008B5FFF7F3FF014B02
:103FF000186008BD600E002008B5FFF7EBFF024B0C
:104000001B68C01A08BD00BF600E0020024B187864
:1040100008B1FFF7DFBF7047640E002010B5074BF3
:10402000074C0122DA654FF48071204605F0DCF977
:104030004FF0FF332363002010BD00BF0028004075
:104040005008002002460021014805F0E4BB00BFF3
:104050005008002002460121014805F0DCBB00BFEA
:104060005008002010B58CB02C220021044601A875
:104070002AF08EFAFFF7D2FF0C4B0D481B681C4448
:104080000023089306934FF00053E4430793012263
:104090004FF4807301A902940B9305F0B9FA08B1AB
:1040A000FFF74CF800200CB010BD00BF600E0020E0
:1040B0005008002038B50546FFF78CFF0221044662
:1040C000074805F0AFFBC4F309024FF47A71A2FB75
:1040D0000121920AA30A2A8043EA805038BD00BF1A
:1040E000500800200148002105F09CBB500800202A
:1040F0000148012105F096BB50080020F8B50F4D8E
:104100002E78CEB90E4C4FF0FF372763FFF718F823
:10411000FFF784FF4FF48071204605F065F92046D3
:10412000276305F023FB32462046022105F073FB8E
:10413000FFF75AFF01232B700020F8BD640E00200A
:1041400050080020014610B54FF47A720023800217
:10415000890DFEF7A9F90146FFF73CFF0446FFF77A
:1041600039FF031B8B4200D310BD00BFF7E710F0EF
:104170007BBF000010B5064C0221204605F052FB23
:104180000221421C2046BDE8104005F044BB00BFA0
:10419000500800201648174A08B54FF4E133C0E92B
:1041A000002300230C22C0E90233C0E90523C0E943
:1041B0000733C0E90933036107F07DFE08B1FEF75C
:1041C000BDFF0B48002107F0EEFF08B1FEF7B6FF78
:1041D0000748002108F007F808B1FEF7AFFF0448D0
:1041E00007F0C1FF18B1BDE80840FEF7A7BF08BD42
:1041F000C80E00200044004070B596B00646142258
:10420000002103A82AF0C4F93822002108A82AF0C6
:10421000BFF93268274B9A424AD10223089308A873
:104220004FF440230A9305F011F808B1FEF786FF1A
:104230004FF0B04300259A6D1F4C42F400329A654E
:104240009A6D02F400320292029ADA6C42F0010294
:10425000DA64DB6C03F001030193019B0C2202235F
:10426000CDE9032303A907234FF090400793CDE93D
:10427000055504F075F9114925621423C4E90013AA
:104280001023C4E9023520468023C4E90435C4E97B
:10429000065503F0A1FE08B1FEF750FF2520F46794
:1042A00000220221A66203F005FE252003F034FE61
:1042B00016B070BD00440040680E0020800002402F
:1042C00002680C4B9A4210B5044612D14FF0B0422E
:1042D0000C21936D23F4003393654FF0904004F06C
:1042E000EBF9E06F03F0EAFEBDE81040252003F093
:1042F00021BE10BD0044004008B50A4601460248F0
:1043000006F058FF002008BDC80E002013B5114B61
:10431000114C18604FF40013009302AB13E9060030
:10432000204607F0C4FE2368DA69D103FCD4DA69B9
:104330005202FCD59A68084842F480029A6007F05D
:10434000FCFE06490448012207F06AFE002002B084
:1043500010BD00BF5C0F0020C80E0020640F0020BD
:1043600008B5074B1860FEF71EFCFFF713FF054A60
:10437000D2F8803043F00063C2F88030002008BDDE
:10438000600F00200008005808B54FF0B0430848FF
:104390009A6B42F400329A639A6B22F400329A6369
:1043A000FFF78EFF112003F0C5FD002008BD00BF00
:1043B000C80E002008B5074807F07DFD08B1FEF7DC
:1043C000BDFE054803F008FE18B1BDE80840FEF741
:1043D000B5BE08BDC80E0020680E00200268044B60
:1043E0009A4203D1034B00201B681847704700BF57
:1043F00000440040600F002002680B4B9A4210B549
:1044000004460FD1094B1B682BB1D0F8902012B98C
:1044100007480121984720460549BDE81040012280
:1044200007F0FEBD10BD00BF004400405C0F00203F
:10443000640F00202DE9F04F9DB0FEF743FA13F012
:10444000BBFA024640B90146644B022010F040FA24
:1044500001201DB0BDE8F08F012013F055FB12F0D4
:1044600051F80446039040B9024601465C4B0220D5
:1044700010F02EFA13F014FBEAE75A4D296812F0F7
:1044800091FC6968204612F0A7FC297A204612F0B8
:10449000D7FC697A204612F007FD6969204612F0C0
:1044A00093FDE868FDF7E0FF81B2204612F016FDAB
:1044B0002969204612F0DEFCA97A204612F0A6FCFB
:1044C0000221204612F058FD1021204612F096FDE0
:1044D000039812F09FF80246049040B90146424BFF
:1044E000022010F0F5F903A812F06CF8C2E703A857
:1044F00012F068F8049812F0F5FB024640B9014644
:104500003A4B022010F0E4F904A812F0A1F9B1E747
:10451000374EDFF8E0A0DFF8E0B0002333604FF063
:104520000208049805AB0A2208A912F0CDF9054645
:1045300028BB02460146314B022010F0C9F9306811
:104540002C49FDF78FFD4FF07C51FDF78BFD30605E
:10455000049812F0F7FB044604A812F079F913F05E
:104560009FFA002C3FF474AF002D3FF471AF00228E
:10457000234B1146032010F0ABF9002069E73168A6
:104580000998FDF767FCBDF81890306000221D4BBC
:10459000CDF800901146022010F09AF908AC0027DF
:1045A000BBB2994504F1080405D8B8F1010FC6D093
:1045B0004FF00108B5E754F8040C5146FDF752FDE1
:1045C000FDF752FF019034F8083C009300225B464F
:1045D0001146022010F07CF90137E1E7E05E0308A4
:1045E000F85E0308200000202D5F0308545F0308D5
:1045F0000C19002000007A44B75F03087D5F0308B0
:10460000CE5F0308A65F030830B5044685B00846B0
:1046100014491546FDF726FDFDF700FFCCB1114901
:1046200002902846FDF71EFDFDF7F8FE0E490190A9
:104630002846FDF70DFC0D49FDF7C8FDFDF714FFF9
:10464000002200900A4B1146032010F041F905B0FA
:1046500030BD0090074B22462146032010F038F968
:10466000F5E700BF00007A44CDCC4C3FCDCCCC3E2A
:10467000E75F0308146003082DE9F04FADF2344DF5
:104680004FF4007200210CA829F082FF4FF4007251
:1046900000218CA8B34E29F07BFF002537464FF050
:1046A00000082C46B9682046FDF7D4FB796804461B
:1046B0002846FDF7CFFB08F10408B8F5007F054652
:1046C00007F11007EED14FF070512046FDF7CAFCFC
:1046D0004FF0705104462846FDF7C4FC0025DFF872
:1046E000848207464FF00009AA46D8F80800214600
:1046F000FDF7AEFB0146FDF7B5FC01465046FDF760
:10470000A9FB39468246D8F80400FDF7A1FB014613
:10471000FDF7A8FC01462846FDF79CFB09F10409BA
:10472000B9F5007F054608F11008DED14FF0705151
:104730005046FDF797FC4FF070510A902846FDF760
:1047400091FC82460A98FCF7FFFF874B00222BF072
:1047500093FECDE904015046FCF7F6FF824B0022A0
:104760002BF08AFEFDF720FB0DF130090546C84607
:1047700000234FF0000BB168B0690693FDF768FBAA
:10478000FDF74CFE0028B8BF4042FDF717FC48F883
:10479000040B01465846FDF75DFB069B0433B3F559
:1047A000FE7F834606F11006E5D17049FDF70EFD48
:1047B0000DF13008064600234FF0000B314658F843
:1047C000040B0693FDF744FB0146FDF74BFC069BEB
:1047D00001461846FDF73EFB0BF1010B1FFA8BFB60
:1047E000BBF17F0F0346E9D16049FDF7EFFCFCF711
:1047F000ABFF5D4B00222BF03FFECDE906010DF52E
:104800000C78C346002200234846D9F800104068BF
:104810000B930892FDF71CFBFDF700FE0028B8BFC4
:104820004042FDF7CBFB089A4BF8040B01461046BB
:10483000FDF710FB0B9B01339BB27E2B09F10409A2
:104840000246E1D14A49FDF7C1FC4FF0000B814619
:104850000023494658F8040B0893FDF7F9FA01467E
:10486000FDF700FC089B01461846FDF7F3FA0BF133
:10487000010B1FFA8BFBBBF17E0F0346E9D13C49CC
:10488000FDF7A4FCFCF760FF374B00222BF0F4FD92
:10489000CDE9080137492846FDF7E4FBFDF7BEFDE9
:1048A000344902905046FDF7DDFBFDF7B7FD314975
:1048B00001903846FDF7D6FBFDF7B0FD002211460A
:1048C0002D4B0090022010F003F82C492C4F284665
:1048D000FDF770FD08B105233B702A4B1A782A4B6F
:1048E0001B889BB29A4280F08C80284B1A78284B08
:1048F0001B889BB29A4206D226492046FDF76EFDE0
:1049000008B101233B70244FDFF890A03B880A9A3E
:1049100001339BB23B803B889BB20A2B04BF002330
:104920003B803B884FF01C0B9BB20BFB03F3DDE994
:1049300004014AF803403B889BB20BFB03A35A6077
:104940003B889BB20BFB03A8FDF72EFA3B88C8F807
:1049500008009BB20BFB03A34FF08641DD603D884E
:1049600030461DE08C1000200000E03F0000FE42B9
:104970000000FC4200007A442A60030800007A43E9
:10498000720F0020A70300206A0F0020A60300205A
:10499000680F0020CDCC4C3F8C180020740F0020F5
:1049A000FDF760FBADB20BFB05A528613D88DDE995
:1049B0000601FDF7F9F94FF08641FDF753FBADB263
:1049C0003B880BFB05A59BB26861324D0BFB03AA2C
:1049D0002A788AF81820DDE90801FDF7E5F94FF09B
:1049E0008641FDF73FFBFDF73FFD2B4BC0B2188022
:1049F0002B78012B05D10022284B114602200FF005
:104A000067FF274F234D3B78DFF89880012B24D197
:104A1000DFF89490254EB9F80030B9F800204FF037
:104A20001C0A9BB292B20AFB03F30AFB0262F05823
:104A30009168FDF70FFA2146FDF7D0FCB0B10223D3
:104A40002B702B78022BD8B204D10022184B1146C0
:104A50000FF03EFF2B78DBB23B702B78DBB23B7064
:104A6000C8F800400DF2344DBDE8F08FB9F80030C1
:104A7000D8F800909BB20AFB03662046B168FDF7A8
:104A8000E9F94946FDF7AAFC10B103232B70E4E7CE
:104A90002870E2E7720F0020660F002070600308A4
:104AA000700F00206C0F00208C180020740F002065
:104AB000B56003082DE9F04F9FB0FDF703FF12F03A
:104AC0007BFF024640B90146A84B03200FF000FFD0
:104AD00001201FB0BDE8F08F012013F015F810F091
:104AE00029FC04460D9040B902460146A04B032024
:104AF0000FF0EEFE12F0D4FFEAE79E4F3B78012B59
:104B0000DDB252D0022D6FD0002D39D1042110F02A
:104B1000D7FF0121204610F001FF9749204610F0F1
:104B200031FF9649204610F013FF9549204610F0BA
:104B3000C1FE9449204610F0D7FE0221204610F015
:104B4000F3FF9149204610F0D5FF214606A810F04A
:104B500033FF8E4A19928E4A1A924FF07C530022EC
:104B600018A9204618931B921C921D9310F050FF19
:104B70002946204610F070FF0321204610F086FFE2
:104B80000D9800243C7010F06BFC02460E9000283B
:104B90006DD1804B014603200FF09AFE0DA810F056
:104BA00037FC0EA810F0EAFCA4E77B4E294610F073
:104BB000B5FE7149204610F0E5FEB168204610F0C0
:104BC00079FEF168204610F08FFE716A204610F0E1
:104BD000BFFEF16C204610F08DFF704B0022114695
:104BE00001200FF075FECBE76B4D012110F096FE12
:104BF000E969204610F0C6FE696A204610F0A8FE5A
:104C0000A968204610F056FEE968204610F06CFEB8
:104C1000A86CFDF729FC81B2204610F085FFE96CF5
:104C2000204610F067FF214606A810F0C5FE2B6B4A
:104C300018936B6B1993AB6B1A93EB6B1B932B6CE9
:104C40001C9318A96B6C1D93204610F0E1FEA86A16
:104C5000FDF70AFCC1B2204610F0FEFE286AFDF7FF
:104C600003FCC1B2204610F079FF4D4BB6E710F0BF
:104C70001BFD38B900224B4B114603200FF028FED4
:104C8000002026E71422214613A829F081FC0026E3
:104C9000DFF8EC80DFF81091DFF810A1212537460E
:104CA0000E980FA910F058FD0246002840F08A80A7
:104CB00001463F4B03200FF00BFEDFF8F8800E9803
:104CC00010F012FDB8F8003000229BB2114600939C
:104CD0000320394B0FF0FCFD0D9D0121284610F0FB
:104CE0001DFE0421284610F0EBFE2349284610F053
:104CF00049FE2249284610F02BFE2149284610F093
:104D0000D9FD2049284610F0EFFD0221284610F079
:104D10000BFF1D49284610F0EDFE294606A810F0AD
:104D20004BFE1A4A1992254A1B924FF07C534FF0C2
:104D30007E5218A928461C9218931A931D9310F0BE
:104D400067FE0021284610F087FE0321284610F058
:104D50009DFE0D990EA810F03BFC0246002840F085
:104D600084800146164B022016E700BFE05E030870
:104D7000FA60030808190020000082429A99993FBE
:104D8000CDCC4C3F000020406666263F000020410D
:104D90000AD7233C7C610308901800201A6103089D
:104DA0004A61030897610308CDCCCC3EA4030020E0
:104DB000B56103088E180020DE610308CDCC4C3E9F
:104DC00013620308119A10999DF83C00FFF71CFC30
:104DD0009DF83C30FBB1DDF844B038465946FDF74C
:104DE00039F8109907463046FDF734F84146064633
:104DF0005846FDF72DF84946FDF7E8F9FDF734FB75
:104E00001EAB80B203EB4000013430F82C3C013380
:104E1000E4B220F82C3C9AF80030012B1ED1DFF8C8
:104E200018B2864ABBF8003011999BB202EB03130B
:104E30009960BBF800309BB202EB0312109B5360E9
:104E4000BBF800309BB25A1C92B2802BABF800200A
:104E500004D1FFF711FC0023ABF800300F20FDF761
:104E6000A9FD013D7FF41CAF27E70E9810F01CFC54
:104E700000283FF4FFAE0DA810F0CAFADFF8C0B169
:104E80004FF021090E980FA910F066FC0546002886
:104E90007CD1024601466B4B03200FF019FDB8F898
:104EA0000030DFF8A491DFF8A4B100229BB21146D4
:104EB00000930320664B0FF00BFD012C94BF0023E1
:104EC000012389F8003099F800300022CDE9004331
:104ED0001146604B03200FF0FBFC0DF14C084FF026
:104EE000000A38F8022B3AB1CDE900A200225B4655
:104EF000114601200FF0ECFC0AF1010ABAF10A0F89
:104F0000EFD155493846FDF7ADF807462046FDF785
:104F100055F8804601463846FDF758F94E49074690
:104F20003046FDF79FF84146FDF750F94B4B1F60A7
:104F30004B4B002118608046FDF728FA0646A8B9B9
:104F40004223404699F80090CDE90343FDF766FA05
:104F500002903846FDF762FA5FFA89F9CDE90090D0
:104F6000404B3246314603200FF0B2FC0E9810F051
:104F7000BBFB04460EA810F001FB12F091FD002CC3
:104F80003FF4A6AD85F00100C0B2A2E5119A1099D8
:104F90009DF83C00FFF738FB9DF84930002B43D1CA
:104FA0009DF83C30FBB1DDF844A038465146FCF793
:104FB00051FF109907463046FCF74CFF2A49064638
:104FC0005046FCF745FF5946FDF700F9FDF74CFA4E
:104FD0001EAB80B203EB4000013430F82C3C0133AF
:104FE000E4B220F82C3C214B1B78012B1CD1B8F8E3
:104FF0000030124A11999BB202EB03139960B8F882
:1050000000309BB202EB0312109B5360B8F80030E3
:105010009BB25A1C92B2802BA8F8002004D1FFF753
:105020002BFB0023A8F800300F20FDF7C3FCB9F1DB
:1050300001097FF427AF32E78E1800208C10002082
:10504000CDCCCC3EB5610308EB180020926203087A
:10505000336203085E62030800007A44E41800200B
:10506000E0180020B2620308CDCC4C3FA40300201E
:105070002DE9F043ADB014230DF10E0204A9ADF8F3
:105080000E3012F021FF044648B902460146194B82
:1050900003200FF01DFC20462DB0BDE8F083002258
:1050A000154B164FDFF85880DFF858901146032053
:1050B0000FF00EFC0025BDF80E30AAB29342EAD9DB
:1050C000AAB22CAB03EBC202032012F89C6C52F87C
:1050D000A03C002E14BF3A464246CDE900320022E1
:1050E0004B4611460FF0F4FB002E05F1010508BFF9
:1050F0003446E0E70C6303082F63030802630308E8
:10510000076303085363030830B5102289B00025F4
:10511000294604460DEB0200039529F039FA14F0F4
:105120007DFA2A46A34B0090294603200FF0D0FBBE
:10513000FDF7C8FB12F040FC8DF80C0012F0E6FC05
:10514000431B18BF012301218DF80D30029012F08E
:10515000FBFC029812F09AFE029812F00FFD0298E2
:10516000FFF786FF002840F0008102A812F0DEFC65
:1051700012F096FC029812F01DFD029812F036FD16
:105180000298FFF775FF002840F0F38002A812F0A4
:10519000CDFC12F085FC029812F044FD0022864BF3
:1051A000114603200FF094FB029812F057FD02986D
:1051B000FFF75EFF002840F0E08002A812F0B6FC86
:1051C00012F06EFC029812F065FD002211467B4B36
:1051D00003200FF07DFB0022794B114603200FF0D6
:1051E00077FB029812F0E2FD0298FFF741FF0028DA
:1051F00040F0C78002A812F099FC12F051FC02980E
:1052000012F0F0FD002211466E4B03200FF060FB00
:1052100000226D4B114603200FF05AFB029812F04A
:10522000FDFD0298FFF724FF002840F0AE8002A8A1
:1052300012F07CFC12F034FC029812F00BFE0022FB
:105240001146624B03200FF043FB0022604B1146D6
:1052500003200FF03DFB029812F038FD0298FFF793
:1052600007FF002840F0958002A812F05FFC12F0C2
:1052700017FC029812F046FD00221146554B032000
:105280000FF026FB0022544B114603200FF020FBA9
:10529000029812F053FD0298FFF7EAFE00287CD135
:1052A00002A812F043FC12F0FBFB029812F062FD20
:1052B00000221146494B03200FF00AFB0022404B0D
:1052C000114603200FF004FB029812F06FFD0298C4
:1052D000FFF7CEFE002864D102A812F027FC12F0DE
:1052E000DFFB029812F07EFD00221146354B0320B1
:1052F0000FF0EEFA0022344B114603200FF0E8FACB
:10530000029812F08BFD0298FFF7B2FE00284CD1F4
:1053100002A812F00BFC12F0C3FB029812F09AFDE7
:1053200000221146294B03200FF0D2FA0022114629
:105330002B4B03200FF0CCFA01238DF8173003AB71
:1053400003CB00222060186861600C23A060114626
:1053500000930320234B0FF0BBFA02A812F0E6FBE8
:1053600012F09EFB002009B030BD01238DF80E30F5
:1053700000E701238DF80F300DE701238DF8103081
:1053800020E701238DF8113039E701238DF8123021
:1053900052E701238DF813306BE701238DF81430A9
:1053A00083E701238DF815309BE701238DF8163034
:1053B000B3E700BF6963030892630308C56303088A
:1053C000F66303082564030852640308876403082E
:1053D000BA640308ED6403081E6503084E650308FC
:1053E0007C650308A965030802480122102103F027
:1053F000DDB900BF0004004802480022102103F07C
:10540000D5B900BF0004004813B5134C23785BB92D
:10541000E37C03F0FF023BB9104B1146022002B0BF
:10542000BDE810400FF054BAFEF76AF800380C4B94
:1054300018BF0120400018701A78022A02BF00220B
:105440002270E2741B7800930022064B1146032061
:105450000FF03EFA02B010BD8D1B0020C865030896
:1054600050190020E465030838B5184C23785BBB5D
:10547000E37C03F0FF023BBB154D2B68012B0CD9DD
:105480002B68042B09D81146124B02200FF020FA8A
:10549000114A0421012000F0F3FE2B68042B13D9DC
:1054A00000220E4B114602200FF012FAFEF728F8E8
:1054B00000380B4B18BF0120400018701B78022BDE
:1054C00002BF00232370E37438BD00BF8D1B002092
:1054D0004C190020FB6503082066030825660308B5
:1054E0005019002010B501214FF0904003F058F9F9
:1054F0000C4B0D4A1870002414701B780B4ADBB259
:1055000002214FF09040137003F04AF9084B094A0A
:10551000187014701B78084ADBB21370BDE8104095
:10552000FEF716B90A0100200A1900200801002020
:1055300009010020091900200701002010B5164BB1
:105540001A78022A26D91B78072B23D8FFF7B2FA3C
:105550001248134A037811785B1A124918BF0123C5
:105560000B7003781048DBB21370104B104A1C7894
:105570000378E31A18BF012313700E4B04701B78D5
:1055800023B100230B700C490B701370BDE8104061
:10559000FEF7DEB810BD00BF06010020EB180020AA
:1055A000E8180020EC180020700F0020720F002077
:1055B000710F002050190020EE18002008B50121BD
:1055C0004FF0904003F0ECF8064B012816BF022282
:1055D00018701A701878044B1978BDE80840FEF767
:1055E0001FB800BF050000200000002038B5324D74
:1055F000324C287BFCF7DEFC3149FCF733FDA06020
:10560000687BFCF7D7FC2E49FCF72CFDE060A87BFB
:10561000FCF7D0FC2A49FCF725FD6062E87BFCF72B
:10562000C9FC2849FCF71EFD274BE0642361287C58
:10563000FCF7C0FC6060687CFCF7BCFCA061A87C47
:10564000FCF7B8FCE061E87CFCF7B4FC2062287D44
:10565000FCF7B0FCA062687DFCF7B0FC1849FCF7D1
:1056600001FD2063A87DFCF7A5FC6063E87DFCF7E5
:10567000A5FC1449FCF7F6FCA063287EFCF79AFC15
:10568000E063687EFCF79AFC0D49FCF7EBFC2064B4
:10569000A87EFCF793FC0A49FCF7E4FC6064E87E12
:1056A000FCF788FCA064287FFCF784FC074BE062D1
:1056B00002221A7038BD00BF580300209018002045
:1056C000CDCCCC3D0AD7233CCDCCCC3E0819002014
:1056D00038B5114D114C287BFCF770FC1049FCF7D4
:1056E000C1FCA060687BFCF769FC0D49FCF7BAFCC3
:1056F000E060A87BFCF762FC0949FCF7B3FC606240
:10570000E87BFCF75BFC0749FCF7ACFC064BE0646C
:1057100001221A7038BD00BF5803002090180020E5
:10572000CDCCCC3D0AD7233C081900207FB5394E9B
:10573000394D33780370394B1B784370044601218F
:105740004FF0904003F02CF82B78A070E37002210A
:105750004FF0904003F024F8314B20711B786371B7
:105760002B78012B52D12F4B1868FCF77DFE2E4B66
:10577000E0801868FCF778FE80B22C4BA0831B7881
:1057800084F82430191F4A424A41A2779BB1284A23
:1057900003EB830302EB8303002200931146254BA6
:1057A00002200FF095F8244B1B8884F82530234BFA
:1057B0001B8884F8263002A80FF0ECFA204B1A78E8
:1057C000FAB1204A1168E1B112681F4A15681F4AF0
:1057D00012681B78AD1AC3EB0313B5EB830F10D916
:1057E00000221B4B114602200FF072F8194B258541
:1057F00001221A701B78184A84F827300823137086
:105800003370164B01221A7004B070BD0020E08086
:10581000B3E700BF05000020EB18002006010020C0
:10582000EA180020E4180020E0180020720F002081
:105830003E000020586603086A0F0020660F002013
:10584000A503002004190020FC180020F8180020EF
:10585000866603088B1B00200600002048190020E4
:10586000024B0122002103200FF032B8A666030884
:10587000024B0122002103200FF02AB8DC66030846
:1058800008B50122074B002103200FF021F8FFF794
:10589000ABFDFFF7ABFE044A00231370034A1370FD
:1058A00008BD00BF2267030808190020891B0020DB
:1058B00010B5104B0122002102200FF009F80E4B09
:1058C00004225A706321012200241A7083F82A10DE
:1058D00083F82B201C635C6383F827401C85FFF74B
:1058E00083FDFFF7C5FFFFF7BBFFFFF7C9FF034BC2
:1058F0001C7010BD5867030810190020891B002078
:105900001FB5114B11491C6858681A7A5B7ACDE9AA
:105910000223FCF7A7FBFCF7A7FD0C4901902046EA
:10592000FCF7A0FBFCF7A0FD0022094B00901146FC
:1059300003200EF0CDFFFEF77DFD642004B0BDE82E
:105940001040FEF7A7B900BF2000002000007A44F5
:105950008F67030870B586B00D460446FFF744FD17
:1059600001F024FEFDF7ECFA9620FEF793F90026ED
:10597000AE420AD101AB03CB1B882381094B2060C7
:10598000002261601A7006B070BDFEF725F801A80C
:10599000FFF7BAFB41F28830FEF77CF90136FFF7DA
:1059A000AFFFE5E7891B002030B585B00446002530
:1059B00003A8ADF80C50FCF789FF70B19DF80C30CE
:1059C0009DF80D20237062702946CDE90032032036
:1059D000034B2A460EF07CFF012005B030BD00BF0E
:1059E000C4670308022801D8FFF7FEBC70470228ED
:1059F00001D8FFF701BD7047022803D802481021E3
:105A000002F0D9BE704700BF0004004808B5FEF799
:105A10008DF8BDE8084000F06BBE4FF0FF300FF08E
:105A2000A1B8704770470000014BD870704700BFA5
:105A300018010020014B1874704700BF18010020A6
:105A400007B5064B00221B5C00931146044B022055
:105A50000EF03EFF03B05DF804FB00BF03680308CF
:105A6000E967030808B5002102200FF043F80A4B4C
:105A70001B7803F0FF014BB9084B1A68042A05D8BC
:105A80001A68102001321A600FF034F8BDE808409F
:105A900003480FF097BA00BF8D1B00204C1900205F
:105AA000F01A0020002101200FF024B813B5104A8D
:105AB000104C42F21073002818BF03460E482360B2
:105AC00013600FF031FA21680B480FF0B5FA0A485D
:105AD0000FF078FA23684FF47A72B3FBF2F30022E6
:105AE00000931146054B01200EF0F2FE02B010BDEE
:105AF0009C03002014010020F01A0020076803080E
:105B000013B50D4C206023680BB90C4B23600C4877
:105B10000FF00AFA21680A480FF08EFA08480FF0D1
:105B200051FA236800930022064B114603200EF021
:105B3000CFFE02B010BD00BF9C030020A086010074
:105B4000541900203368030837B5044600283AD0BA
:105B500090F90650002D43D125480FF0E5F92A466B
:105B60002946244B02200EF0B3FEE379012B0CBF33
:105B7000214B224B2A4629460220214D0EF0A8FE39
:105B8000E3792B701F4B1868FFF7BAFF1E4B18689C
:105B9000FFF78CFF29781D4A1D4B012908BF1346CA
:105BA0000022009311461B4B01200EF091FE94F948
:105BB0000530019394F9043000930022164B1146EE
:105BC00003200EF085FE154B0122002102201A70E1
:105BD0000EF090FF124803B0BDE830400FF0F2B96C
:105BE0000022104B114602200EF072FEDFE700BFCC
:105BF0009C190020786803088D680308AA680308C8
:105C00008A1B00209C030020140100206F680308F9
:105C100073680308C7680308FF680308881B00202F
:105C200084190020E66803080A460149FDF742B9D5
:105C300000F0030870B516480FF076F906F034FF4F
:105C4000044650B10022134B114602200EF040FED4
:105C5000BDE8704010480FF0B5B9104D104B02462A
:105C6000014602200EF034FE01260E4B2E70224615
:105C7000214602200EF02CFE0B4806F0A9FD2878E4
:105C8000314606F0FDFA02480FF09CF9E0E700BF4C
:105C9000F01A002028690308D81A00207C0100208F
:105CA000466903085A69030818010020F0B599B045
:105CB000FDF76EFF054606F0DDFB074600283ED1E6
:105CC0006F4C0AA8FFF732FD132323706D4B1A782F
:105CD00002F0FF06002A43D01F70142323706A4B82
:105CE00062681B7863F07F031370636828B200EB6F
:105CF000400000EB4010FE22B0FBF2F0587002238F
:105D0000624A1278012A88BF00236370604C637A6C
:105D100033B106F09BFB012802D120460FF004F9B5
:105D20005C4B5748D978002206F0BAFB01460028A0
:105D300040F091800122584B10460EF0C9FD00241E
:105D400056480FF0F1F8564B54481968A14238BF35
:105D500021460FF071F951480FF034F919B0F0BD38
:105D6000504A117801F0FF030029C9D0464B167044
:105D70001B78626863F07F03137063689DF8285096
:105D80005D7062689DF82930937062689DF82A10F2
:105D9000D17062689DF82B10117162689DF82C100B
:105DA000517162689DF82D109171BDF82E206168C7
:105DB000120ACA716068BDF82E200272BDF8442034
:105DC000120A4272BDF8442082729DF84620C272C7
:105DD0009DF84C2002739DF84F204273BDF850206F
:105DE000120A8273BDF85020C27303EB83032E4A5C
:105DF00003EB8303134401932C4B05EB850503EB65
:105E00004503009332462A4B314601200EF060FDD7
:105E10009DF84C300893BDF84A3007939DF8463002
:105E20000693BDF844300593BDF82E3004939DF8D9
:105E30002D3003939DF82C3002939DF82B30019365
:105E40009DF82A30009332461A4B314601200EF05D
:105E50003FFD102354E706317FF471AF06F0F0FAEE
:105E6000044600283FF46BAF01224FF47A730021FF
:105E7000B0FBF3F3104600930F4B0EF029FD5FE7E4
:105E80000C010020881B0020E4190020501900207C
:105E90009C19002018010020B86A0308F01A00209D
:105EA00014010020481900207D010020F402002088
:105EB00079690308A4690308C76A030800B50346A3
:105EC0008DB000282CD0407802280AD003282AD090
:105ED000164B0022114602200DB05DF804EB0EF0C7
:105EE000F7BC1A7F0B92DA7E0A929A7E09925A7E4A
:105EF00008921A7E0792DA7D06929A7D05925A6878
:105F00000492DA68039293F914200292B3F91220F2
:105F100001921B7C00930022054B11460EF0D8FC29
:105F20000DB05DF804FB034BD3E700BFE56A03083F
:105F3000FC6A03086E6B030801284FF000020CBFD7
:105F4000024B034B114602200EF0C2BC8D6B0308BE
:105F50009F6B03081FB50446002831D00378002B3F
:105F60002ED01D480FF02EF8002211461B4B0220A8
:105F70000EF0AEFC94F91830039394F90A300293B2
:105F8000237C0193E368009300221146144B032005
:105F90000EF09EFC0022134B114603200EF098FCDD
:105FA000237A012B0ED1617A0F4A104B002918BFBA
:105FB00013460022009311460D4B03200EF088FC7F
:105FC00004B010BD00220B4B1146032004B0BDE805
:105FD00010400EF07DBC00BFCC190020B86B030848
:105FE000E96B03081A6C0308B46B0308B36B03086E
:105FF000276C0308386C030808B5104B01220021F8
:1060000002201A700EF076FD0D480EF0DBFF0D4BEE
:106010001B788BB10C4B1A7872B9DB7C63B90B4BD4
:106020001A68042A9EBF1A6801321A600021BDE86E
:10603000084010200EF05EBD08BD00BF881B002088
:10604000541900208A1B00208D1B00204C190020B1
:1060500008B5002140200EF04DFD074B1B7853B1D1
:10606000064B1A78012A06D100211970BDE80840B4
:1060700002200EF03FBD08BD8A1B0020EC18002056
:10608000044B1B78022B03D1002108200EF032BDF7
:10609000704700BF7C010020044B1B78012B03D00C
:1060A000002180200EF026BD704700BF06010020B1
:1060B00008B506F002FD80B906F0C8F901280CD138
:1060C000BFF34F8F0549064BCA6802F4E0621343E1
:1060D000CB60BFF34F8F00BFFDE708BD00ED00E0D0
:1060E0000400FA0538B504460D4607484FF4006130
:1060F000FCF700FF30B92A4621460348BDE8384086
:10610000FCF7FEBD38BD00BF00F0030810B506F077
:1061100069FD10F1080F07D1064B0022BDE81040C1
:10612000114602200EF0D4BB013001D1024BF4E73E
:1061300010BD00BF466C03085C6C030810B5114825
:10614000042102F038FB104B1B78012B19D00F4BA8
:106150001A78082A10D10E4C2378142153B102204A
:10616000FDF7CAFA237883F001032370BDE81040DD
:10617000FDF7E4BA0320F3E718781421FDF7BCFA21
:10618000F4E710BD000400480601002005000020CF
:106190009803002070470000022837B5044634D029
:1061A000402853D0012854D12B4B1B78002B50D0C2
:1061B000FA20FDF76FFD21464FF0904002F0F0FA13
:1061C000264B214618704FF0904002F0E9FA214624
:1061D00005464FF0904002F0E3FA214B214A002897
:1061E00008BF1346CDE900531F4B00221146022081
:1061F0000EF06EFB002120200EF07CFC002102201E
:1062000003B0BDE830400EF075BC184B1B7803B3EB
:10621000FA20FDF73FFD21464FF0904002F0C0FA12
:10622000134B214618704FF0904002F0B9FA214606
:1062300005464FF0904002F0B3FA0E4B0E4A00288C
:1062400008BF1346CDE900530C4BCEE700210420D4
:10625000D6E703B030BD00BF0A19002003000020BC
:10626000806C0308746C0308A66C030809190020ED
:1062700002000020996C03088C6C0308CC6C0308A6
:1062800073B505460C46164606F0F4F8034600289A
:1062900040D000242A480EF047FE2A4B28481968AF
:1062A000A14238BF21460EF0C7FE254802B0BDE826
:1062B00070400EF087BE4A68F05CD0540133DAB209
:1062C0009442F8D8204B0D701A781B78012A88BFA9
:1062D00000244C700022CDE900341C4C1C4B1146AC
:1062E00001200EF0F5FA637A33B106F0AFF8012819
:1062F00002D120460EF018FE164B1748D97800221E
:1063000006F0CEF8014638B9144B012203200EF0F6
:10631000DFFABEE71049D2E70631BAD106F090F8AD
:1063200004460028B6D04FF47A730122B0FBF3F391
:106330000021009303200A4B0EF0CAFAAAE700BF1F
:10634000F01A002014010020501900209C19002090
:10635000F16C0308180100200C010020B86A030842
:10636000C76A0308044B1B7823B9044A052101209E
:10637000FFF786BF704700BF50190020226D030849
:1063800010B5002490B03C22214601A8009428F0CA
:10639000FFF8354B2022DA7219788DF80010597801
:1063A0008DF8011099788DF80210D9788DF80310C6
:1063B00019798DF8041059798DF8051099798DF8AF
:1063C0000610D9798DF80710197A8DF80810597AC6
:1063D0008DF80910997A8DF80A108DF80B20214656
:1063E0000DF10B0258180131007B02F8010F1C2936
:1063F000F8D193F828208DF8282093F829208DF8DB
:10640000292093F82A208DF82A2093F82B2093F83E
:1064100028108DF82B20154A19BB93F8291001F08C
:10642000FF00F1B9107093F82C206AB193F83F2067
:1064300052B10DF12B0100229818013290F82C0076
:1064400001F8010F142AF7D109484FF40061FCF755
:1064500051FD20B9064840226946FCF751FC10B0B6
:1064600010BD01211170DEE758030020A4030020B5
:1064700000F8030810B5002204461146054B02201F
:106480000EF026FA20460449BDE8104040220EF0E6
:1064900025BB00BF286D030800F8030873B54B4CFB
:1064A000207963794D2BC0B25ED1C0EB0010800023
:1064B0000A2838BF0A204FF47A735843444B1860B7
:1064C000A379E2794D2ADBB256D1C3EB03139B00CB
:1064D0004FF47A7202FB03F594F82C30002B53D161
:1064E00094F83F30002B4FD142F21070FFF7DEFAE4
:1064F000384B1868FFF704FB237A374A3749DBB279
:106500001370374B01221A70637A364ADBB213706C
:1065100094F82830344A03EB83035B00DBB213703A
:1065200094F82930314A03EB83035B00DBB213702C
:1065300094F82B302E4A03EB83035B00DBB213701D
:106540000023E21892F82C20D2B2CA540133142B43
:10655000F7D1A378012B37D1E37A202B34D102B0C5
:10656000BDE87040FFF7A4B96379482B0ABF4FF428
:106570006163637958439BE7E279482A0ABF4FF485
:106580006162E2795343A3E71A4EFFF78FFA356051
:10659000336813B942F21073336017480EF0C4FC2D
:1065A000316815480EF048FD13480EF00BFD3368B6
:1065B0004FF47A72B3FBF2F30022009311460F4BB3
:1065C00001200EF085F997E702B070BD5803002056
:1065D000140100209C030020060100208D1B0020D8
:1065E0000500002050190020A7030020A60300206A
:1065F000A5030020A00300206C1900203C6D0308B7
:1066000010B590B000213C2201A8009127F0C0FFF6
:106610004022344968460EF061FA9DF800203AB9EC
:106620009DF80100102803D19DF8021001290FD018
:1066300000222D4B114602200EF04AF9FFF7A0FE72
:106640004FF47A70FDF726FBFFF728FF10B010BD5E
:10665000264B1A70587099709DF80310D9709DF8E8
:10666000041019719DF8051059719DF80610997163
:106670009DF80710D9719DF8081019729DF809103E
:1066800059729DF80A1099729DF80B1001F03F01A4
:10669000D972D87AD1B288421BD89DF8282083F8C5
:1066A00028209DF8292083F829209DF82A2083F8A6
:1066B0002A209DF82B2083F82B200DF12B0100229E
:1066C0009818013211F8014F80F82C40142AF7D1A4
:1066D000BAE701F140006844194410F8340C08731B
:1066E0000132D6E700F80308756D0308580300204F
:1066F000F0B50C238BB0052600240125CDE90563F8
:1067000018221023CDE9033221466D4B0294224614
:106710000327CDE90055022009940EF0D9F8694B02
:10672000029422462146CDE9005702200EF0D0F80F
:10673000CDE901640226644B00962246214630468C
:106740000EF0C6F8614B009522462146CDE9017452
:1067500030460EF0BDF809A9204606F093F9099BD2
:10676000C3F307220292C3F307421B0E0192009368
:106770002246574B214630460EF0AAF809A9284672
:1067800006F080F9099BDAB20392C3F30722029262
:10679000C3F307421B0E0192009322464D4B214644
:1067A00030460EF095F84C4B4C48009422464FF47E
:1067B000FA710EF05BFB4A4B4A48009422464FF4B4
:1067C000FA710EF053FB484B484800942A464FF4A8
:1067D000FA710EF04BFB464B464800942A464FF4A4
:1067E000FA710EF043FB2046FCF784FA08B1FCF77F
:1067F000A5FC414B009400224FF4FA613F480EF093
:1068000035FB3F4A002101200EF030FA3D4A0021BD
:1068100002200EF02BFA3C4A002104200EF026FA4A
:106820003A4A002108200EF021FA00F019FE3849FA
:10683000384806F0DDF8384805F0CAFF2B480EF05E
:10684000C1FB364B0021187805F01AFD344900943D
:10685000344B0968344800220EF008FB32480EF031
:10686000B1FBFFF7CDFE314A002110200EF0FEF9FA
:106870002F4A002120200EF0F9F92E4A0021402055
:106880000EF0F4F92C4A002180200EF0EFF92B4B8A
:106890002B4819682B4B009401220EF0E7FA284888
:1068A0000EF090FB284B29481968294B00940122CF
:1068B0000EF0DCFA25480EF085FB0BB0F0BD00BFF2
:1068C000B56D0308F56D0308166E0308376E0308EF
:1068D000586E0308796E0308235A0008CC1900206B
:1068E00095610008B4190020996000089C190020E7
:1068F0003D6100088419002081600008D81A00203A
:10690000D5C50008AD5C00080D610008355C0008C5
:106910000000030130010020180100207C0100204C
:1069200014010020655A0008F01A0020695400087C
:10693000E55400083D550008BD550008A00300209F
:106940006C190020516000089C030020541900209D
:10695000F95F000873B50D4D00262E60FEF7D0FFDD
:10696000C820FDF797F928683146FBF70FFD04466C
:106970000028F3D12868FBF751FD054B0090224613
:10698000214601200DF0A4FF02B070BD0C190020BB
:106990009D6E030830B50024A5B07C22214605A8D1
:1069A000049427F0F5FD53238DF8103001254FF4A2
:1069B0008873ADF81230ADF800408DF81450FDF733
:1069C000E7F8FE23B0FBF3F000EB400000EB4010D3
:1069D0003A4B8DF815002246214603200DF078FF32
:1069E0006846FEF7E1FF9DF800309DF80120134353
:1069F00014D158238DF81630072480220021304806
:106A000027F0C6FD224604A92D4827F057FE2C4A40
:106A100021460120FFF734FC25B030BD0E23294666
:106A200001A8CDE901448DF81630ADF80C40FEF711
:106A300091FF01AB03CB234C1B88CDF81B10ADF8A5
:106A40001F30CDF81700FEF75BFF2068FBF70CFD49
:106A50000A254FF47A7380B2B0FBF3F0B0FBF5F384
:106A600005FB130030308DF821002068FBF7FCFC9B
:106A7000642380B2B0FBF3F0B0FBF5F305FB130029
:106A800030308DF822002068FBF7EEFC80B2B0FBBE
:106A9000F5F0B0FBF5F305FB130030308DF8230063
:106AA0002068FBF7E1FC80B2B0FBF5F305FB1300B7
:106AB00030308DF8240015249FE700BFD06E030806
:106AC000081B00200C1900202DE9F047044694B063
:106AD000BD480D46802200210EF00AF82378592B7C
:106AE00040F04082052D5ED86378443B162B5AD87F
:106AF000DFE813F07C015900590159006101590088
:106B0000590059005900BD0059004401590059006D
:106B10005900D70159005900E700590059005900A0
:106B20001700A678482E17D1A84A14210120FFF794
:106B3000A7FB41F28830FDF7ADF80022A44B1146C7
:106B400003200DF0C5FE40F6B830FDF7A3F814B0F1
:106B5000BDE8F047FFF7ACBA532E0DD1FFF71AFF8F
:106B600041F28830FDF796F8974A1521012014B0BC
:106B7000BDE8F047FFF784BB432E17D1002404A8DB
:106B80008DF8104005F09CFD8F4A4C2313701023A4
:106B900093709DF81030547001204133D070137100
:106BA0000521FFF76DFB14B0BDE8F087442EFAD144
:106BB000854C884DA670592323705A236370FFF7C4
:106BC000C9FE2868FBF72AFC0022834B009011467F
:106BD00003200DF07DFE7F220021601C27F0D8FCF1
:106BE000102326700126A370E6702671FCF7D0FFF3
:106BF000FE23B0FBF3F000EB4000042300EB401059
:106C00006071A3712868FBF72FFC0A274FF47A7391
:106C100080B2B0FBF3F0B0FBF7F307FB13003030AA
:106C2000E0712868FBF720FC642380B2B0FBF3F02E
:106C3000B0FBF7F307FB1300303020722868FBF736
:106C400013FC80B2B0FBF7F0B0FBF7F307FB1300C7
:106C5000303060722868FBF707FC80B2B0FBF7F3B6
:106C600007FB13003030A07222460B217EE7A37889
:106C7000303BDBB2092B96D8584C594A2370237805
:106C8000DBB25372504A592313704D23537023784B
:106C90000321303301209370FFF7F2FA2378009339
:106CA0000022504B114601200DF012FEFFF768FB49
:106CB00023780BB1FCF7A4FC14B0BDE8F047FCF757
:106CC00047BDA578482D1BD13F4C56232370102378
:106CD000A37018236371052301200025A3712246A8
:106CE0000C230821E3716570E0702071FFF7C8FA8A
:106CF0003D4B00942A46114602200DF0E9FD52E773
:106D0000432D7FF450AF00213C2205A82E4C049166
:106D100027F03EFC04A8FFF7ADFB9DF81030637030
:106D20009DF81130A3709DF81230E3709DF8133078
:106D300023719DF8143063719DF81530A3719DF88F
:106D40001630E3719DF81730257023729DF81B50A3
:106D50009DF8183063729DF81930A3722A469DF889
:106D60001A30E37207A904F10D00257327F0A6FC81
:106D700005F10D012246C9B2012012E7A078392899
:106D80000CD83038C0B2FEF72DFE0F4A23781370AE
:106D900063785370A37893700321E7E614B0BDE8DD
:106DA000F047FFF7DFBAA0783928F7D83038C0B2FB
:106DB000FEF71DFEE9E7A0783928EFD83038C0B2D9
:106DC000FEF71AFEE1E700BF081B0020E96E03088A
:106DD000FE6E03080C190020206F030850190020D4
:106DE00058030020436F03086C6F0308A378303BFF
:106DF000DAB2092AD2D8E578303DEAB2092ACDD8EC
:106E00002179A1F14802D2B20B2AC7D87A4840FAB8
:106E100002F2D007C2D40A224D2902FB03553BD10E
:106E20003C235D43754B4FF47A7068431860744B94
:106E30001860FEF73BFE734A237813706378537033
:106E4000A3789370E378D37005212379137101201F
:106E5000FFF716FA6C4B002610221E705A700122A2
:106E60009A70DA70A178303901EB8100E17830391D
:106E700001EB4001C9B2197122795A71634A127843
:106E8000D2B21A72624A1278D2B25A72FFF778FA04
:106E9000604B009532462EE74829C3D14FF4616319
:106EA000BFE7A378303BDAB2092A3FF677AFE5783F
:106EB000303DEAB2092A3FF671AF2179A1F14802CB
:106EC000D2B20B2A3FF66AAF4B4840FA02F2D20721
:106ED0003FF564AF0A224D2902FB03553DD13C2307
:106EE0005D43474B4FF47A7606FB05F21A6018684B
:106EF000FEF706FE434A2378137063785370A37835
:106F00009370E378D3700521237913710120FFF783
:106F1000B7F93D4B002710221F705A7001229A705A
:106F2000DA70A178303901EB8102E178303901EB78
:106F30004201C9B299712279DA71344A1278D2B217
:106F40001A72334A1278D2B25A72FFF719FAB5FBA5
:106F5000F6F5314B00953A46CDE64829C1D14FF4BC
:106F60006163BDE7502B40F0A881022D7FF61BAE78
:106F70006178A1F13003012B3FF615AEA378312BD8
:106F80007FF411AE052D4FD1E378302B40F0C48053
:106F90001E4D224E00232B702B7803F0FF0253B9B5
:106FA0002379303BDBB233703378009311461C4BAE
:106FB00002200DF08DFC16491A4A00230B7033781D
:106FC000DBB213702B78104ADBB213720B78DBB292
:106FD0005372FFF7D5F90B4B22781A7062785A700A
:106FE000A2789A70E278DA7022791A71FCF7B0FB15
:106FF0000521044ABAE500BFDEF7FFFF14010020B7
:107000009C030020081B00205803002006010020DC
:1070100050190020966F0308CD6F0308040000206C
:107020001770030805000020082D69D1E378462B6E
:1070300040F0EC802579A5F13000C0B2092800F2BB
:107040003A816179A1F13003092B00F23481A279F0
:10705000A2F13003092B00F22E81E379A3F130066F
:10706000092E00F2288105EB85067600B04D20360A
:1070700001EB8101F6B249002E702031AD4E263A67
:10708000C9B2D2B2317002EB8202AB4903EB830387
:1070900052005B000A802033A84ADBB21370A84A72
:1070A00082F828006379303BDBB282F82930A3797B
:1070B000263BDBB282F82A30E379303BDBB282F840
:1070C0002B302B782BB9337803F0FF020BB99D4B93
:1070D0001A70FFF755F99C4B22781A7062785A7033
:1070E000A2789A70E278DA7022791A7162795A710C
:1070F000A2799A71E279DA71FCF72AFB082178E724
:10710000042D2FD1E278A2F13003DBB2092B11D983
:10711000A2F14103192B0AD9FFF724F900228B4B66
:107120001146012014B0BDE8F0470DF0D1BBA2F12B
:107130003703DBB286480370834B207859703121C6
:1071400018709970DA70824B7D4A1B78DBB213722B
:10715000804B1B78DBB25372FFF712F9FCF7F8FA99
:10716000042146E71D2D4FD9A61C0025DFF8D0913C
:10717000DFF8E4A13746A84617F8012F303AD2B21B
:10718000092A3ED809EB050303201A731B7BCDE9BE
:1071900002533B780022CDE90053114653460DF0CF
:1071A00097FB01351E2DE7D1B8F1000FB4D1FEF7E2
:1071B0001DFA654B50221A7000225A7010229A70E4
:1071C0000122DA7003F8042F203416F8012F03F897
:1071D000012FB442F9D15A4B00221A7010225A7072
:1071E00001229A70DA705A4A1278D2B21A72594A47
:1071F0001278D2B25A721E22DA72FFF7C1F8232136
:10720000F7E64FF00108CCE7072D85D900254C4F54
:10721000DFF8448102342E4614F8012F303AD2B2FE
:10722000092A46D8791903200A730B7BCDE902534A
:1072300023780022CDE90053114643460DF048FB68
:107240000135082DE8D1002E7FF466AFFEF740FA35
:107250003D4B3B4C50221A7010229A70002501229F
:107260005D70DA7003F8042F62190135127B082D66
:1072700002F1300203F8012FF6D10022502311460B
:1072800000930120354B0DF023FB002323701023C6
:1072900063700123A370E3702D4B1B78DBB2237264
:1072A0002C4B1B78DBB26372E572FFF769F80D2196
:1072B0009FE60126C4E700219BE6412B7FF473ACD7
:1072C0006378432B7FF46FAC162D7FF46CAC244DA8
:1072D000621C002312F8011FE9540133142BF9D169
:1072E000FEF792F81F4B5B7D012B1DD11449002343
:1072F000EA5CC8180133D2B2142B80F82C20F7D1E5
:10730000144B00221A701B78DBB24B72FFF738F86F
:107310000D4A631E153413F8011F02F8011B9C422D
:10732000F9D1094A162121E40A4B02221A70EFE72B
:10733000A7030020A60300203C000020A503002096
:1073400058030020A4030020081B002076700308C7
:107350000601002050190020337003085B700308F9
:107360008D1B0020AC09002070B5054688B00C4686
:10737000002951D033480DF025FE26789EB3002D0C
:107380005ED068682E7870B3032E0BD0132E45D0D4
:10739000022E28D16978012925D00B0623D4FFF7C6
:1073A00093FB20E06B78012B07D10078012802D0F5
:1073B000022800D008B905F03DF900250DF11F00A5
:1073C0008DF81F5005F07CF91F4A4C2313701023D1
:1073D00093709DF81F305570012041330521D07006
:1073E0001371FEF74DFF237C052B15D894F90A2065
:1073F000059294F909200492144A52F82330039319
:1074000094F90830CDE901630022E3680093114646
:107410000F4B03200DF05CFA08B070BD6B78012BA8
:10742000E1D102780B4B02F001021A702AB90A4B23
:10743000114603200DF04CFAD5E7084B0022F7E780
:107440002E46D0E7B4190020081B00200071030865
:10745000AE700308E41900209B700308A5700308B0
:10746000034B0022C3E902220122C3E90022704734
:10747000A41B002000487047A41B00204FF0B0431D
:1074800082B0DA6C0243DA64DB6C03400193019B47
:1074900002B070472DE9F04186B000240220154D5E
:1074A0000594FFF7EBFF0420FFF7E8FF124F03946A
:1074B0004FF4807601230DEB0001CDE901632846EE
:1074C000032304934FF4005801F04AF801A9384609
:1074D000CDF8048001F044F822464146384601F0D8
:1074E00065F928462246314601F060F9204606B08B
:1074F000BDE8F0810004004800080048032810B5EA
:107500000ED8012810D868B902460B484FF4807194
:1075100001F04CF9002209484FF4005101F046F9FE
:10752000002010BD0122F0E7002203484FF48071D3
:1075300001F03CF90122EEE7000400480008004891
:10754000022070470020704701207047002814BFB8
:1075500016200F20704700000D48854600F025F8E2
:107560000C480D490D4A002302E0D458C45004339E
:10757000C4188C42F9D30A4A0A4C002301E0136074
:107580000432A242FBD327F06BF8FBF7B9FDFEE70C
:107590000000012000000020C8070020E0D60308FA
:1075A000C8070020403B0020FEE7704710B50320CD
:1075B00000F06EFC01F07CFA064B18600F20FCF71F
:1075C0005FFB044618B9FBF711FF204610BD0124EC
:1075D000FBE700BFA80300204FF0E022136923F06F
:1075E0000203136170474FF0E022136943F0020376
:1075F00013617047014BD3F8900570470070FF1F6F
:10760000014BD3F8940570470070FF1F014BD3F86E
:10761000980570470070FF1F024A536843F001034A
:1076200053607047002004E0024A536843F00203AD
:1076300053607047002004E0024A536843F004039B
:1076400053607047002004E08068C0F380007047FA
:10765000F7B5002301930446002800F0E980856D0A
:1076600025B9FBF7D7F9E56584F8545023689A6883
:10767000D00040F1A1809A68D10000F1B480A26DE1
:1076800042F01002A265E26D42F00102E2650125BE
:107690001846FFF7D9FFA26D02F01002024340F036
:1076A000C980A26D206922F4817242F00202A265B3
:1076B0009A68D2075DD4226BA67E94F82CC0003A5B
:1076C00018BF01221703D4E902120A43217E42EABD
:1076D0008132617E42EAC13242EA4632002842EA01
:1076E0004C02B4BF20F000414FF400113A430A436A
:1076F00094F82010012903D1002E76D142F4803273
:10770000616A21B1A66A01F4E07131430A43D96884
:10771000E66C21F4FE3121F4FF711143D96094F835
:107720003C206168012A01F0404C4CEA060609D170
:10773000D4E910273A433243A66C324342EA0C02A2
:1077400042F001061F693E4A3A4032431A6121F075
:107750000042B2F1804F0CD0B1F1004F09D0394E48
:10776000D6F8082701F4701122F470120A43C6F803
:1077700008275A69666BA16B22F0070232435A61EF
:107780005A6922F0700242EA01125A61002835D18A
:107790009A6A62F00F029A625B6903F007039E42E5
:1077A0003CD10023E365A36D23F0030343F0010301
:1077B000A365284603B0F0BD9A68234922F0104221
:1077C00022F0170242F080529A60204A1268B2FBFF
:1077D000F1F2013252000192019A002A3FF44BAFBC
:1077E000019A013AF7E7002552E7A16D41F0200127
:1077F000A165E16D41F00101E16581E7B0F5001F90
:10780000CAD19A6AE269013A92006FF00F0102F060
:107810001C0201FA02F2216E0A43BCE7A36D23F0B9
:10782000120343F01003A365E36D43F00103E36526
:107830000125BEE7A36D43F01003A365F8E700BF81
:1078400002FCFF1F00200140400D0300A8030020A0
:10785000F8B54569082D04460E460AD00368DB6872
:10786000D80705D5A36D43F02003A3650120F8BD1B
:107870000425FCF707FA074623681A682A4220D035
:10788000A26D42F40072A265DA6812F4406F14D15E
:10789000A27E92B91A6812070FD51846FFF7D4FED8
:1078A00020BB5A6822F00C025A60A26D22F480724A
:1078B00022F0010242F00102A265227EFAB100200C
:1078C000D5E7711CD9D0FCF7DDF9C01BB04201D857
:1078D000002ED1D123681B682B40CDD1A26D84F836
:1078E000543042F00402A2650320C0E7A26D42F0CA
:1078F0002002A265E26D42F00102E265DDE70C22A2
:107900001A60DCE70368186C70470000F7B50023C5
:10791000019390F85430012B044600F0C0800568B4
:107920000269012380F854302846FFF78DFE0028B5
:1079300040F0AF80D1E90030022822F004027ED06E
:10794000B2F1004FC3F3110E35D1AA6A42EA0E021A
:10795000AA628A68686902EA032222F07C4222F065
:10796000FF0220EA03210A43002B6A611DDA4D4A17
:107970004D4DD2F80817AB4201F0E07043D10D0233
:1079800013D4D2F8083723F0E073034343F4000321
:10799000C2F80837454B1A68454BB2FBF3F20C238B
:1079A00002FB03330193019B53BB0020002384F8A7
:1079B000543003B0F0BD226E00F01F074FF00F0CE3
:1079C0000CFA07FC6FEA0C0622EA0C0CBEF1000F61
:1079D00011D1C3F38462BA4042EA0C0222668008E5
:1079E000E26901309042B4D8A86AC3F38362BA4016
:1079F00006403243ACE793FAA3F2B2FA82F2EAE726
:107A0000019B013BCEE72B4DAB420BD1C901CCD43E
:107A1000D2F8083723F0E073034343F08073C2F8D1
:107A20000837C2E7244DAB42BFD14B02BDD4D2F8D8
:107A3000083723F0E073034343F48003EFE7B2F128
:107A4000004F01BFAA6AC3F311018A43AA62002B47
:107A5000ABDA154813498342D1F8082709D1D1F888
:107A6000083702F0A07223F0E0731A43C1F8082728
:107A70009BE71048834204D1D1F8083702F4400252
:107A8000F1E70D48834290D1D1F8083702F0C07277
:107A9000E9E7A26D42F02002A265184686E70220BF
:107AA00087E700BF00200140001000B0A8030020BD
:107AB000400D0300004000B8002000B4026838B553
:107AC00004461046FFF7C0FD08B9002038BD936892
:107AD000990707D4936823F0004323F0170343F07A
:107AE00010039360FCF7CEF8054623689B685B079C
:107AF000EBD5FCF7C7F8401B0228F6D923689B6832
:107B00005A07F2D5A36D43F01003A365E36D43F06C
:107B10000103E3650120D9E773B5002302680193EF
:107B20009368DD07044602D5002002B070BD91685D
:107B3000214B194209D0A36D43F01003A365E36DF7
:107B400043F00103E3650120EFE7936823F000436E
:107B500023F0170343F001039360184BD3F8083761
:107B600018021CD4637E012BDED0FCF78BF8144E78
:107B7000054622681368DB07D6D49368D9075FBF30
:107B80009368334043F001039360FCF77BF8401B9C
:107B90000228EED923681B68DA07EAD4CBE7094B41
:107BA000094A1B68B3FBF2F301330193019B002BDD
:107BB000D8D0019B013BF8E717000080002001406E
:107BC000E8FFFF7FA8030020400D030038B50446FE
:107BD0000068FFF739FD054620BB94F85430012BAF
:107BE00020D0012384F854302046FFF795FFB0B928
:107BF000A36D226823F4706323F0010343F48073C0
:107C0000A3651C23E065136084F85400936823F097
:107C1000004323F0170343F00403936038BD84F856
:107C20005450FBE70220F9E7026838B59368916881
:107C30000446C80701D4002038BD9907FBD49368D7
:107C400003F00503012B19D1936823F0004323F0BF
:107C5000170343F00203936003231360FCF712F849
:107C6000054623689B68DB07E5D5FCF70BF8401B4E
:107C70000228F6D923689B68DA07F2D5A36D43F092
:107C80001003A365E36D43F00103E3650120D3E72F
:107C900070B5044600284BD0836D43F00203836522
:107CA000FFF70CFF054668B92046FFF7BDFF054604
:107CB00008B90123A3652268936823F0104323F0D9
:107CC0001703936023685A6822F4677222F0030254
:107CD0005A6040F29F321A60D968164A0A40DA6048
:107CE0001A6922F040421A615A6922F007025A6169
:107CF0001A6A02F0F0221A625A6A02F0F0225A62FC
:107D0000DA6A02F0F022DA629A6A0B4A00269E6270
:107D1000D2F8083723F0FE73C2F808372046FAF786
:107D20008DFEE6652666A66584F85460284670BD1B
:107D30000125FBE700023E830020014010B590F8CA
:107D40005430012B044615D0012380F85430FFF73E
:107D5000B5FE58B92046FFF767FF38B9A36D23F485
:107D6000807323F0010343F00103A365002384F82B
:107D7000543010BD0220FCE7F7B50023019390F8C2
:107D80005430012B04467FD0012380F85430FFF794
:107D90004BFF23689A6812F00102054607D0A36DD5
:107DA00043F01003A365002384F854302DE0A16D47
:107DB000364F21F4817141F00201A165DE68D96876
:107DC00026F4FF4626F07C0621F40041360421F01B
:107DD0000301360CD96008209968394041F0004110
:107DE00099609968002913DA01990131019101998B
:107DF000B1F52E3FF5D3A36D23F0120343F010032A
:107E0000A365002384F854300125284603B0F0BD53
:107E1000D3F8B410013801F07F010A44DCD199682D
:107E20001A48014041F001019960D3F8B41021F0E3
:107E30007F0141EAD202C3F8B4209A68024042F0BE
:107E400002029A60FBF71EFF074623689A68D20772
:107E500008D4DA683243DA60A36D23F0030343F0F9
:107E600001039FE7FBF70EFFC01B0228EDD9236833
:107E70009B68D907E9D5A36D43F01003A365E36DB3
:107E800043F00103E365BFE70225BEE7E8FFFF7F9C
:107E90000749CA6822F4E0620302120403F4E063B3
:107EA000120C134343F0BF6343F40033CB607047BD
:107EB00000ED00E0164B30B5DC68C4F30224C4F1D9
:107EC0000703251D042B28BF0423062D4FF0FF3583
:107ED0008CBF033C002405FA03F321EA0303A54009
:107EE00022EA0502A340002843EA0203ACBF00F1E6
:107EF0006040084A4FEA0313B8BF00F00F00DBB23E
:107F0000AABF00F56140135480F8003330BD00BFB4
:107F100000ED00E014ED00E0002807DB044A410911
:107F2000012300F01F00834042F82130704700BF5A
:107F300000E100E000280CDB4309064900F01F00C7
:107F400020330122824041F82320BFF34F8FBFF33B
:107F50006F8F704700E100E070B5D0E913456560B0
:107F6000446D14B1D0E916456560D0E9105404F0B1
:107F70001C060124B4406C60046863608368102BA5
:107F80000BBFA260A160E160E26070BD0268416C5D
:107F9000D3B210B5083B1424B3FBF4F30B4CA2424C
:107FA00088BF0B4A21F0030199BF01F1804202F51D
:107FB0000232521807338264064AC26403F01F0378
:107FC000012202FA03F3036510BD00BF070402405B
:107FD0001C0802408008024038B500285CD00268C6
:107FE0002E4B9A424FF014014AD82D4B1344B3FB49
:107FF000F1F32C499B00C0E91013022380F82530CF
:108000001368056923F4FF4323F070031360D0E97C
:10801000024323432B43456911682B4385692B4356
:10802000C5692B43056A2B430B431360FFF7AEFF73
:10803000B4F5804F04BF002343604368816C03F0B4
:108040007F020A60D0E91314013B032B4C601ED859
:10805000154B1649816513449B000121013A01FA31
:1080600002F200214365C2651960114B5A64002376
:108070000122C36380F8243080F82520184638BDDB
:108080000C4B1344B3FBF1F30B499B00B3E7002304
:10809000C0E91533C365EAE70120F0E707040240B1
:1080A000F8FFFDBF000002403F820010400902407F
:1080B00000090240F8FBFDBF0004024038B500286B
:1080C00041D00268136823F0010313601F4B9A42EA
:1080D0004FF0140130D81E4B1344B3FBF1F31D498C
:1080E0009B00C0E91013012403F01C0304FA03F3FE
:1080F000002515604B60FFF749FF836C41681D60E8
:10810000D0E913325A604A1E032A06D8124B0B4498
:108110009B0094401D60114B5C640023C363C0E965
:108120001533C0E90B33C0E90D33C36580F8253042
:1081300080F82430184638BD094B1344B3FBF1F3E3
:1081400008499B00CDE70120F5E700BF0704024086
:10815000F8FFFDBF000002403F820010000902400E
:10816000F8FBFDBF0004024070B590F82450012DCB
:1081700004463BD090F825600125AE4280F824509B
:108180004FF000062CD1022580F825500568C66303
:108190002E6826F001062E60FFF7DEFE036BBBB1F2
:1081A0002B6843F00E032B60A36C1A68D20342BF06
:1081B0001A6842F480721A60636D1BB11A6842F447
:1081C00080721A602B6843F001032B60002070BDA1
:1081D0002B6823F004032B602B6843F00A03E2E7CB
:1081E0008023C36380F824602846F0E70220EEE78E
:1081F000034640B190F82520022A06D00422C2632B
:10820000002280F82420012070470268806C1168E9
:1082100021F00E011160016821F480710160116884
:1082200021F001011160D3E9100202F01C010122CA
:108230008A404260D3E9132151605A6D32B111680E
:1082400021F480711160D3E91621516001220020D0
:1082500083F8252083F82400704708B590F825306E
:10826000022B03D00423C363012008BD03681A68EE
:1082700022F00E021A601A6822F001021A60826C63
:10828000136823F480731360D0E9101303F01C0209
:10829000012393404B60D0E913325A60436D33B1F0
:1082A0001A6822F480721A60D0E916325A600123EB
:1082B00080F82530002380F82430836B03B1984781
:1082C0000020D2E770B4426C046C036826681D6815
:1082D00002F01C020421914031420FD015F0040F2E
:1082E0000CD01A6892065EBF1A6822F004021A6067
:1082F000036B6160002B33D070BC184702219140A2
:10830000314217D015F0020F14D01A68940606D423
:108310001A6822F00A021A60012280F82520114A08
:1083200093428CBF104B114B5960002380F82430CE
:10833000C36ADFE708219140314211D029070FD5E8
:10834000196821F00E011960012303FA02F262603C
:10835000C36380F82530002380F82430436BC9E7DD
:1083600070BC7047800002400004024000000240E0
:108370000A4A536943F4802330B55361EFF3108404
:1083800072B60023CD58C5500433B3F5807FF9D1C0
:108390001369DB03FCD484F3108830BD004000581F
:1083A000064B5A69002ABFBF054A9A6002F188321B
:1083B0009A60BABF5869C00F00207047004000584B
:1083C00023016745044B5A6942F000425A615869DB
:1083D000C043C00F704700BF0040005870B505464D
:1083E000FBF750FC124E04463369D90313D43369AA
:1083F000DA0744BF012232614CF2FA32134011D144
:108400000B4E306910F480200BD0FBF73BFC001BB7
:10841000A842F6D304E0FBF735FC001BA842E3D3E7
:10842000032070BD024A1361024A01205360F8E73D
:1084300000400058B41B00202DE9F041184D98462B
:108440002B78012B06460C46174626D001232B70AD
:108450004FF47A7000236B60FFF7C0FFA0B9012EC4
:1084600016D1104A536943F0010353612760BFF3EB
:108470006F8FC4F804804FF47A70FFF7AFFF094A9A
:10848000536923EA0603536100232B70BDE8F08192
:1084900039462046FFF76CFFEDE70220F6E700BF04
:1084A000B41B002000400058054A536923F47E7332
:1084B00043EAC00040F4803040F002005061704751
:1084C000004000582DE9F041234F3B78012B054631
:1084D00088463FD001233B704FF47A7000237B60C5
:1084E000FFF77CFF044688B92B68042B13D11B4A85
:1084F000536943F4803343F0040353614FF47A70BB
:10850000FFF76CFF0446154B1A681B6800233B708D
:108510002046BDE8F0814FF0FF33C8F800306E68A8
:10852000D5E901321344B3420AD93046FFF7BCFF04
:108530004FF47A70FFF752FF50B1C8F8006004465C
:10854000064A536923F47E7323F002035361DAE78A
:108550000136E5E70224DBE7B41B002000400058A9
:108560002DE9F04F524C00234FF00F090A6832FA00
:1085700003F501D1BDE8F08F012505FA03F818EAEB
:10858000020200F08E804E68032706F003054FEAD2
:10859000430E07FA0EFC6F1E012F6FEA0C0C32D847
:1085A000876807EA0C0ACF6807FA0EF747EA0A0756
:1085B0008760476827EA0808C6F300179F4047EA24
:1085C00008074760C76807EA0C088F6807FA0EF7C4
:1085D00047EA0807022DC76017D14FEAD30800EB1E
:1085E000880803F0070AD8F820704FEA8A0A09FAC7
:1085F0000AFB27EA0B0B0F6907FA0AF747EA0B0792
:10860000C8F8207001E0032DDCD1076805FA0EF5EB
:1086100007EA0C073D4316F4403F056041D023F0C4
:10862000030707F1804707F5803703F0030CBD68A7
:108630004FEA8C0C4FF0070E0EFA0CFEB0F1904F83
:1086400025EA0E0E2FD01B4DA8422ED005F58065D1
:10865000A84214BF0725022505FA0CF545EA0E05C8
:10866000BD602568D74316F4801F0CBF3D401543FD
:108670002560656816F4001F0CBF3D40154365601A
:10868000D4F8805016F4803F0CBF3D401543C4F829
:108690008050D4F88450B60354BF3D401543C4F80D
:1086A0008450013362E70025D6E70125D4E700BFF7
:1086B0000008005800040048374A2DE9F04F002315
:1086C0004FF0010A4FF0070B4FF00F0931FA03F496
:1086D00001D1BDE8F08F0AFA03FC1CEA010654D070
:1086E00023F0030404F1804404F5803403F003070D
:1086F000A568BF000BFA07F8B0F1904F08EA050E25
:1087000045D0264DA84244D005F58065A8420CBF4F
:1087100002250725BD40754517D1D2F8805025EABE
:108720000605C2F88050D2F8845025EA0605C2F842
:108730008450156825EA06051560556825EA060582
:108740005560A56825EA0805A560056803265C0054
:1087500006FA04F423FA06F6254300EB86060560C4
:1087600003F00705376AAD0009FA05F527EA0507A2
:108770003762856825EA04058560456825EA0C05A9
:108780004560C56825EA0404C46001339EE70025FE
:10879000C0E70125BEE700BF0008005800040048FC
:1087A0000369194214BF0120002070470AB181619A
:1087B000704781627047436901EA030221EA0301BD
:1087C00041EA024181617047044AD168014208B51B
:1087D00002D0D060FDF7E0FC08BD00BF00080058E3
:1087E000024A136843F48073136070470004005812
:1087F0000D4B10B55B690C4628B99A0507D500F0FA
:1088000027F820B110BD9B0501D400F019F8074AE4
:108810001369012C23F00403136101D130BFF1E788
:1088200040BF20BF20BFEDE70004005800ED00E08E
:10883000024B186800F4C060704700BF0004005885
:10884000024A136843F480431360704700040058E1
:108850000C4A136823F4804313600B4B1B683221CE
:108860004B430A49B3FBF1F35169890500D533B98C
:10887000536913F4007F14BF032000207047013BAD
:10888000F2E700BF00040058A803002040420F0098
:108890000B4A136823F0070343F002031360094BEC
:1088A0001A69012842F004021A6105D130BF1A6921
:1088B00022F004021A61704740BF20BF20BFF6E7D4
:1088C0000004005800ED00E04FF0B0431868C0F31A
:1088D000404070474FF0B0431868C0F34000704705
:1088E0004FF0B042536823F47F4343EA00235360C0
:1088F00070474FF0B0431868C0F340607047000005
:108900007FB54FF0B0432C4AD3F80831C0F30310C1
:1089100003F00F0352F82040284A52F82330B4FBEA
:10892000F3F4FFF785FF264B054693E80700B5F5FE
:10893000007F04AB03E9070010D0224B9C4218D300
:1089400003F5B70303F67F539C4229D903F574134B
:1089500003F510639C4225D802230BE01A4B9C427E
:1089600007D91A4B9C421BD903F5370303F5D8539B
:10897000F0E7002304AA02EB830353F80C4C144DD8
:108980002B6823F0070323432B60FBF77BF9064694
:108990002B6803F007039C4206D1002004B070BD91
:1089A0000123E7E70024EAE7FBF76CF9801B0228C4
:1089B000EED90320F2E700BF1871030878710308AD
:1089C000781B0308C0CF6A00BFEA21013F9334023D
:1089D000004000584FF0B04310B59A68D96812F0C3
:1089E0000C0205D00C2A4AD101F00303012B51D10E
:1089F0004FF0B0412B480B6813F0080306D00B680A
:108A000013F0080337D1D1F8941007E00C6824075D
:108A100056BFD1F894300968C3F3032350F82330CC
:108A2000002A0CBF184600204FF0B0418A6802F0BF
:108A30000C020C2A1ED1CA6802F00302022A2ED0B0
:108A4000032A06D10B68184A13F4801F174B18BF6E
:108A500013464FF0B042D068D168D268C0F3062008
:108A60005843C1F302130133B0FBF3F0530F01334A
:108A7000B0FBF3F010BD0B68C3F30313CEE7042A79
:108A800005D0082A06D11B6813F4801305D00648C8
:108A90000023C9E700231846C6E70448C4E7024B91
:108AA000D7E700BF187103080024F4000048E8016C
:108AB00008B5FFF78FFF4FF0B043044A9B68C3F33C
:108AC000031352F82330B0FBF3F008BD78710308AC
:108AD0002DE9F0410446002853D04FF0B0439D6883
:108AE000DE6803689B0605F00C0506F0030668D5F2
:108AF000026A1DB10C2D46D1012E44D1002A40D06E
:108B00004FF0B043A16A1A68170756BFD3F89430E4
:108B10001B681B0903F0F00399421FD90846FFF7B1
:108B2000EFFE00282DD14FF0B042136843F0080348
:108B300013601368A16A23F0F0030B431360606AAB
:108B4000FFF7CEFEFFF7B4FFAB4B1860AB4B1868D6
:108B5000FBF796F8002834D0BDE8F0814FF0B04222
:108B6000136843F008031360136823F0F0030B430A
:108B70001360606AFFF7B4FE0846FFF7C1FE0028E5
:108B8000E0D00120E8E74FF0B043002A54D01A6843
:108B900042F001021A60FBF775F80746FFF79AFEEC
:108BA000002842D04FF0B042136843F0080313602E
:108BB0001368A16A23F0F0030B431360606AFFF7A8
:108BC0008FFE2368D80748D42368990700F18C806A
:108BD00023681E0740F1FA80A3694FF0B046002BCE
:108BE00000F0E180D6F89430E16903F01002914280
:108BF00000F0C48003F00302022AC2D0D80740F17B
:108C0000B380D6F8943023F00103C6F89430FBF714
:108C100039F80746D6F89430990740F1A580FBF75C
:108C200031F8C31B112BF5D904E0FBF72BF8C01B5F
:108C30000228B3D903208FE71A6822F001021A60D4
:108C4000FBF720F80746FFF745FE0028B9D0FBF7F1
:108C500019F8C01B0228F6D9ECE7082D03D00C2D1B
:108C600005D1032E03D16368002BADD189E74FF006
:108C7000B043A1681A6822F480120A431A6062683D
:108C8000B2F5803F10D11A6842F480321A60FAF7C8
:108C9000F9FF0746FFF718FE002895D1FAF7F2FF13
:108CA000C01B6428F6D9C5E7B2F5041F04D11A68C1
:108CB00042F400121A60E6E7196821F48031196065
:108CC000196821F400111960002AE0D1FAF7DAFFDF
:108CD0000746FFF7F9FD00283FF476AFFAF7D2FF19
:108CE000C01B6428F5D9A5E7042D236903D00C2DFA
:108CF0000ED1022E0CD1002B3FF443AF4FF0B04207
:108D00006169536823F0FE4343EA016353605FE700
:108D10004FF0B046BBB1336843F480733360FAF769
:108D2000B1FF074633685A0505D4FAF7ABFFC31BFA
:108D3000022BF7D97EE77368626923F0FE4343EAAA
:108D40000263736044E7336823F480733360FAF797
:108D500099FF074633685B057FF53AAFFAF792FF54
:108D6000C31B022BF6D965E74FF0B042E169D2F898
:108D7000943023F010030B43C2F894304FF0B04707
:108D8000D7F8943043F00103C7F89430FAF77AFF2C
:108D90000646D7F894309A0718D4FAF773FF831B66
:108DA000112BF6D946E7D6F8943023F00103C6F824
:108DB0009430FAF767FF0746D6F894309B0705D53D
:108DC000FAF760FFC31B112BF6D933E72368580766
:108DD00054D50B4F3B68D90514D4FFF701FDFAF7C2
:108DE00051FF06463B68DA050CD4FAF74BFF831BAC
:108DF000022BF7D91EE700BFA8030020AC03002018
:108E000000040058E3684FF0B046002B58D023F020
:108E10008003052B02BFD6F8903043F00403C6F858
:108E200090304FF0B046FAF72DFFD6F8903043F06F
:108E300001030746C6F8903041F28838D6F89030E2
:108E40009B0705D4FAF71EFFC31B4345F6D9F1E68D
:108E5000E36823F00403812B1BD1FAF713FFD6F844
:108E6000903043F08003C6F8903007464FF0B0468C
:108E700041F28838D6F89030180504D5E36A002B03
:108E80004AD1002068E6FAF7FDFEC01B4045F1D943
:108E9000D0E6FAF7F7FED6F8903023F08003C6F854
:108EA000903007464FF0B04641F28838D6F89030FF
:108EB0001905E3D5FAF7E6FEC01B4045F6D9B9E639
:108EC000FAF7E0FED6F8903023F080030746C6F8A4
:108ED000903041F28838D6F890301A0516D4FAF757
:108EE000D1FED6F8903023F00103C6F89030074643
:108EF0004FF0B04841F28836D8F890309B07BDD586
:108F0000FAF7C0FEC31BB342F6D993E6FAF7BAFEEE
:108F1000C01B4045DFD98DE60C2D4ED0022B4FF003
:108F2000B0431A6822F080721A6033D1FAF7AAFEB1
:108F30000546FFF7DEFC38BBD4E90C314FF0B042F8
:108F40000B43D0682D4901400B43E16B0B43216C6F
:108F50000B43616C0B43A16B43EA0123D36013689D
:108F600043F080731360D36843F08053D360FAF703
:108F700089FE0446FFF7BDFC002882D1FAF782FE85
:108F8000001B0A28F6D955E6FAF77CFE401B0A2892
:108F9000CFD94FE6FAF776FE0446FFF7AAFC30B9C0
:108FA0004FF0B042164BD1680B40D36069E7FAF737
:108FB00069FE001B0A28F0D93CE6012B3FF4E1AD25
:108FC0004FF0B043D868236B00F003029A427FF45D
:108FD000D8AD626B00F0700393427FF4D2ADA26B08
:108FE00000F4FE43B3EB022F7FF4CBAD636C00F0D3
:108FF0006040C01A18BF0120AEE500BF8C80C111CF
:10900000FCFFFEEE2DE9F0410D46044610B90120AB
:10901000BDE8F081684E336803F007038B4216D336
:1090200023689A0727D54FF0B047A268BB6823F0A2
:10903000F0031343BB60FAF725FE0646BB68DB036B
:1090400019D4FAF71FFE831B022BF7D911E03368FE
:1090500023F007030B433360FAF714FE0746336827
:1090600003F00703AB42DBD0FAF70CFEC01B02286B
:10907000F5D90320CCE72368580617D54FF0B04741
:109080006269D7F8083123F00F0343EA1213C7F8D7
:109090000831FAF7F7FD0646D7F80831D90305D4A9
:1090A000FAF7F0FD831B022BF6D9E2E723685A0793
:1090B00013D54FF0B047E268BB6823F4E063134375
:1090C000BB60FAF7DFFD0646BB689B0305D4FAF7E1
:1090D000D9FD831B022BF7D9CBE72368180714D5DA
:1090E0004FF0B0472269BB6823F4605343EAC203E0
:1090F000BB60FAF7C7FD0646BB68590305D4FAF70B
:10910000C1FD831B022BF7D9B3E72368DA070FD41D
:10911000294C236803F00703AB4239D8FFF7C8FC9A
:10912000264B1860264BBDE8F0411868FAF7A8BD39
:109130006268022A1DD1FFF7C7FB00283FF467AF22
:109140004FF0B04641F28838B36823F0030313436D
:10915000B360FAF797FD0746B368626803F00C0343
:10916000B3EB820FD4D0FAF78DFDC01B4045F3D985
:109170007FE7032A02D1FFF7BCFBDEE712B9FFF756
:10918000A9FBDAE74FF0B0431B685B05D8D43EE794
:10919000236823F007032B432360FAF773FD064689
:1091A000236803F00703AB42B8D0FAF76BFD801BCE
:1091B0000228F5D95DE700BF00400058A803002051
:1091C000AC03002008B5FFF773FC4FF0B043044A2E
:1091D0009B68C3F3022352F82330D84008BD00BF78
:1091E0005871030808B5FFF763FC4FF0B043044A19
:1091F0009B68C3F3C22352F82330D84008BD00BF98
:10920000587103084FF0B043D3F89000C0F340000A
:1092100070474FF0B0410209D1F8883002F47F2244
:10922000000123EA020300F47F200343C1F88830E1
:1092300070474FF0B041020CD1F88830120423EA95
:10924000020343EA0040C1F8880070470368DA036C
:1092500070B5044639D5FFF7C3FAFAF713FD614E2E
:1092600005463368DB0532D54FF0B043616BD3F868
:10927000902002F4407291421DD0D3F89010D3F8A0
:10928000902042F48032C3F89020D3F8902021F44B
:10929000407022F480328D07C3F89020C3F890000C
:1092A00009D5FAF7EFFC41F288360546FFF7AAFF29
:1092B000012840F090804FF0B042616BD2F89030BE
:1092C00023F440730B43C2F89030002605E0FAF710
:1092D000D9FC401B0228C4D903262568E8070AD513
:1092E0004FF0B0416268D1F8883023EA124392B25D
:1092F0001343C1F88830A9070AD54FF0B041A268DE
:10930000D1F8883023EA124392B21343C1F888306F
:10931000AA0609D54FF0B0422169D2F8883023F46B
:1093200040630B43C2F88830AB0502D5206AFFF7D3
:1093300080FF680502D5606AFFF77BFF290502D52B
:10934000A06AFFF776FF6A0602D56069FFF761FF42
:109350002B0602D5A069FFF75CFFE80502D5E0699E
:10936000FFF757FFE90610D54FF0B042E168D2F899
:10937000883023F440730B43C2F88830B1F5807F06
:1093800002BFD36843F08073D3602A040ED54FF038
:10939000B042216BD2F8883023F040430B43C2F82F
:1093A000883019B9D36843F08073D3606B0410D54B
:1093B0004FF0B042E16AD2F8883023F040530B43BB
:1093C000B1F1005FC2F8883003D1D36843F4803331
:1093D000D360304670BDFAF755FC401BB0427FF6B3
:1093E00065AF79E70004005830B590F82C30012BB8
:1093F00002464FF0020022D0174B82F82D00CA24FB
:10940000012582F82C505C6253245C62B1F5807FA8
:10941000146B996914D121F488519961596C24F025
:10942000010421F0004159641463DD650A4BFF21FA
:1094300059620020012382F82D3082F82C0030BDC3
:1094400021F408519961D96C24F0020421F0004103
:10945000D9641463D865E9E70028004070B50B4E65
:10946000036B756D1D40EA07044603D50123F365C0
:10947000FAF77DFEAB0704D50223F365204600F022
:10948000C9F9012384F82D3070BD00BF00280040C9
:1094900038B50A4CE36823F02003E360FAF7F2FBE7
:1094A0000546E3689B0601D5002038BDFAF7EAFBC4
:1094B000401BB0F57A7FF4D90320F6E7002800407E
:1094C000F8B5114DEC6814F0400406461AD1EB686B
:1094D00043F08003EB60FAF7D5FB23460746EC68C0
:1094E00014F0400401D1032B01D11846F8BDFAF75E
:1094F000C9FBC01BB0F57A7F234684BF032386F8DF
:109500002D30ECE70023F0E70028004038B50F4C81
:10951000E36823F08003E360A3699B06054606D455
:10952000FFF7B6FF10B1032085F82D0038BDA36901
:1095300023F02003A361FFF7ABFF10B1032085F8F0
:109540002D00A36943F02003A361EFE7002800404A
:1095500038B5044600284BD090F82D3003F0FF02B8
:109560001BB980F82C20F9F725FE0223214D84F841
:109570002D30EB68DB0636D4CA236B6253236B6253
:109580002046FFF79DFF10B1FF236B6238BDAB692A
:1095900023F08E6323F04003AB6121696368AA69FD
:1095A0000B431343A2691343AB61D4E9022343EA9B
:1095B00002432B61D4E90931EA680B4322F4F852E3
:1095C0001343EB602046FFF7A1FF0028DCD1D4E96C
:1095D0000713AA690B4322F06042134362691343E5
:1095E000AB61FF236B62012384F82D300020CDE7AF
:1095F0000120CBE7002800400023092803D840EAD7
:109600000310C0B270470A380133C0B2F5E700005A
:109610002DE9F04790F82C30012B05464FF0020061
:1096200069D0012385F82C304E4B85F82D00DE687B
:1096300006F44076B6F5807F78D04C69087891F8CA
:10964000019091F802A091F82470002A55D19B69ED
:1096500013F0400308BFCB70FFF7CEFF80464846AB
:10966000FFF7CAFF02465046FFF7C6FF814638465D
:10967000FFF7C2FF0B6ACF78234343EA875343EADD
:10968000090343EA084343EA022343EA0063354AF5
:10969000CA205062532050628C6A8869B4F5807F7A
:1096A000946945D124F4885494610124D465B6F5B5
:1096B000807F09BFCB6913640343536418BF5064B0
:1096C000284B4A681A672A6B42F001022A639A699A
:1096D00042F488529A61244AD2F8803043F400332D
:1096E000C2F880301F4BFF225A620020012385F808
:1096F0002D3085F82C00BDE8F087B4F1803F07D00D
:10970000B4F5000F04D09B6913F0400308BFCB7081
:109710000B6ACA781C4344EA0A0444EA004343EA59
:10972000092343EA825343EA0763B0E70023AEE725
:1097300024F4085494610224D465B6F5807F09BFEF
:10974000CB6993640343D36418BFD064054B4A6864
:109750005A672A6B42F002022A639A6942F408525D
:10976000B8E700BF002800400008005890F82C20FF
:10977000012A03464FF0020012D00A4A83F82D0056
:10978000CA21516253215162916941F020019161D6
:10979000FF2151620020012283F82D2083F82C0044
:1097A000704700BF0028004090F82C20012A034693
:1097B0004FF0020019D00D4A83F82D00CA215162E2
:1097C0005321516291690A4841F080019161D0F8BA
:1097D000801041F48021C0F88010FF2151620020E8
:1097E000012283F82D2083F82C00704700280040C8
:1097F00000080058064B5A6D520610B5044603D5B2
:109800004022DA65FAF7B6FC012384F82D3010BD4A
:10981000002800407047890001F1804101F5314185
:109820000A607047890001F1804101F53141086803
:10983000704700002DE9F3471F46894690460446CD
:10984000FAF720FA0A9D3D442D1AFAF71BFA264B27
:109850001E68C6F3CB366E43824601962268936833
:1098600039EA03030CBF01230023434501D1002043
:109870002EE07B1CF3D0FAF705FAA0EB0A00A84211
:1098800029D323685A6822F0E0025A606268B2F570
:10989000827F0AD1A268B2F5004F02D0B2F5806F84
:1098A00003D11A6822F040021A60A26AB2F5005F82
:1098B00007D11A6822F400521A601A6842F4005262
:1098C0001A60012384F85D30002384F85C300320A3
:1098D00002B0BDE8F087019A019B002A03F1FF3333
:1098E000019308BF1546B9E7A80300202DE9F74FFB
:1098F000994600238DF80330044688461746FAF748
:10990000C1F90C9D4D442D1AFAF7BCF92C4BD4F833
:1099100000B01E6823235E43360D6E4382460196D7
:109920002268936803EA0803BB4201D100203AE0B1
:10993000B8F5C06F07D137B99BF80C30DBB28DF8A2
:1099400003309DF80330B9F1FF3FEAD0FAF79AF9F6
:10995000A0EB0A00A84229D323685A6822F0E0024B
:109960005A606268B2F5827F0AD1A268B2F5004FF0
:1099700002D0B2F5806F03D11A6822F040021A605B
:10998000A26AB2F5005F07D11A6822F400521A6089
:109990001A6842F400521A60012384F85D300023F3
:1099A00084F85C30032003B0BDE8F08F019A019B7E
:1099B000002A03F1FF33019308BF1546B0E700BF4B
:1099C000A803002073B50B4600920D4616464FF4CF
:1099D000C05100220446FFF789FF024630B1236ED2
:1099E00043F020032366032002B070BD00962B468F
:1099F00080212046FFF71EFF02460028EFD1009687
:109A00002B464FF4C0612046FFF770FF0028EBD0D3
:109A1000E5E74368B3F5827FF7B504460E4617467F
:109A20000BD18368B3F5004F02D0B3F5806F04D13A
:109A30002268136823F04003136000973346002226
:109A400080212046FFF7F6FE054628B1236E43F03D
:109A500020032366032514E06368B3F5827F10D1E9
:109A6000A368B3F5004F02D0B3F5806F09D100971A
:109A7000334600224FF4C0612046FFF737FF00282D
:109A8000E4D1284603B0F0BDF8B5044600287ED0E6
:109A9000436A002B50D14268B2F5827F00D0C36187
:109AA00094F85D3003F0FF0223B984F85C2020466F
:109AB000F9F7E6FB2268E068022384F85D3013685A
:109AC000B0F5E06F23F0400313604FF0000337D987
:109AD0001D46B0F5706F18BFA362A7686368A169DF
:109AE000A66A07F4044703F482733B43276907F02F
:109AF00002073B43676907F001073B4301F4007726
:109B00003B43E76907F038073B43276A07F08007C4
:109B10003B4306F400573B43B6F5005F136014D196
:109B2000236B8BBBB0F5E06F0DD902232363136861
:109B300043F40063136008E00023C0E90433AFE797
:109B40004FF48055C7E701232363636A676B03F013
:109B5000100307F0080700F470603B43090C03434F
:109B600001F004010B432B43B6F5005F536004BFC3
:109B7000A38D1361D36923F40063D3610020012313
:109B8000206684F85D30F8BD022BDED1CFE70120DE
:109B9000F9E7000070B5044690F85C00012800F079
:109BA000CF80012084F85C0094F85D00666801288D
:109BB000C5B20AD0B6F5827F40F0C080A068002808
:109BC00040F0BC80042D40F0B980002951D0002A1B
:109BD0004FD0002B4DD094F85D00A16304281CBF2A
:109BE000052084F85D0000202066C4E91300A06A07
:109BF000E387B0F5005F2168A3872264A4F84430AE
:109C0000A4F8463007D1086820F4005008600868BE
:109C100040F400500860486820F4C0404860E068A4
:109C2000B0F5E06FA06D29D94B6823F480534B60E9
:109C300094F85D30434E444D042B444B18BF1D46F1
:109C4000434B18BF3346C0E90B35424B43630023F7
:109C50008363B4F846300C319BB2FEF785FA0346B5
:109C6000002848D0236E43F010032366012384F8B4
:109C70005D300120002384F85C3070BD4D6845F4F0
:109C800080554D60656DAD69B5F5806F0AD113F0F3
:109C9000010F4B681ED123F480434B60E38FC3F365
:109CA0004E03E3878369B3F5806FC1D14B6823F41A
:109CB00080534B60B4F8463013F0010F4B6811D15C
:109CC00023F400534B60B4F84630C3F34E03A4F8BA
:109CD0004630ADE743F480434B60E38FC3F34E035C
:109CE0000133DEE743F400534B60B4F84630C3F36E
:109CF0004E030133EBE72268606D516841F00101CA
:109D00005160C0E90B33C0E90D33E38FA16B9BB207
:109D10000C32FEF729FA0028A4D123681A685206EB
:109D20005EBF1A6842F040021A605A6842F0200290
:109D30005A605A6842F002025A609BE7022099E793
:109D400002209AE78D9E00085D9D0008699D00082D
:109D5000979D0008759D00087047704708B5806A98
:109D6000FFF7FBFF08BD704708B5806AFFF7FBFFF0
:109D700008BD7047806A026808B5536823F0030382
:109D80005360036E43F010030366012380F85D30D7
:109D9000FFF7EFFF08BD7FB5064600230393846AF3
:109DA0008DF80B30F9F76EFF33681B689A0605468D
:109DB00068D42268536823F020035360A36AB3F584
:109DC000005F13D101220090642311462046FFF763
:109DD00031FD18B1236E43F002032366E368266861
:109DE000B3F5E06F2ED9F3680393039BA268236851
:109DF000002A43D16268B2F5827F3FD15A6822F0CF
:109E000003025A6064212A462046FFF702FE08B189
:109E1000202323660023A4F846302268012384F817
:109E20005D309368DB0606D5236E43F0020323669C
:109E30004FF6EF739360236E23B32046FFF799FF2D
:109E400004B070BD337BDBB28DF80B309DF80B3066
:109E5000236B022BCAD101220095642311462046B0
:109E6000FFF7E8FC18B1236E43F002032366337B4F
:109E7000DBB28DF80B309DF80B30B7E75A6822F053
:109E80000102BEE72046FFF767FFD9E77FB5064628
:109E900000230393846A8DF80B30F9F7F3FE3368DF
:109EA0001B68990605465ED42268536823F0200398
:109EB0005360A36AB3F5005F1BD1E368B3F5E06FAD
:109EC0003ED1236B012B3BD1009064234FF40072F1
:109ED0004FF4C0612046FFF709FD18B1236E43F02F
:109EE0000203236623681B7BDBB28DF80B309DF8E1
:109EF0000B302A4664212046FFF764FD18B1236E1B
:109F000043F02003236623685A6822F003025A6054
:109F10000022E287A4F84620012284F85D209A6896
:109F2000D20606D5226E42F0020222664FF6EF728A
:109F30009A60236EBBB12046FFF71BFF04B070BDD3
:109F4000009564234FF480624FF4C0612046FFF710
:109F5000CDFC18B1236E43F0020323662368DB684F
:109F60000393039BC5E72046F8F7A6FCE6E700004D
:109F7000036830B559689A6802F04105012D85B033
:109F8000044606D14D0604D5C36C05B0BDE830408B
:109F90001847950704D5080602D5236D2046F4E737
:109FA00012F4B07F59D08D0657D550060FD594F8CE
:109FB0005D0003284FF0000549D0206E40F00400FA
:109FC00020660095D86800909868009000989506E3
:109FD0000CD5206E40F001002066002002909868A9
:109FE0000290186820F0400018600298D00508D54B
:109FF000226E42F008022266002203929A680392BF
:10A00000039A226E4AB35A6822F0E0025A60012293
:10A0100084F85D208A0722D05A68A06D22F00302DE
:10A020005A6040B1104B8363FEF717F918B1236EE5
:10A0300043F040032366606D78B10B4B8363FEF7FA
:10A040000CF950B1236E43F04003236605E00195FF
:10A05000DA6801929B680193019B05B030BD2046F0
:10A06000FFF787FEF9E700BF6DA0000808B5806A1A
:10A070000023A0F84630C387FFF77BFE08BD000031
:10A08000034AD2F8903043F40043C2F8903070474E
:10A0900000040058034AD2F8903023F40043C2F879
:10A0A0009030704700040058074B1A6822F04002B5
:10A0B0001A6040F441704FF4B85218605A601A6840
:10A0C00042F040021A6070470000015837B505465B
:10A0D00000284ED0837903F0FF046BB1032C0BD022
:10A0E000254B4FF400629A612868FFF7DDFF0024DA
:10A0F00001232B71AC602FE000236B712846F9F728
:10A10000D5FC1E4AD2F8903043F48053C2F8903008
:10A11000002CE5D102234FF0B042AB71D2F894305D
:10A1200023F40043C2F89430154B1B681C214B43A9
:10A13000DB0C64214B430193019B93B90124AC6078
:10A14000FFF79EFF0C4B9A6842F400629A604FF44E
:10A1500000629A61002CC7D00123AB71204603B086
:10A1600030BD019B013B0193D2F894305B04E3D4F2
:10A17000E6E70124F2E700BF000400580008005899
:10A18000A803002037B5174D2B6802461C20434317
:10A19000DB0C6420434314480193019B93B90120D5
:10A1A0009060114C21732B681C214B43DB0C642104
:10A1B0004B430193019B6BB9012090600A4BDB6814
:10A1C00003B030BD019B013B019383689C07E4D53C
:10A1D0000020E6E7019B013B0193A368DB07E9D57B
:10A1E000ECE700BFA80300200000015837B5184D68
:10A1F0002B6802461C204343DB0C64204343154874
:10A200000193019BA3B901209060124CFF2323739B
:10A210002B681C256B43DB0C64256B430193019B6E
:10A2200073B9012090600B4BDB680B7003B030BD3D
:10A23000019B013B019383689C07E2D50020E4E782
:10A24000019B013B0193A368DB07E8D5EBE700BF67
:10A25000A8030020000001580E4B0F491B6818226C
:10A26000534382B01B0D6422534301934B69019AFF
:10A27000C3F3800322B902238360012002B0704738
:10A28000019A013A01924A69920701D5002BEDD15A
:10A290000020F3E7A80300200004005807B5037965
:10A2A000012B0FD10A4B1B68182253431B0C01933F
:10A2B000FFF7F0FE019B013B0193019B002BF9D1BD
:10A2C000FFF7DEFE03B05DF804EBFFF7C5BF00BF8C
:10A2D000A8030020F8B51E468379012B15460446D5
:10A2E0000F46DAB22DD14379012B2AD002234271D5
:10A2F0008371FFF7D3FF0D212046FFF7CBFEFFF759
:10A3000041FF390A2046FFF73DFFF9B22046FFF72B
:10A3100039FF2E44B5420ED12046FFF7B1FEFFF7BC
:10A320009BFFA06801230038A3714FF0000318BF02
:10A3300001206371F8BD15F8011B2046FFF722FFCD
:10A34000E8E70220F6E7F8B51E468379012B1546AB
:10A3500004460F46DAB22FD14379012B2CD042713B
:10A36000FFF79CFF1D212046FFF794FEFFF70AFF31
:10A37000390A2046FFF706FFF9B22046FFF702FF31
:10A3800000212046FFF7FEFE2E44B5420ED12046A6
:10A39000FFF776FEFFF760FFA06801230038A37186
:10A3A0004FF0000318BF01206371F8BD2946204615
:10A3B000FFF71CFF0135E8E70220F6E7F8B51F4676
:10A3C0008379012B154604460E46DAB22CD1437927
:10A3D000012B29D04271FFF761FF06F0EF03A3F1D3
:10A3E000840253425341237131462046FFF752FE07
:10A3F000FFF7C8FE2F44AF4210D1FFF741FE842E75
:10A4000002D02046FFF728FFA06801230038A3717F
:10A410004FF0000318BF01206371F8BD15F8011B50
:10A420002046FFF7AFFEE6E70220F6E7F8B51E4646
:10A430008379012B154604460F46DAB227D14379BA
:10A44000012B24D04271FFF729FF39462046FFF740
:10A4500021FEFFF797FE00212046FFF793FE2E44D2
:10A46000B5420ED12046FFF70BFEFFF7F5FEA068C0
:10A4700001230038A3714FF0000318BF012063715E
:10A48000F8BD29462046FFF7B1FE0135E8E7022076
:10A49000F6E737B50023ADF8043001AA02231221F4
:10A4A0000546FFF7C3FFBDF80440022364BA01AAC2
:10A4B000A4B219462846FFF781FFE20702D52846D5
:10A4C0000AF09EF8A30702D528460AF09FF8600715
:10A4D00002D528460AF0C4F8210702D528460AF01A
:10A4E000C5F8E20602D528460AF0C6F8A30602D54A
:10A4F00028460AF0AFF8600602D528460AF08CF824
:10A50000210606D514F4807118BF012128460AF0EF
:10A5100089F8A20502D528460AF094F8630402D50A
:10A5200028460AF0AFF803B030BDF8B51E4683796F
:10A53000012B154604460F46DAB227D14379012B89
:10A5400024D04271FFF7AAFE0E212046FFF7A2FD9C
:10A55000FFF718FE39462046FFF714FE2E44B54299
:10A560000ED12046FFF78CFDFFF776FEA068012391
:10A570000038A3714FF0000318BF01206371F8BDCC
:10A5800015F8011B2046FFF7FDFDE8E70220F6E77E
:10A59000F8B51E468379012B154604460F46DAB2FC
:10A5A0002BD14379012B28D04271FFF777FE1E2172
:10A5B0002046FFF76FFDFFF7E5FD39462046FFF720
:10A5C000E1FD00212046FFF7DDFD2E44B5420ED10E
:10A5D0002046FFF755FDFFF73FFEA0680123003836
:10A5E000A3714FF0000318BF01206371F8BD294625
:10A5F0002046FFF7FBFD0135E8E70220F6E7000003
:10A60000036A23F001030362036A70B54468826938
:10A610000D6822F4803222F073022A438D6823F001
:10A6200002032B43124DA84206D0124EB04203D073
:10A63000A6F58066B04214D1CE6823F008033343F8
:10A64000A84223F0040306D00B4DA84203D005F521
:10A650008065A84205D124F44075D1E9054634430C
:10A660002C43446082614A684263036270BD00BF4C
:10A67000002C01400048014000440140036A23F4DB
:10A6800080730362036A426870B5C4690D6824F47C
:10A69000803424F073042C438D6823F4007343EA60
:10A6A00005230F4DA8420ED1CD6823F4006343EA81
:10A6B000052323F48063D1E9055622F44052354343
:10A6C00042EA051206E0074DA842F4D005F5806580
:10A6D000A842F0D042604A68C461C263036270BDA0
:10A6E000002C014000440140036A23F480530362BC
:10A6F000026A30B54468C3690D6823F0807323F49F
:10A70000E64343EA05238D6822F4005242EA05320B
:10A710000A4DA84207D005F5C055A84203D005F55B
:10A720008065A84204D14D6924F4804444EA85142C
:10A730004460C3614B680364026230BD002C014079
:10A74000036A23F480330362026A30B54468436DC0
:10A750000D6823F4803323F070032B438D6822F4BB
:10A76000003242EA05420B4DA84207D005F5C0551C
:10A77000A84203D005F58065A84204D14D6924F4B0
:10A78000803444EA0524446043654B688365026273
:10A7900030BD00BF002C0140036A23F48013036224
:10A7A000026A30B54468436D0D6823F0807323F46A
:10A7B000E04343EA05238D6822F4001242EA055281
:10A7C0000A4DA84207D005F5C055A84203D005F5AB
:10A7D0008065A84204D14D6924F4802444EA85248C
:10A7E000446043654B68C365026230BD002C014084
:10A7F000704710B5846A626A82420BD101232377C5
:10A80000D2690AB984F83E302046F9F7DDF8002312
:10A81000237710BDA36A834208D102222277DB6925
:10A82000002BF1D1012384F83F30EDE7E36A834246
:10A8300008D104222277DB69002BE5D1012384F8BB
:10A840004030E1E7236B8342DED108222277DB69C7
:10A85000002BD9D1012384F84130D5E7704710B5DA
:10A86000846A636A834207D1012323772046FFF776
:10A87000F5FF0023237710BDA36A834201D1022391
:10A88000F3E7E36A834201D10423EEE7236B8342BB
:10A89000ECD10823E9E7704710B5846A636A834204
:10A8A00009D10123237784F83E302046FFF7F3FFD8
:10A8B0000023237710BDA36A834205D102232377A7
:10A8C000012384F83F30F0E7E36A83424FF001034D
:10A8D00004D10422227784F84030E6E7226B8242DA
:10A8E00003BF0822227784F8413084F83D30DCE74A
:10A8F0001A4A0368904210B502D0B0F1804F09D1D6
:10A900004C6823F07003904243EA040309D0B0F18D
:10A91000804F06D0124A904203D002F580629042E6
:10A9200003D1CA6823F4407313434A6923F08003B8
:10A93000134303608B68C3620B688362074B9842C2
:10A9400007D003F5C053984203D003F580639842C3
:10A9500001D10B6903630123436110BD002C014049
:10A960000044014010B5044650B390F83D3003F068
:10A97000FF021BB980F83C20F9F75CFA022320683B
:10A9800084F83D30211DFFF7B3FF012384F84830E0
:10A99000002084F83E3084F83F3084F8403084F85A
:10A9A000413084F8423084F8433084F8443084F8ED
:10A9B000453084F8463084F8473084F83D3010BD87
:10A9C0000120FCE710B5044650B390F83D3003F089
:10A9D000FF021BB980F83C20FFF70AFF0223206822
:10A9E00084F83D30211DFFF783FF012384F84830B0
:10A9F000002084F83E3084F83F3084F8403084F8FA
:10AA0000413084F8423084F8433084F8443084F88C
:10AA1000453084F8463084F8473084F83D3010BD26
:10AA20000120FCE7036A23F010030362036A426813
:10AA300070B584690D6824F0807424F4E64444EA17
:10AA400005248D6823F0200343EA05130F4DA84227
:10AA50000ED1CD6823F0800343EA051323F04003B1
:10AA6000D1E9055622F44062354342EA850206E008
:10AA7000074DA842F4D005F58065A842F0D04260A9
:10AA80004A6884618263036270BD00BF002C01408C
:10AA90000044014038B590F83C30012B044673D097
:10AAA00001200C2A84F83C004ED008D8042A2BD070
:10AAB000082A39D0BAB1002384F83C3038BD102AB6
:10AAC00052D0142AF7D12068FFF766FE436D0A6959
:10AAD00043F400634365436D23F480634365436D32
:10AAE00043EA02234EE02068FFF78AFD83690A6982
:10AAF00043F008038361836923F00403836183695E
:10AB0000134383610020D6E72068FFF78BFF83693A
:10AB10000A6943F400638361836923F4806383617A
:10AB2000836943EA0223ECE72068FFF7A7FDC369C6
:10AB30000A6943F00803C361C36923F00403C361D6
:10AB4000C3691343C361DDE72068FFF7CDFDC36927
:10AB50000A6943F40063C361C36923F48063C3617A
:10AB6000C36943EA0223EDE72068FFF7E9FD436D7F
:10AB70000A6943F008034365436D23F0040343650A
:10AB8000436D13434365BDE7022097E710B5846822
:10AB90000A4324F47F4442EA03222243826010BD28
:10ABA00038B590F83C30012B04464FF0020000F01D
:10ABB000958084F83D000122206884F83C20856857
:10ABC000474B2B4083600B68602B54D037D8402B09
:10ABD0006BD019D8202B0DD00AD833F0100109D032
:10ABE000012384F83D30002384F83C30104638BD02
:10ABF000302BF5D1826822F4401222F070021A4301
:10AC000042F0070282602BE0502BE9D14A68CD6800
:10AC1000016A036A23F001030362836921F00A01D8
:10AC200023F0F00343EA05130A4383610262836859
:10AC300023F4401323F0700343F057030FE0B3F500
:10AC4000805F0DD0B3F5005F0CD0702BC8D1CB68FE
:10AC5000D1E90121FFF79AFF836843F0770383600E
:10AC60000022BDE7CB68D1E90121FFF78FFF8368A0
:10AC700043F48043F3E7036A4D68C96823F0100387
:10AC800003628269036A22F4704223F0A00343EA5C
:10AC9000051342EA013282610362836823F44013A0
:10ACA00023F0700343F06703D9E74A68CD68016A6F
:10ACB000036A23F001030362836921F00A0123F090
:10ACC000F00343EA05130A4383610262836823F4B5
:10ACD000401323F0700343F04703C0E7024685E7C3
:10ACE0008800CEFF036A01F01F0110B501248C40DB
:10ACF00023EA04030362036A8A401A43026210BD16
:10AD0000082908B518D005D859B1042911D090F8F0
:10AD1000433008E00C2912D01029F8D190F84230C5
:10AD200001E090F83E30013B18BF012353B10120F0
:10AD300041E090F83F30F6E790F84030F3E790F8C4
:10AD40004130F0E708294FF002033CD007D869B141
:10AD5000042931D0042980F84330E8D12EE00C29B1
:10AD600038D01029F6D180F84230E0E7026880F848
:10AD70003E30D36843F002030068D3600122FFF73E
:10AD8000B1FF1B4A90422CD01A4B984229D003F5B0
:10AD90008063984225D0B0F1804F07D18268164B6E
:10ADA0001340062B06D0B3F5803F03D0036843F071
:10ADB00001030360002008BD80F83F300268D368BB
:10ADC00043F00403D8E7026880F84030D36843F0CA
:10ADD0000803D1E7026880F84130D36843F01003DC
:10ADE000CAE7436C904243F400434364D6D0D2E7B1
:10ADF000002C01400044014007000100FFF780BF24
:10AE000038B50D46082D044611461BD005D85DB156
:10AE1000042D14D094F8430008E00C2D15D0102D0B
:10AE2000F8D190F8420001E090F83E00A0F1020C49
:10AE3000DCF1000040EB0C0050B1022076E090F80D
:10AE40003F00F3E790F84000F0E790F84100EDE7AD
:10AE5000082D1AD007D86DB1042D13D094F84320D3
:10AE6000012A19D00CE00C2D27D0102DF6D194F822
:10AE700042000CE094F83E20501E424242415AB932
:10AE8000012053E094F83F20F6E794F84000421E7A
:10AE9000504250410028F3D00029F1D0002BEFD0D0
:10AEA000082D4FF0020256D00AD885B1042D3ED0AD
:10AEB000042D84F84320E3D13BE094F84100E6E719
:10AEC0000C2D5CD0102DF3D184F84220D8E7606AB5
:10AED00084F83E203A4AC2623A4A02633A4A4263DE
:10AEE00022683432FDF740F90028C9D12268D368BE
:10AEF00043F400732068D36029460122FFF7F2FE75
:10AF0000324A904250D0324B98424DD003F5806384
:10AF1000984249D0B0F1804F4DD182682D4B1340FB
:10AF2000062B02D0B3F5803F45D1002038BD84F810
:10AF30003F20A06A224AC262224A0263224A426336
:10AF400022683832FDF710F9002899D12268D368B9
:10AF500043F48063CEE7E06A84F84020184AC26276
:10AF6000184A0263184A426322683C32FDF7FCF833
:10AF7000002885D12268D36843F40063BAE7206BC8
:10AF800084F841200E4AC2620E4A02630E4A4263AE
:10AF900022684032FDF7E8F800287FF471AF22689C
:10AFA000D36843F48053A5E7436C904243F40043D5
:10AFB0004364B2D0AEE7036843F001030360B4E733
:10AFC000F3A700085FA8000899A80008002C01401A
:10AFD0000044014007000100FFF712BF082938B5FF
:10AFE00004460D464FD004D861B1042944D0012055
:10AFF00038BD0C29FBD10268006BD36823F4805361
:10B00000D36005E00268406AD36823F40073D3601C
:10B01000FDF723F9206800222946FFF763FE2A4B3B
:10B02000984207D003F5C053984203D003F58063DC
:10B0300098420DD1026A41F211131A4208D1026AF4
:10B0400040F244431A4202BF436C23F4004343647A
:10B05000026A41F211131A4208D1026A40F24443D3
:10B060001A4202BF036823F00103036001238DB974
:10B0700084F83E300020BBE70268806AD36823F47E
:10B080008063D360C4E70268C06AD36823F40063B6
:10B09000D360BDE70C2D13D007D8042D0AD0082D9E
:10B0A0000BD0012384F84330E4E7102DF9D184F864
:10B0B0004230DFE784F83F30DCE784F84030D9E7FE
:10B0C00084F84130D6E700BF002C0140FFF786BF6F
:10B0D00070B590F83C30012B02464FF0020020D0B2
:10B0E00082F83D000F4D106843688468A84202BF93
:10B0F0004E6823F4700333430E6823F07003334328
:10B10000A842436002D0B0F1804F04D1896824F096
:10B1100080030B4383600123002082F83D3082F8D6
:10B120003C0070BD002C0140026852E8003F23F053
:10B13000C00342E8003102680029F5D102F108039A
:10B1400053E8003F23F4000302F1080C4CE80031FF
:10B150000029F3D12023C0F88830704710B5026869
:10B1600052E8003F23F4907342E80031026800295E
:10B17000F5D10F4C02F1080353E8003F234002F1E0
:10B18000080C4CE800310029F4D1C36E012B07D123
:10B1900052E8003F23F0100342E800310029F7D1C4
:10B1A0002023C0F88C300023C366436710BD00BF66
:10B1B000FEFFFFEFF8B504461346D4F88850202D63
:10B1C00032D1F1B1EAB1E06FA4F85620A4F85420CE
:10B1D00000262122C4F890602165C4F888202268E6
:10B1E00088B1124FC762124F0763124F2832C0E96D
:10B1F0000D76FCF7B9FF30B11023C4F89030C4F8D5
:10B2000088500120F8BD236840221A62226802F1AA
:10B21000080353E8003F43F0800302F1080141E8CE
:10B2200000300028F3D1EDE70220EBE739B2000847
:10B2300081B200088DB2000808B50346806A1B6819
:10B240001B6813F0200317D1A0F85630026802F1F2
:10B25000080353E8003F23F08003083242E800313E
:10B2600002680029F2D152E8003F43F0400342E86F
:10B2700000310029F7D108BDF9F7B0F8FBE77047B6
:10B2800008B5806AFFF7FBFF08BD7047806A38B5D4
:10B290000468D0F88830D0F88C50A268120606D521
:10B2A000212B04D10023A0F85630FFF73DFFA368FF
:10B2B0005B0606D5222D04D10023A0F85E30FFF7EF
:10B2C0004DFFD0F8903043F01003C0F89030FFF7F6
:10B2D000DCFF38BD08B5806A0023A0F85E30A0F816
:10B2E0005630FFF7D2FF08BD704700000368D969E8
:10B2F0001A682DE9F04140F60F0631429D68044678
:10B3000010D18E0640F1978002F0200605F080579C
:10B310003E4300F09080436F002B00F08580BDE835
:10B32000F0411847AB4EAC482E401040304300F07F
:10B330008280CF0709D5D00507D501201862D4F83F
:10B34000900040F00100C4F890008F0709D5E8078D
:10B3500007D502201862D4F8900040F00400C4F829
:10B3600090004F0709D5E80707D504201862D4F8E4
:10B37000900040F00200C4F890000F070BD502F0D7
:10B380002000304307D008201862D4F8900040F025
:10B390000800C4F890000E050AD5500108D54FF4F6
:10B3A00000601862D4F8903043F02003C4F8903065
:10B3B000D4F89030002B37D08B0609D502F020024C
:10B3C00005F080552A4303D0636F0BB120469847A0
:10B3D0002668D4F89020B36802F0280203F04003F6
:10B3E00053EA0205204621D0FFF7B8FEB3685F0696
:10B3F00017D5226802F1080353E8003F23F0400309
:10B40000083242E800310029F3D1D4F8800040B17D
:10B41000724B8363FCF721FF30B1D4F88000836B5B
:10B420007DE72046FFF731FFBDE8F081FFF72DFFF4
:10B43000C4F89050F8E7E06E012840F08980CE060D
:10B4400040F18680D00640F1838010221A629A680B
:10B4500051064BD5D4F8802011684A6892B2002A70
:10B46000E2D0B4F85C009042DED9A4F85E200A680D
:10B4700092062FD453E8002F22F4807243E8002173
:10B480000029F7D103F1080252E8002F22F001024F
:10B4900003F1080040E800210029F3D103F108027C
:10B4A00052E8002F22F0400203F1080040E800219A
:10B4B0000029F3D12022C4F88C20E16653E8002F44
:10B4C00022F0100243E800210029F7D1D4F88000CF
:10B4D000FCF78EFE02232367B4F85E30B4F85C10EC
:10B4E000C91A89B22046FFF7FFFE9DE7B4F85E2037
:10B4F000B4F85E00B4F85C1080B292B2002893D029
:10B50000891A89B200298FD053E8002F22F4907253
:10B5100043E800200028F7D1314D03F1080252E83A
:10B52000002F2A4003F1080646E800200028F4D145
:10B530002022C4F88C206067E06653E8002F22F0D8
:10B54000100243E800200028F7D102232367C9E74F
:10B55000CF0209D56E0207D54FF4801220461A6239
:10B56000BDE8F04100F0A0BD08060BD502F0800058
:10B5700005F40005284305D0A36F002B3FF454AF1A
:10B580002046CCE64F0611D556060FD553E8002FBE
:10B5900022F0400243E800210029F7D12023C4F81B
:10B5A0008830A1672046F8F719FF3DE70D0206D560
:10B5B000500004D52046BDE8F04100F077BDCB0136
:10B5C0007FF532AF002ABFF62FAF2046BDE8F0412D
:10B5D00000F06BBD0100001020010004D5B200088E
:10B5E000FEFFFFEFD0F88C20B0F86010222A08B5DB
:10B5F000036855D15B6A826D0B401370836D013314
:10B600008365B0F85E30013B9BB2A0F85E30B0F8C5
:10B610005E309BB2002B42D1026852E8003F23F417
:10B62000907342E8003103680029F5D103F1080264
:10B6300052E8002F22F0010203F1080C4CE800212F
:10B640000029F3D12022C0F88C20184A4167934288
:10B65000016705D1C26E012A0ED0F8F7CDFE1EE0BB
:10B660005A681102F6D553E8002F22F0806243E8B1
:10B6700000210029F7D1EDE70022C26653E8002F30
:10B6800022F0100243E800210029F7D1DA69B0F86E
:10B690005C10D20644BF10221A62FFF725FE08BDD7
:10B6A0009A6942F008029A61F9E700BF0080004001
:10B6B000D0F88C20B0F86010222A08B5036852D167
:10B6C0005A6A1140826D22F8021B8265B0F85E2032
:10B6D000013A92B2A0F85E20B0F85E2092B2002A41
:10B6E00040D153E8002F22F4907243E80021002952
:10B6F000F7D103F1080252E8002F22F0010203F112
:10B70000080C4CE800210029F3D12022C0F88C203D
:10B71000174A41679342016705D1C26E012A0ED0D4
:10B72000F8F76AFE1EE05A681102F6D553E8002FBA
:10B7300022F0806243E800210029F7D1EDE70022E2
:10B74000C26653E8002F22F0100243E800210029CE
:10B75000F7D1DA69B0F85C10D20644BF10221A6241
:10B76000FFF7C2FD08BD9A6942F008029A61F9E745
:10B77000008000402DE9F84F0368B0F86060D3F80E
:10B780001CB01F689D68D0F88C20222A044640F027
:10B79000B980B0F8683043B1DFF87491DFF874A174
:10B7A0004FF000081BF0200F20D1B4F85E309BB2A0
:10B7B000D3B1B4F868209A4216D9226802F108037E
:10B7C00053E8003F23F08053083242E800312268FA
:10B7D0000029F2D1504B636752E8003F43F0200349
:10B7E00042E800310029F7D1BDE8F88F2368A26D47
:10B7F0005B6A33401370A36D0133A365B4F85E3008
:10B80000013B9BB2A4F85E302368D3F81CB01BF058
:10B81000070F2ED01BF0010F09D0F90507D5012223
:10B820001A62D4F8902042F00102C4F890201BF074
:10B83000020F09D0EA0707D502221A62D4F8902035
:10B8400042F00402C4F890201BF0040F09D0E8076E
:10B8500007D504221A62D4F8903043F00203C4F8EA
:10B860009030D4F8903023B12046FFF70EFDC4F895
:10B870009080B4F85E309BB2002B93D1226852E8DE
:10B88000003F23F4807342E8003123680029F5D19A
:10B8900003F1080252E8002F02EA090203F108004E
:10B8A00040E800210029F3D120225345C4F88C2020
:10B8B000616721670AD05A68110207D553E8002F43
:10B8C00022F0806243E800210029F7D1E26E012ACC
:10B8D00014D10022E26653E8002F22F0100243E860
:10B8E00000210029F7D1DA69B4F85C10D20644BF10
:10B8F00010221A622046FFF7F7FC53E72046F8F7BC
:10B900007BFD4FE79A6942F008029A616CE700BF3D
:10B91000FEFFFFEF00800040E5B500082DE9F84F7D
:10B920000368B0F86060D3F81CB01F689D68D0F859
:10B930008C20222A044640F0B780B0F8683043B12A
:10B94000DFF87091DFF870A14FF000081BF0200FB6
:10B9500020D1B4F85E309BB2D3B1B4F868209A42DB
:10B9600016D9226802F1080353E8003F23F0805300
:10B97000083242E8003122680029F2D14F4B636758
:10B9800052E8003F43F0200342E800310029F7D19C
:10B99000BDE8F88F2368A26D596A314022F8021B76
:10B9A000A265B4F85E20013A92B2A4F85E20D3F802
:10B9B0001CB01BF0070F2ED01BF0010F09D0F905AA
:10B9C00007D501221A62D4F8902042F00102C4F88F
:10B9D00090201BF0020F09D0EA0707D502221A6255
:10B9E000D4F8902042F00402C4F890201BF0040F19
:10B9F00009D0E80707D504221A62D4F8903043F042
:10BA00000203C4F89030D4F8903023B12046FFF7F9
:10BA10003CFCC4F89080B4F85E309BB2002B95D10A
:10BA2000226852E8003F23F4807342E80031236823
:10BA30000029F5D103F1080252E8002F02EA0902B9
:10BA400003F1080040E800210029F3D120225345EA
:10BA5000C4F88C20616721670AD05A68110207D5A3
:10BA600053E8002F22F0806243E800210029F7D13B
:10BA7000E26E012A14D10022E26653E8002F22F080
:10BA8000100243E800210029F7D1DA69B4F85C100C
:10BA9000D20644BF10221A622046FFF725FC55E764
:10BAA0002046F8F7A9FC51E79A6942F008029A612A
:10BAB0006EE700BFFEFFFFEF00800040B1B6000858
:10BAC00038B5044603682169A2681D68C0690A4345
:10BAD00061690A437749024329400A431A605A6858
:10BAE000E16822F440520A435A60734AA1699342C2
:10BAF0001CBF226A11439A6822F06E4222F430621F
:10BB00000A439A60DA6A616A22F00F020A43DA6233
:10BB10006A4A934219D14FF0B043694AD3F888304A
:10BB200003F0030343F44033934200F0B480B3F1D5
:10BB3000031F24D0013A934240F0B580B0F5004F86
:10BB400040F08F80FCF746FF6EE05E4A93421CD1C6
:10BB50004FF0B0435C49D3F8883003F00C0343F452
:10BB600040228A4200F0978006D8002B7CD0574BA9
:10BB70009A42E3D0012026E0B2F10C1FFAD1B0F5D1
:10BB8000004F53D04FF4004075E04B4A9342F1D13F
:10BB90004FF0B043D3F8883003F44063B3F5006F3F
:10BBA00018D006D85BB1B3F5806FE3D1FCF712FF74
:10BBB00007E0B3F5406FDDD14FF400400BE0FDF737
:10BBC00001FB40B900204FF00113A3660023C4E934
:10BBD0001D3338BD3E4865683E4B626A05EB450142
:10BBE00033F81220B0FBF2F39942C3D8B3EB053F10
:10BBF000C0D800231946F6F757FC090241EA106144
:10BC00006B080002C0182A464FF0000341F1000102
:10BC1000F6F74AFC304BA0F540729A42AAD8236846
:10BC2000D860CFE7FDF7CEFA0028CBD06168294B6A
:10BC3000626A33F81220B0FBF2F24B0803EB4203C6
:10BC40004FF6EF72B3FBF1F3A3F11001914291D8DB
:10BC500023F00F02216892B2C3F342031343CB6077
:10BC6000B0E7FCF7B7FE04E0B0F5004FDAD0FDF71F
:10BC7000A9FA0028A6D06368616A164A32F8112032
:10BC8000B0FBF2F000EB5300B0FBF3F04FF6EF73B4
:10BC9000A0F11002C1E7B0F5004F0D48EBD1C5E7A8
:10BCA000FDF7A0FAC0E7B0F5004FF9D0FDF79AFA1A
:10BCB000DFE700BFF369FFCF00800040003801409C
:10BCC000020003000044004008000C0004000C00C7
:10BCD0000024F400B8710308FFFC0F00836ADA0740
:10BCE00010B506D50168C46A4A6822F400322243BE
:10BCF0004A609C0706D50168046B4A6822F48032CA
:10BD000022434A60590706D50168446B4A6822F409
:10BD1000802222434A601A0706D50168846B4A686C
:10BD200022F4004222434A60DC0606D50168C46B57
:10BD30008A6822F4805222438A60990606D50168F7
:10BD4000046C8A6822F4005222438A605A060FD596
:10BD50000168446C4A6822F480122243B4F5801FC3
:10BD60004A6005D14A68846C22F4C00222434A60CA
:10BD70001B0606D50268C16C536823F400230B43ED
:10BD8000536010BD2DE9F843DDF8209005460F46BD
:10BD9000164698462A68D36937EA03030CBF012385
:10BDA0000023B34201D0002029E0B9F1FF3FF2D0D7
:10BDB000F7F768FFA0EB080048452C6802D8B9F1F6
:10BDC000000F1ED154E8003F23F4D07344E8003242
:10BDD000002AF7D104F1080353E8003F23F00103E0
:10BDE00004F1080141E80032002AF3D12023C5F80C
:10BDF0008830C5F88C30002385F884300320BDE8F6
:10BE0000F88323685A07C5D5E3691B05C2D54FF4EB
:10BE10000063236254E8003F23F4D07344E8003207
:10BE2000002AF7D104F1080353E8003F23F001038F
:10BE300004F1080141E80032002AF3D12023C5F8BB
:10BE40008830C5F88C30C5F89030D4E773B5044617
:10BE50000026C0F89060F7F715FF23681B681A07E3
:10BE6000054619D423681B685B070AD56FF07E432B
:10BE7000009300222B464FF480012046FFF782FFFB
:10BE8000B0B900202023C4F8883084F88400C4F8B6
:10BE90008C30E06620670CE06FF07E430093324602
:10BEA00003464FF400112046FFF76CFF0028D9D05D
:10BEB000032002B070BD10B5044650B3D0F88830EE
:10BEC0001BB980F88430F8F797F922682423C4F866
:10BED0008830136823F0010313602046FFF7F0FD5C
:10BEE000012816D0A36A13B12046FFF7F7FE236896
:10BEF0005A6822F490425A609A6822F02A029A60A4
:10BF00001A6842F0010220461A60BDE81040FFF7AF
:10BF10009DBF012010BD000030B581658168A0F88B
:10BF20005C200023B1F5805FA0F85E20436735D127
:10BF30000369002B40F2FF1318BFFF23A0F8603005
:10BF40000023C0F890302223C0F88C30016801F142
:10BF5000080353E8003F43F00103083141E800348F
:10BF60000368002CF2D1456E84680169B5F1005F69
:10BF700032D1B0F8685095422ED8B4F5805F244A8B
:10BF800003D1244C002908BF22464267B1B153E8CF
:10BF9000002F42F4807243E80021F7E729B90369D2
:10BFA000002B14BF7F23FF23C8E7B1F1805FC5D109
:10BFB0000369002B14BF3F237F23BFE703F108026F
:10BFC00052E8002F42F0805203F1080040E80021BF
:10BFD0000029F3D1002030BDB4F5805F0E4A03D1B3
:10BFE0000E4C002908BF2246426741B153E8002F9A
:10BFF00042F4907243E800210029F7D1EAE753E8C0
:10C00000002F42F0200243E800210029F7D1E1E7A8
:10C0100075B700081DB90008E5B50008B1B60008FD
:10C02000D0F88C30202B30B415D1B9B1B2B1002387
:10C030000468C3660A4B9C420AD063681B0207D59A
:10C0400054E8003F43F0806344E80035002DF7D109
:10C0500030BCFFF761BF022030BC70470120FBE716
:10C0600000800040436E30B52BB90123A0F86A3040
:10C07000A0F8683030BD0368094D9A689968094C8A
:10C08000490FC2F342626B5C615CDB00B3FBF1F30E
:10C09000A0F86A30AB5CA25CDB00B3FBF2F3E7E72D
:10C0A000D8710308D07103087047704770471FB5F7
:10C0B00004AB03E9060090F88430012B04463AD023
:10C0C000012380F884302423C0F8883003681A687C
:10C0D00022F001021A609A6822F440120A439A6020
:10C0E00071B95A68BDF80C009DF80E1022F01002CC
:10C0F00002435A605A6822F07F4242EA01625A6063
:10C100001A6842F001021A60F7F7BCFD6FF07E4238
:10C11000034600924FF4800100222046FFF732FED2
:10C1200038B92023C4F88830002384F8843004B060
:10C1300010BD0320F8E70220F9E790F88430012BC6
:10C140000FD0012380F88430016851E8002F42F0BD
:10C15000020241E80023002BF6D180F88430184613
:10C1600070470220704710B590F88430012B0446C8
:10C1700017D02423C0F8883003681A68196821F0A2
:10C180000101196042F000524FF0005141661A60FF
:10C19000FFF768FF2023C0F88830002084F884006F
:10C1A00010BD0220FCE770B590F88430012B0446E6
:10C1B00017D005682423C0F888302E682B6823F038
:10C1C00001032B60AB6823F060431943A960FFF7BC
:10C1D00049FF20232E60C0F88830002084F88400B6
:10C1E00070BD0220FCE770B590F88430012B044646
:10C1F00017D005682423C0F888302E682B6823F0F8
:10C2000001032B60AB6823F060631943A960FFF75B
:10C2100029FF20232E60C0F88830002084F8840095
:10C2200070BD0220FCE7000038B5084D052455F824
:10C23000043B2BB9013C14F0FF04F8D1204638BD73
:10C24000DB6898470028F5D0F9E700BF081D0020FB
:10C25000034BD870034B1B681B6C03B11847704726
:10C26000F01C0020EC1C0020034B1874034B1B68CF
:10C270005B6C03B118477047F01C0020EC1C0020D9
:10C28000F0B5314D314B95F90420314E91B00C464B
:10C29000012795F905108DF8047002288DF8092002
:10C2A0008DF80A1010D18DF80800D8711C7202F0B8
:10C2B00063FD337803B114B101A803F0C1F9254B34
:10C2C000059A1A6011B0F0BD59714FF480711A715E
:10C2D000D9801C7233788DF8087053BB1F2306A8D1
:10C2E0008DF81C208DF8183002F024FF20238DF8E3
:10C2F000183006A82B798DF81C3002F01BFF222382
:10C300008DF8183006A86B798DF81C3002F012FFFA
:10C3100021238DF8183006A86B798DF81C3002F0B7
:10C3200009FF29238DF8183006A80B4B079302F05C
:10C3300001FF02F021FD012306A88DF818308DF8C9
:10C340001C3002F0F7FEB4E7F01C0020E0030020F0
:10C35000CC1B0020C01C0020000400017FB5092375
:10C3600001A88DF8043003F06BF90038044B059AEE
:10C370001A6018BF0120404207B05DF804FB00BFFF
:10C38000C01C002070B504460B46144962784A7000
:10C390000020A2780A7208701A884A729A788A7203
:10C3A000DB780B746368CB600D4B1B68DA6A2AB1CB
:10C3B000237803F0FB030A2B00D09047094E002599
:10C3C00056F8043B1BB15B6A0BB120469847013518
:10C3D000EBB2052B6DB2F3D170BD00BFB0030020EE
:10C3E000EC1C0020081D002070B5044611480123F4
:10C3F000037063784370A3788372E368C360E37863
:10C40000037623694376237943720B4B1B689B6A3F
:10C4100003B19847094E002556F8043B1BB19B69B0
:10C420000BB1204698470135EBB2052B6DB2F3D125
:10C4300070BD00BFC4030020EC1C0020081D0020BC
:10C44000014B1868704700BFC01C002000B58BB0BE
:10C45000012368468DF8003002F046FD38B99DF89A
:10C460000400003818BF01200BB05DF804FB002069
:10C47000FAE7000008B501F037FE40B9FFF7E6FF24
:10C48000012806D0054B197AD879FFF7F9FE01206B
:10C4900008BDBDE80840FFF7C7BE00BFE0030020AD
:10C4A0002DE9F04186B005460E46174601F01CFE08
:10C4B000002873D101F030FE044640B9FFF7C6FFF3
:10C4C00001280AD03D4B197AD879FFF7D9FE6FF0D1
:10C4D0000204204606B0BDE8F081DFF8E48088F869
:10C4E0000860003E18BF01268DF80460354E68785C
:10C4F00033798DF81230694602F094FC00283FD061
:10C500008DF804400394ADF810406FF0060495E8F0
:10C5100003002D4B83E80300337988F80A3039464D
:10C5200001A803F091F9294B059A1A6011283FD808
:10C5300001A353F820F000BFA3C500089DC5000863
:10C54000B1C50008B1C50008B1C50008B1C50008F3
:10C55000B1C50008CFC40008B1C50008B1C50008C6
:10C56000B1C5000897C50008B1C50008B1C50008ED
:10C570009DC500089DC500089DC50008B7C50008F9
:10C580002B788DF808306B78ADF810306B6803931A
:10C590004FF0FF34BBE76FF005049AE76FF001043A
:10C5A00097E70B4B00221A70E31D18BF144690E763
:10C5B0004FF0FF348DE76FF004048AE7E0030020BA
:10C5C000C4030020F01C0020D4030020C01C002065
:10C5D000BF1C002037B501F0A9FD134D052455F807
:10C5E000043B4BB11A693AB19B682BB1984718B11B
:10C5F00055F8043C1B699847013C14F0FF04EED148
:10C60000FFF712FE68B9094D2B7853B1084BADF80E
:10C610000040D978019422466846FFF741FF00B9EF
:10C620002C7003B030BD00BF081D0020BF1C0020CF
:10C63000F01C002030B58BB0044601F055FD0546D6
:10C64000002835D1FFF702FF012834D168468DF864
:10C65000005002F049FC40BB9DF80430A34204D0D6
:10C66000012C22D0022C12D014B100200BB030BD0E
:10C67000002BFAD068468DF8044002F05BFDA0B9AB
:10C680000E4B1B681B6B002BEFD09847EDE763B98F
:10C6900068468DF8044002F04DFD30B9074B1B6829
:10C6A0001B6B002BE1D02046EFE74FF0FF30DDE7BA
:10C6B0006FF00100DAE76FF00200D7E7EC1C002012
:10C6C00010B504468AB018B94FF0FF300AB010BD5B
:10C6D000002368468DF8003002F006FC0028F3D1F4
:10C6E0009DF804302370F1E77FB500220B46204906
:10C6F0008DF8072001220A7042784A700446002A09
:10C7000033D102790A721A884A729A788A72DB786F
:10C710000B740369CB60C378164D8DF80830037B2A
:10C720008DF80930836803932B68DB6A0BB102A88C
:10C7300098472B689B6B13B1227E02B198470E4E2F
:10C74000052556F8043B1BB1DB690BB12046984721
:10C75000013D15F0FF05F4D10DF10700FFF7B0FF23
:10C76000637913B1054B01221A7004B070BD00BF8C
:10C77000B0030020EC1C0020081D0020BF1C00207E
:10C7800010B504468AB018B94FF0FF300AB010BD9A
:10C79000202368468DF8003002F0A6FB0028F3D174
:10C7A000024A9DF9043023701371EFE7F01C00205A
:10C7B00000B58BB02323019068468DF8003002F05D
:10C7C000B9FC003818BF012040420BB05DF804FBF3
:10C7D00070B5654C01468EB01822204606F08CF8E4
:10C7E000624B00221A70FAF745FE23784068012256
:10C7F00002FA03F1014004D15D4B084608F068F8E5
:10C80000FEE75C495C481A4602F0F8F818B14FF0B0
:10C81000FF300EB070BD272304A88DF8103002F051
:10C8200089FC564E564D002870D1012333702B6879
:10C83000DB690BB100209847272304A88DF810303E
:10C8400002F052FB059B93F84820227093F81821C0
:10C8500093F81A316270A370464BD3E9020105F0D8
:10C860003BFF05460028D2D1464E062304A88DF88A
:10C87000103002F039FB059B736104A802F05AFCEA
:10C88000022304A88DF81030059602F02DFB08361F
:10C89000032304A88DF81030059602F025FB0F261F
:10C8A00005F0E0FF012304A88DF814308DF8106026
:10C8B00002F040FC10230DEB03008DF810308DF8D2
:10C8C000145002F037FC04238DF8103004A8A3782C
:10C8D0008DF8143002F02EFC3A238DF8103004A8A5
:10C8E0006369059302F026FC02A920788DF80860A0
:10C8F00004F09CF8003818BF0120E0711420FFF705
:10C9000057FFE07903F062F9284682E728238DF883
:10C9100010302B681B6943B104A802F0E5FA2B68BC
:10C9200005981B6940F2C4519847272304A88DF845
:10C93000103002F0FFFB50B9012304A88DF810302D
:10C9400002F0D2FA9DF81430002B7FF46EAF3378EA
:10C95000002B7FF46CAF052204A88DF810200593FE
:10C9600002F0E8FB78E700BFF01C0020BF1C0020AD
:10C97000E0710308C41C0020DC1C0020CC1B00203C
:10C98000EC1C00202C1D002037B500230D46019320
:10C990000446D0B900F0A8FB0190019BD3B10F4A27
:10C9A00042F824300E4A9A620E4A1268916B19635B
:10C9B000916C596392690C49D9625A6128465B6847
:10C9C0000A49F2229847002006E001A900F092FBF4
:10C9D0000028E2D04FF0FF3003B030BD081D00202A
:10C9E00081C20008EC1C00205DC30008CD1B0020A4
:10C9F000194B07B51860194B194A1A60194A5A6041
:10CA0000194A9A60194ADA60194B02681A6042683A
:10CA10005A6082689A60C268DA60164A1A6182694E
:10CA20005A61154BC26B5A60144A019119609A60A1
:10CA30001946134ADA600020FFF7A6FF48B901A89B
:10CA400000F056FB003818BF0120404203B05DF8EB
:10CA500004FB4FF0FF30F9E7EC1C0020DC1C002049
:10CA6000E9C30008E9C60008FDCA000885C300083C
:10CA7000C41C0020DD0901081C1D002051C2000853
:10CA800069C2000849B118B1012804D000207047DC
:10CA9000034B0B60FAE7034BFBE74FF0FF307047A7
:10CAA000000400010100010208B503F0ABF8002802
:10CAB00014BF6FF00100002008BD08B502F084F932
:10CAC000002814BF6FF00100002008BD10B5044617
:10CAD0008AB018B94FF0FF300AB010BD2123684664
:10CAE0008DF8003002F000FA0028F3D1024A9DF9D7
:10CAF000043023705371EFE7F01C00202DE9F04162
:10CB00002F4D304F00232B7043786B703B689B6A2E
:10CB10008AB004460BB128469847DFF8AC8000265F
:10CB200058F8043B1BB11B6A0BB1204698470136ED
:10CB3000F3B2052B76B2F3D12378052B2FD00B2B34
:10CB400035D0012B25D1214C062368468DF80030C5
:10CB500002F0CAF90199E07905F004FE10B91C4B06
:10CB6000019A5A611B48FFF70BFE1B48FFF7AEFF07
:10CB70006B788BB9A371194B5878FFF75BFD3B6855
:10CB80005B6A0BB1114898476B7813B9E07905F0EF
:10CB90007BFE0AB0BDE8F081FF23A371EFE7104BE5
:10CBA00001225A74227A9A74627ADA74F1E763780D
:10CBB000002BEED00AB0BDE8F041FFF7CFBB00BFBD
:10CBC000C4030020EC1C0020081D0020E00300200E
:10CBD0002C1D0020E4030020E5030020F01C0020B1
:10CBE000B003002030B58BB0FFF767FF0446F0B903
:10CBF00003F0FCFE831C1DD0F8B9134D2B685B6954
:10CC0000DBB1272368468DF8003002F06DF92B6800
:10CC100001985B694FF4B961984703F0F9FE78B960
:10CC20002CB9094B1B68DB690BB1012098472046E2
:10CC30000BB030BD6FF00704EFE74FF0FF34ECE7C7
:10CC40004FF0FF34F3E700BFEC1C0020014B1878D5
:10CC5000704700BF601D0020014B5878704700BF2F
:10CC6000601D002070470000044B9A7A0AB101222F
:10CC70005A70034B5B6903B118477047601D002071
:10CC8000EC03002073B5224C6378002B33D008F0FE
:10CC900007F966680546FFF7D3FB0644AE4214D297
:10CCA000A37A93B1E0228DF800208DF80130217A2B
:10CCB000E368019301226846FFF7F2FB08B10730F1
:10CCC00010D100236370A372656094F83430EBB127
:10CCD000002384F834300F4B5B6BBBB102B0BDE86E
:10CCE0007040184740F2DC510B4808F0A5F90A489B
:10CCF00008F068F9E8E794F83520002AE5D094F8C0
:10CD0000360084F83530FFF795FCDEE702B070BDE1
:10CD1000601D0020EC030020441D002037B5104D9D
:10CD2000104CC8B1C1B16272012300222860E160D9
:10CD300023700D480D4B00924FF0FF3108F096F82C
:10CD400000250B4825822022294605F0E9FD657063
:10CD5000A574A58603B030BD00232B602370EFE7D8
:10CD60005C1D0020601D0020441D002069CC0008CF
:10CD7000741D00202DE9F0478E4C23788CB0002BD9
:10CD800056D0C2780AB9837B13B1238A0133238238
:10CD9000437B002B4CD0E02A4AD10023A372876842
:10CDA00097F80080B8F1220F27D8B8F1220F30D8B9
:10CDB000DFE818F04100FB0052005A0061006E00ED
:10CDC00075008E009D00B400C7002F002F002F00BB
:10CDD0002F002F002F002F002F002F002F002F00DB
:10CDE0002F002F002F002F002F002F002F002F00CB
:10CDF0002F002F00C900D000D400B8F17E0F00F042
:10CE0000CC80B8F17F0F00F0DF80B8F17D0F00F02B
:10CE1000AB80A57A002D00F05B81674C637A3BB94B
:10CE20004FF47A71204608F007F9204608F0CAF856
:10CE30000CB0BDE8F087E36801220021A2721970EE
:10CE4000A37AE1689818A0720620C854A37AE16812
:10CE50009818A072CA54DCE7584B9B6A002BD8D0B4
:10CE6000012102209847D4E77B7884F836300123EB
:10CE700084F83530CDE704238DF804307B78003B0F
:10CE800018BF012301A88DF8083002F053F9C0E75C
:10CE90007878003818BF012002F098FEB9E7484EB4
:10CEA0000FCE01AD0FC50FCE0FC596E8070085E880
:10CEB00007007B780A2BACD8424A12685268002AD5
:10CEC000A7D00CA901EB830353F82C0C9047A0E7E3
:10CED0007878431E012B9CD83A4B01381B6818BF49
:10CEE000012020729B68002B93D0984791E7E2685D
:10CEF00001230821A3721170627A057BA17AAA42EC
:10CF000028BF2A46934284D285685A1CEB5CE568A8
:10CF100001334E1CA6726B54D3B2EDE7E3680122D5
:10CF2000A27209221A70A37AE268218A581CA072A0
:10CF3000D154A27A238AE1681B0A501CA0728B5438
:10CF400067E7238265E705238DF8043001A802F026
:10CF500077FB5EE7194BDB6A98475AE7194B7878FD
:10CF60001B686075DB68BEE7037B072B7FF451AF5E
:10CF700006238DF80430B7F80130ADF808307B791E
:10CF80003A791B0443EA0223FA7813436422534399
:10CF90000393BB798DF81030D8E73B2201A88DF8B8
:10CFA00004208DF8083002F0C5F8012384F83430ED
:10CFB0002FE700BF601D0020441D0020EC0300206F
:10CFC000841B03085C1D00202A2301A88DF804306F
:10CFD00001F08AFF94F80A90E6689DF808009DF831
:10CFE00009509DF80A709DF80BC09DF80D309DF812
:10CFF0000E209DF80F109DF80CE009F1010A84F84D
:10D000000AA006F80980354E94F80A903668D4F8DC
:10D010000C8009F1010A84F80AA096F803A008F828
:10D0200009A094F80A90D4F80C8009F1010A84F858
:10D030000AA096F802A008F809A094F80A90D4F87B
:10D040000C8009F1010A84F80AA096F801A008F8FA
:10D0500009A094F80A9009F1010A84F80AA096F848
:10D060000080E66806F8098094F80A80E66808F10E
:10D07000010984F80A9006F808C094F80AC0E66826
:10D080000CF1010884F80A8006F80C70A77AE668AB
:10D0900007F1010C84F80AC0F555A57AE6686F1C03
:10D0A000A7727055A07AE568461CA6722954A17A29
:10D0B000E0684D1CA5724254A27AE168501CA0722F
:10D0C0008B54A37AE268591CA17202F803E0A0E62F
:10D0D000034807F029FF6570AAE600BF5C1D002029
:10D0E000441D00207047000000487047EC030020FA
:10D0F000002070474FF0FF3070470000044B054A96
:10D1000093F81831022B18BF062382F89034704729
:10D1100004240020C8290020034BD3F8483313B15E
:10D120005B6903B118477047C8290020034A137888
:10D1300043F004031370FFF7EFBF00BFAC1D0020E6
:10D140001FB50A4B8DF8090093F87C208DF80A2052
:10D1500093F88C2093F848000D3202A98DF808202E
:10D1600003F064FCC0B205B05DF804FB04240020A9
:10D1700008B5074807F0D8FE064B93F81A2412B1F9
:10D18000012283F81924BDE80840FFF7C5BF00BF9E
:10D19000C82D0020C829002010B50C4CD4F840330D
:10D1A00043F08003C4F8403394F81A3413B10020DC
:10D1B000FFF7DEFF94F8913423F0120343F01203DB
:10D1C00084F89134BDE81040FFF798BFC8290020CB
:10D1D0002DE9F041DFF8AC8098F81831022B0646B3
:10D1E0000D4602D0284BDB6A984702F0A6FD0446A4
:10D1F00028B1022002F097FD002002F099FD98F876
:10D200001831012B17D102F09AFD074630B10020EA
:10D2100002F08AFD002002F08CFD3C4602F091FDF8
:10D2200048B1002002F081FD002002F083FDBDE83E
:10D23000F041FFF763BF002CF9D1144C94F890240F
:10D2400094F81A34BAB90BB184F84164304602F04C
:10D2500017FFD8F82C0007F02DFED4F8B43398420D
:10D26000E5D30B4807F060FE94F8913443F01003C7
:10D2700084F89134DBE70BB184F84154284602F07E
:10D28000FFFEF1E70424002058790308C829002094
:10D29000602D0020074A10B5137843F00203137085
:10D2A000FFF73AFFBDE81040034B012200210220A6
:10D2B00007F00EBBAC1D002029720308074A10B509
:10D2C000137843F008031370FFF726FFBDE8104002
:10D2D000034B01220021022007F0FABAAC1D002006
:10D2E000397203082DE9F0410F4616461D46804667
:10D2F00007F0D6FD0B4A0C4C1378278123F011035D
:10D3000043F01103C4E90008137066812573FFF729
:10D3100003FFBDE8F041054B01220021022007F088
:10D32000D7BA00BFAC1D0020981D00204972030829
:10D3300013B507F0B5FD0D4B6C461860204607F09D
:10D3400003FD94E803000A4A0A4B83E803001378BC
:10D3500043F020031370FFF7DFFE074B012200218B
:10D36000022002B0BDE8104007F0B2BAA81D0020AC
:10D37000AC1D0020002D0020567203082DE9F0415D
:10D3800092B0064602F0D9FC002840F05881AD4D1D
:10D3900095F81831012B09D02B6BAB4C93B194F855
:10D3A0000431BBB1042B6FD0032003E002F0C7FCB3
:10D3B00018B10F2012B0BDE8F08102F0C2FC0028C5
:10D3C000EAD0F6E7B5F82031D4F81C24013B5343EA
:10D3D0002B63E4E79D4803F060FA002840F01281D7
:10D3E00094F80C3123802B6B0C930DF1180895F8F1
:10D3F00039308DF83830404695F81C318DF83A3088
:10D4000007F0C8FCD5F82831009302AF98E8060071
:10D41000D5F82431384607F054FC97E803000FABE9
:10D4200083E80300EB6A0D9300238DF844302388D2
:10D43000ADF8463095F8303101228DF839201BB90E
:10D440008DF844208DF83930814B0093814B95F84D
:10D450004800A3F179020CA903F05DFBC0B10B28D1
:10D46000A8D1D4F8941499B1002EA3D0D4F84033A5
:10D47000794843F02003C4F8403307F0DDFD7648D7
:10D4800007F0A0FD002095E7704803F03AFAA4E702
:10D4900095F8487095F9693095F9392095F87D101F
:10D4A0006E4E384603F044FB009641B2EB6C95F8A3
:10D4B00050203846183603F0DFFA0096EB6C95F8EA
:10D4C000502095F9701095F8480003F0D5FAD4F87B
:10D4D000C413AB6DD4F8DC230B44C4F8B033EB6D4C
:10D4E0001344C4F8B43394F80431042B07D02B6EE2
:10D4F0000B44C4F8B0336B6E1344C4F8B433002348
:10D50000089395F83031002B40D100238DF813306B
:10D5100095F839308DF8213095F838308DF8223073
:10D52000D5F880300993D5F884300A932388ADF874
:10D530002C3095F8303194F81B648DF82E3095F826
:10D540004800474B8DF820600DF1130208A903F045
:10D55000A7FA012384F8413495F8393084F842342D
:10D560009DF8133084F84334D4F81C34C4F8506464
:10D57000C4F84834C4F8583402F0E5FBC8B1D4F814
:10D580001C0402F0F2FBA0B1102013E708A802F07F
:10D59000A7FC60B995F9390094F837629DF82070BE
:10D5A000FFF7CEFD3E44B042AFD2082002E7132081
:10D5B00000E795F81831012B01D102F0D8FB02F0F9
:10D5C000C5FB0023059394F8043195F9395094F87C
:10D5D0001B649BB1042B7FF4E7AE05A802F0B4FEF8
:10D5E00058BB94F8183413B1059B013B0593174BB6
:10D5F00005983246E9B202F00DFF02E0134802F04E
:10D60000DDFE08B11120D5E6D4F8403394F80C11B2
:10D61000218043F00203C4F8403394F818341148D1
:10D620000133DBB284F8183484F845340E4B0025FE
:10D630009B6AC4F89854984724E71220BAE60E2053
:10D64000B8E600BF04240020C8290020D02A00200A
:10D65000342400205C2E0020302D0020802D00205E
:10D66000E42D0020CA2900205879030873B5134D12
:10D67000134E0096EB6C95F8502095F9781095F8BC
:10D68000480003F0F9F995F83031337595F8480002
:10D6900040F2012306F13C023146738203F0F8F9AF
:10D6A00050B196F83C3086F88230064B00205B6B18
:10D6B0009847F37C86F8A83002B070BD042400209F
:10D6C000B02D002058790308F8B5324C94F8183181
:10D6D000012B05460ED0022B4ED0002B57D138B966
:10D6E000D4E91B0104F1740383E803000020F8BDB2
:10D6F000012806D102F02CFB0028F8D184F818513B
:10D70000F5E7022843D1244E84F8180106F5747C0D
:10D71000BCE80F0006F57A770FC79CE8030094F881
:10D72000E92094F8003187E8030086F8FB53D2B172
:10D73000022B18D1D4F804316367C6F8EC3394F89F
:10D740007D3094F8082186F8F83394F88C3084F80A
:10D75000782086F8F93396F81B2486F8E82340F2FF
:10D760000133A6F8FA33002386F81A340B4BDB6A30
:10D770009847FFF77BFFB9E748B9074B84F81801D2
:10D78000062283F89024054BDB6A9847AEE7032016
:10D79000ADE700BF04240020C82900205879030801
:10D7A000F0B5504C504EB4F8DC202287D4E92D015E
:10D7B00094F8B12084F8692004F16C0282E8030037
:10D7C000D4E92F0104F1740282E80300B4F8C42004
:10D7D000A4F87C2091B0D4F8CC20D4F8C810C4F8B8
:10D7E00084200025D4F8D020C4F888200123A4F890
:10D7F0002031C4F8801084F83051A56284F81B51A0
:10D8000084F83A5084F81D5184F81E51C4F83451FC
:10D81000C6F89854A6F8185486F81A54A4F8385143
:10D820008DF8183004F50973039304F50A7394F81E
:10D830004800049303A92D4B84F84551C4E94F5582
:10D84000A4F84651059303F0FFF8E36EC6F8D4330D
:10D8500094F87D3086F8E03394F88C3086F8E13324
:10D860004FF48073A6F8E23386F8D05394F8303141
:10D8700086F8E43306F574770FCF06F57A740FC493
:10D8800097E8030040F2012384E80300A6F8FA3386
:10D89000D6F8483386F81B54CDE901551BB15A68B8
:10D8A0005B6901920293124B0793A3F1480208921D
:10D8B000A3F1140209920F4A0B9229330A93A2F1A1
:10D8C0009C030C93A2F198030D93131D0E9301A9D1
:10D8D00002F14C0307A802F599620F9302F022FAB5
:10D8E00011B0F0BD04240020C8290020B01D002084
:10D8F000302E0020E8240020F8B50D4F0D4E0C46C8
:10D9000007F012FB3B6B98470B4A96F848002146FC
:10D9100003F0BEF850B1094D706D95F8243485F8C8
:10D920006A347B6B9847E37C85F89034F8BD00BF80
:10D930005879030804240020EC2D0020C829002079
:10D940000F4890F81B3480F8B8330E4B93F86920D9
:10D9500080F8BB2393F87D2080F8C82393F88C20AF
:10D9600080F8C92393F8303180F8CC330022A0F836
:10D97000CA2300F56E7100F56070FFF7BDBF00BFF0
:10D98000C829002004240020114890F89034EBB1FD
:10D9900090F81B3480F8D0330E4BDA6EC0F8D423E5
:10D9A00093F87D2080F8E02393F88C2080F8E12321
:10D9B00093F8303180F8E4334FF48072A0F8E2231A
:10D9C00000F5747100F56670FFF796BF704700BFF1
:10D9D000C82900200424002070B5344C242120469E
:10D9E00004F0A0FF636A984218BF60624FF01C0108
:10D9F0002F4814BF0125002504F094FF636C984262
:10DA000018BF60644FF480712A4818BF45F00205C2
:10DA100004F088FFD4F84831984218BFC4F8480190
:10DA20004FF0D401244818BF45F0040504F07AFFF4
:10DA3000D4F82032984218BFC4F820024FF00001F9
:10DA40001E4818BF45F0080504F06CFFD4F82432D6
:10DA5000984218BFC4F824024FF46071184818BFE8
:10DA600045F0100504F05EFFD4F8A835984218BFC1
:10DA7000C4F8A8054FF01401124818BF45F020055E
:10DA800004F050FFD4F8C03598420F4B18BFC4F8CB
:10DA9000C005D3F8483318BF45F040052BB11B69CA
:10DAA0001BB12846BDE87040184770BD0424002013
:10DAB0002C2400204C240020502500202826002063
:10DAC0002C260020B0290020C82900202DE9F04F85
:10DAD0008FB04FF00009012B06460F4690468DF897
:10DAE0000D90ADF8109002D84C46BC4202D30FB056
:10DAF000BDE8F08F305D02F033FA2044B842F6DC26
:10DB0000335D651C023BEDB2112BF0D801A252F837
:10DB100023F000BF5DDB000887DB000885DC000820
:10DB2000ADDC00082BDD000851DD0008B7DD000882
:10DB3000DFDD000865DE0008EFDA0008EFDA000834
:10DB4000B9DE0008EFDA0008EFDA000861DF00084C
:10DB500089DF0008C1DF0008F5DF0008052002F0BA
:10DB6000A7FA70B10521002002F068FA725DBA4B85
:10DB7000E51C0234E4B283F85C24325D83F85D2452
:10DB8000EDB22C46B1E700238DF80E308DF80F3042
:10DB90008DF814308DF81830B9F1000F6DD1AF4CFD
:10DBA0004FF0050994F87C208DF831206B1E94F815
:10DBB00039208DF83320334494F838200B938DF8B6
:10DBC000342094F81A3194F868208DF83520D4F870
:10DBD0002C218DF832300A9273B37B1C5B1BDBB2B5
:10DBE0008DF8303006AB019305AB009394F84800F4
:10DBF0000DF10F030DF10E020AA902F05DFF8DF881
:10DC00000D0000F00700072813D194F939209DF981
:10DC10000E3084F839309A429DF80F3084F838304D
:10DC2000B8BF01229DF81430B8BF84F81D2184F8D4
:10DC300068304FF0000A09E00523D1E701220DF119
:10DC40000D01032002F0A4F80AF1010A5FFA8AF23A
:10DC50009DF81830B3FBF9F19142EFD82B44DDB2B7
:10DC60006B1EDBB29F420BD9F25C032A9AD0AF4203
:10DC700088BF1D464FF0010983E70534E5B2F9E797
:10DC80001D46F7E7735D754903F00F03012281F824
:10DC90001B31023402FA03F3A1F82031E4B200226E
:10DCA00004A9042002F074F825466AE707238DF8DA
:10DCB0000D30735DC3F3021203F00F038DF82830AB
:10DCC000E31CDBB28DF82920F25C231DDBB2651D5D
:10DCD000F35C0234E4B21B0443EA0223325D5F4C7E
:10DCE00013436422534394F848000B930AA902F0AB
:10DCF000F2FE00F00703072BEDB28DF80D000CD1FA
:10DD00009DF8283084F8703084F878300B9BE366F7
:10DD100063679DF8293084F869308DF8100001227E
:10DD200004A9052002F034F82BE74B4BD3F8483315
:10DD300063B11B6853B1984708F03F038DF810009A
:10DD40008DF81130022204A90620EBE7FF20F3E74B
:10DD500003238DF80D30735D8DF81C300AAB0693EC
:10DD6000E31CDBB2A51DF25C231DDBB206A9F35C4C
:10DD70001B0443EA0223A21CD2B20534B25C134353
:10DD800064225343E4B20A9300230B93335D8DF86E
:10DD90003030324B93F8480002F0A3FEC3B20028A3
:10DDA000EDB28DF80D30FFF6ECAE8DF8103001229B
:10DDB00004A90720B6E7735D03F00F03012B4FF4AE
:10DDC0007A7238BF01235343244A0234936503F522
:10DDD0007A73D365E4B2002204A9082062E7735D78
:10DDE0001E4DC3F340128DF8152095F84800C3F37B
:10DDF000001205A903F00F038DF814208DF81630DA
:10DE000002F075FE02340130E4B23FF44DAFBDF8CC
:10DE10001430134AA5F87C309DF816309DF814A0F4
:10DE2000D05CF4F7C7F80223C5F880000AA995F87A
:10DE300048008DF828308DF82AA002F0F7FD95F9FA
:10DE40003930069040B29842B8BF184685F839007C
:10DE5000002204A9092025E7C82900200424002065
:10DE60006372030803238DF80D30735D8DF828303D
:10DE7000E31CDBB2651DF25C231DDBB20234F35CF4
:10DE8000E4B21B0443EA0223325D1343642253438A
:10DE90000B93644B0AA993F8480002F02EFEC3B21C
:10DEA0000028EDB28DF80D30FFF66BAE8DF8103016
:10DEB000012204A90A2035E7092002F0F9F8DFF869
:10DEC00068B1002849D00921002002F0B7F80023EA
:10DED000ADF81E30A31CDBB2F25CE31CDBB216F81B
:10DEE00003A0735D4FEA0A4A4AEA022A4AEA030A91
:10DEF000231DDBB2A51D0534F35CE4B24AEA036AD4
:10DF0000335D4FF47A7253430AAC1B122046ADF8CE
:10DF10001C3006F019FF454B53440693DBF83C33A5
:10DF200000930DF1180A9AE80600DBF8383308A8C8
:10DF300006F0C7FE099B009394E80600089B504634
:10DF400006F0A4FE9AE8030006F0D6FE01F00AFFF0
:10DF50000123EDB28BF8383413E68BF8380410E661
:10DF60000C2002F0A5F800283FF40BAE0C21002095
:10DF700002F064F82C4B93F89034043B012B7FF6AD
:10DF800000AE01F0EBFEFCE5A31CDBB2725DF15CC0
:10DF9000E31CDBB2651DF35C0434E4B21B04305DAA
:10DFA00043EA012313436421594300F00F0001F0B9
:10DFB000D6FEEDB28DF81000012204A91120B1E6C1
:10DFC0000D2002F075F800283FF4DBAD0D21002094
:10DFD00002F034F8A31CDBB2154AF05C735D1268E2
:10DFE000251D0334E4B243EA0020315DEDB201F0B7
:10DFF000B8FEC6E5725DA31C251D0334DBB2E4B296
:10E00000F15C335D1B0443EA01231343642058434E
:10E0100001F0A9FEEDB28DF81000012204A9132031
:10E0200080E600BF04240020C8290020803DD512CE
:10E03000981D00200E4B93F89124920703D593F876
:10E040008F24012A08D90B4991F81A2122B18A6A32
:10E05000501C18BF01328A620022A3F8182483F8EA
:10E060001A24D3F8402322F00202C3F84023704759
:10E07000C82900200424002070B5184C1848194DF8
:10E0800006F052FFD4F84033D4F89804D5F89060E5
:10E0900023F02003C4F8403338B106F00BFF86426A
:10E0A00003D2002385F83A3070BD0120FFF766F9EE
:10E0B0000028F9D00B28F7D095F8393084F842348D
:10E0C000092094F8183484F8453484F8410401F0A8
:10E0D000D7FFBDE87040FFF7ADBF00BFC8290020E3
:10E0E000302D002004240020094BD3F84023012ABE
:10E0F0000AD008490978C90708D43AB993F89204B4
:10E10000013818BF01207047002070470120704778
:10E11000C8290020AC1D0020034BD3F84003431E48
:10E1200058425841704700BFC82900202DE9F04FE0
:10E13000A9B0EFF3108272B6DFF8F0B20021DBF87D
:10E140000030CBF8001082F31088B94C002B00F09F
:10E15000E180DAB29B06039264D5B64D95F818318A
:10E16000022B02D0B44BDB6A9847EFF3108872B6EB
:10E17000B24F06F095FE3E68D4F8B013361A31441B
:10E18000AF4806F059FFAE4806F01CFFD4F8B413B0
:10E19000AC48314406F050FFAA4806F013FF88F35C
:10E1A000108894F81A34002B00F06B81152312A903
:10E1B00095F848008DF8483002F038FCD4F8B413D4
:10E1C0000F900144A04806F037FF9F4806F0FAFE82
:10E1D0003B6894F81B24EB620DAF38468DF8702035
:10E1E0001D9306F0D7FDD5F82831009306AE97E8C9
:10E1F0000600D5F82431304606F063FD96E80300AA
:10E200001FAB83E80300D4F81C341E9395F830311B
:10E2100095F84800003B18BF01231CA98DF8713008
:10E2200002F00DFC039BDF0648D5824DDFF81CA2EF
:10E23000D5F8E42004929BF80020BAF90A809AF9F4
:10E240000C90A4F88C84002363F300020A9384F8F2
:10E250004434A4F8223484F82534C4F82834A4F8CB
:10E260002C3484F82E34C4F8303484F82034C4F8C4
:10E27000343484F83834C4F83C346F4B8BF80020C5
:10E2800094F89024DB6A84F88E9484F88F24DAF86A
:10E290000470BAF80860984794F88F3413B9694845
:10E2A00006F042FE3146384601F045FD834600281F
:10E2B00000F0EA80A4F87E8484F88094039B190718
:10E2C0001AD55C4B93F81831022B02D05A4BDB6AFB
:10E2D00098470220FEF712FF84F8410401F0D0FEB7
:10E2E00094F81A3413B1012384F8193494F8913452
:10E2F00043F0100384F89134039B5A0703D5062199
:10E300000520FEF765FF039B9B0703D5042103202F
:10E31000FEF75EFF01F02DFD94F89124D7065FD53E
:10E32000002384F89234D4F840331E0644BF23F00F
:10E330008203C4F8403312F0050F00F0FB820B207B
:10E3400001F0B6FE002800F0F58294F89134DD0764
:10E3500000F1F082580740F10783D4F8403323F0EE
:10E360000203C4F84033D4F8402382BB94F891549C
:10E3700015F001011EBF2B4662F3000384F89134AF
:10E3800094F891345E0744BF6FF3820384F89134AC
:10E39000012384F8923421B1D4F844332C481B680B
:10E3A00098476D070BD52B4801F08EFE01F0BCFE9F
:10E3B00028B194F8913443F0040384F8913401F0C7
:10E3C000C6FC94F891346FF3041384F8913401235C
:10E3D00084F8923494F8913443F0200384F8913413
:10E3E00094F8913418070AD56FF3C3031A4984F8D7
:10E3F0009134D4F84433A1F12400DB68984794F8B1
:10E40000913499070AD56FF34103134984F8913485
:10E41000D4F84433A1F16C005B68984794F89034C9
:10E42000022B1BD1FFF722F918E000BFAC1D002022
:10E43000C82900200424002058790308A81D0020C2
:10E44000482D0020602D0020C82D0020981D0020A0
:10E45000082E00201C2E0020542E002094F8913409
:10E460009A0640F1C4826FF3451384F89134D4F8CE
:10E470004033002B40F0BB8229B0BDE8F04FFFF7DE
:10E48000ABBA84F84134A3E695F81831012B0CD1CE
:10E4900001F055FC804668B1584601F045FC5846ED
:10E4A00001F047FC042384F88F347EB9012384F8FB
:10E4B00021344FE101F045FC0028F6D0404601F040
:10E4C00034FC404601F036FC0523ECE73B7805932D
:10E4D0005B09013B062B00F21782DFE813F007000F
:10E4E000150295001502920015020602102EDDD9C4
:10E4F00095F830311297F6B28DF84C60002BD5D1DB
:10E500001CA804F021F912AA1CA9FF2002F09EF811
:10E510009DF85830C3F3030307468DF82C3095F867
:10E52000480095F87D308DF82D3007220BA902F0B8
:10E5300090FA002F5DD100285BD09DF853309DF8F4
:10E5400052201599C5F8E4101B0443EA02239DF8F4
:10E55000512002201343C5F8E03004F003F99DF880
:10E56000583095F8480085F82E71C3F30212C3F3B2
:10E57000030385F8703085F878309DF8593085F8B8
:10E580006920012B38BF01234FF47A725343AB65E6
:10E590001344EB650DF15A034FF001081093113E3F
:10E5A00094F81B348DF83C300FA985F868808DF8FD
:10E5B000446002F056FA0223404685F8303101F0FB
:10E5C00077FD18B14146384601F038FD94F88F3494
:10E5D000012B00F2A78194F81A34002B40F09A81A5
:10E5E00094F8913443F0100384F89134FEF786FDDB
:10E5F00064E6012001F05CFD0028E7D0012107203E
:10E60000E2E7012384F8203495F87D308DF82E3030
:10E6100094F824348DF82D3095F88C3095F8480016
:10E620000D330BA98DF82C3002F000FAA6F10D0382
:10E630001BB2099023EAE37300B283423FF736AF7F
:10E640000B2E7FF633AFBA4B25931CA8FF231C97E4
:10E650008DF874608DF8983002F0C4F807460028F1
:10E660007FF424AF95F81831012B13D101F067FB2B
:10E67000002872D0384601F057FB384601F059FBAC
:10E6800004239DF87C101E9884F88F34C1F3001188
:10E6900001F06EFB9DF87C301E99C4F8341413F021
:10E6A0000F0203D09DF89000002862D19DF89800D9
:10E6B000002861D0002A7FF4F9AE9DF89020002A4E
:10E6C00014BF4FF003084FF0020800220A92D5F859
:10E6D000EC2095F8E900914251D100284FD0D5F8AF
:10E6E0000C1195F8EAB009680A9195F818110229F9
:10E6F00002D1032184F88F14B8F1030F7FF4D6AE52
:10E7000013F0600F7FF4D2AE0492012795F82E31FA
:10E71000BBF1000F36D0BBF1010F13D1012B33D168
:10E720006FF0090646FA08F606F00106C6F1020681
:10E73000F6B2BDF87E100AAA304601F011FE38B3D9
:10E74000072823D0012384F821340A9BC4F83034ED
:10E75000C4F86C34FEF720FDB0E501F0F2FA0028B1
:10E7600098D0384601F0E1FA384601F0E3FA052383
:10E7700087E74FF00008A8E74FF00108A5E74FF042
:10E78000010BC3E70426D4E70326D2E70823DAE720
:10E790001CAB009304990A9B3246584601F0A2FE36
:10E7A00020B1022814BF0B230A2380E60A9BC4F879
:10E7B0003034C4F86C349DF87C3084F82104C3F301
:10E7C000401384F82E3484F8443494F88F3484F859
:10E7D0002274012B9EBF0122A86285F81E21012F01
:10E7E000C4F8280484F82C0484F8410438D10222A7
:10E7F00084F8202495F83A20002A4AD19DF87C20FC
:10E80000D60646D4012B94F840149DF87C2005D8F8
:10E81000012901D1900601D501F04CFBB8F1020F9E
:10E8200094F88F3443D0B8F1030F0AD09DF87C10D0
:10E83000B8F1010F4A4601F00F0120A83BD0FFF7C5
:10E8400045F99DF8903084F82334259BC4F828348A
:10E850009DF8983084F82C34012384F82D3430E06E
:10E86000059A02F0E002A02A1BD195F82E11012290
:10E8700085F83A2009B927996963012B84F8202487
:10E8800007D9D5F89020C4F83C24DAF80020C4F861
:10E89000982495F81821002AB4D1012284F825245F
:10E8A000B0E7002285F83A2084F82024A6E79DF8F6
:10E8B000981025984A46FFF709F99DF8903084F89A
:10E8C00023349DF89020E02A08D195F81F312BB908
:10E8D00084F82324C4F82834A4F82C3494F8913410
:10E8E00043F0020384F8913470E6114D013EB2B258
:10E8F000791C284604F000F80323A4F82034C4F857
:10E90000285484F82C64E9E7012384F82134FEF7C5
:10E9100043FC5BE694F84434002B3FF461AE0020E6
:10E92000FEF726FC94F88F34022B3FF45FAE57E6D7
:10E93000002C002094F89134590715D5012001F0DE
:10E94000B7FB60B1012001F08BFB08B984F8180413
:10E95000D4F8403323F00203C4F8403304E0062027
:10E9600001F0A6FB0028F3D194F89134DA077FF583
:10E97000FAAC94F840240AB1032A18D11D4A94F83D
:10E98000181492F86820914205D29B0723D594F879
:10E990008F34012B1FD8184806F0C6FAD4F840333C
:10E9A00023F02003C4F84033FFF744FBDBE4012AE3
:10E9B00011D194F81924002A3FF4D5AC0D4A94F8EB
:10E9C000181492F868209142E5D29F0703D594F875
:10E9D0004434002BDFD194F8913400206FF30413FA
:10E9E00084F8913484F81904FFF746FBBBE429B09E
:10E9F000BDE8F08F04240020302D00202DE9F04FD9
:10EA000089468DB090460746002800F08F81002986
:10EA100000F08C810368002B00F088814368002B94
:10EA200000F084818368002B00F08081C368002B94
:10EA300000F07C81104601F0F5FF002800F078819D
:10EA4000BD4CBE4D384601F0AFFA40F2C452002131
:10EA5000204603F065FF40F21C520021284603F0D7
:10EA60005FFFB74BC4F82C3104F50973089304F524
:10EA70000A7300264046099308A9B24B84F84880DF
:10EA80000A9384F8186184F88C608DF82C6001F08A
:10EA9000DBFF0F2306A994F848008DF8183001F029
:10EAA000C5FF801B18BF01204FF00A0B84F81C0122
:10EAB00006A994F848008DF818B001F0B7FF4FF0A0
:10EAC000060A84F8DC0006A994F848008DF818A01E
:10EAD00001F0ACFF102384F8DD0006A994F848008B
:10EAE0008DF8183001F0A2FF1123C4F89C0006A98C
:10EAF00094F848008DF8183001F098FF1223C4F8FC
:10EB0000A00006A994F848008DF8183001F08EFF97
:10EB10001323C4F8A40006A994F848008DF818300F
:10EB200001F084FF1423C4F8A80006A994F8480053
:10EB30008DF8183001F07AFF1623C4F8AC0006A94E
:10EB400094F848008DF8183001F070FF172384F80E
:10EB5000B10006A994F848008DF8183001F066FF5E
:10EB600018230DEB0301C4F8B400C4F8BC0094F8FA
:10EB700048008DF8183001F059FFC0B21D2384F809
:10EB8000B80084F8C00006A994F848008DF8183041
:10EB900001F04CFF1E2384F8C40006A994F8480035
:10EBA0008DF8183001F042FF1F2384F8C50006A934
:10EBB00094F848008DF8183001F038FF2023C4F88D
:10EBC000C80006A994F848008DF8183001F02EFF0F
:10EBD0000B23C4F8CC0006A994F848008DF818302F
:10EBE00001F024FF0C2306A9A4F8D00094F84800F3
:10EBF0008DF8183001F01AFFD4F89C306365D4F812
:10EC0000A030A365D4F8A430E365D4F8A830236617
:10EC10004FF00108D4F8AC300590A4F8D200636638
:10EC200084F8B080C4F894B084F898A0C4F84CB0CC
:10EC300084F850A084F8688084F81F81C5F8489350
:10EC4000FEF7AEFDC5F84473C4E90B663E4B84F88D
:10EC5000198185F89164C5F8408332464FF0FF3141
:10EC6000009605F55A7006F001F9384B00963246C9
:10EC70004FF0FF3105F5607006F0F8F8344B009660
:10EC800032464FF0FF3105F5667006F0EFF802AF3F
:10EC9000304B009632464FF0FF3105F5806006F0AC
:10ECA000E5F8384606F076F897E8030004F5927325
:10ECB00083E80300284B294F1E60294BC5F84C33CD
:10ECC000284BC5F85433284BC5F85C33274BC5F89F
:10ECD0005033274BC5F8583305F553703B689847B8
:10ECE00004F5A67003F04CFB20B1112630460DB0A0
:10ECF000BDE8F08F204601F003FB0028F5D101F0BC
:10ED000039F8B8B91B4801F04DFB06460028ECD194
:10ED10007B69984703F0CEFDBB6D94F819019847C5
:10ED2000FB6A9847012385F89234DFE70326DDE785
:10ED30000926DBE71326D9E704240020C829002090
:10ED400000040001B01D002079E0000841D900084E
:10ED500089D9000871D10008AC1D0020587903083A
:10ED600031D30008E5D200082DD10008BDD200083B
:10ED700095D20008EC24002008B5034B0020C3F80E
:10ED80004003FEF7BBF908BDC829002010B5FFF706
:10ED9000ABF90A4C60B90A4B93F81831022B02D137
:10EDA000084BDB6A98470123C4F84033002010BDAC
:10EDB000D4F84003013818BF0120F8E7C829002023
:10EDC000042400205879030838B5124C204606F078
:10EDD000ABF804F1180006F0A7F804F1300006F0D3
:10EDE000A3F804F1980006F09FF800F0AFFF0A4B7B
:10EDF0000025DB6A984744F8285CFEF7EDFD0749DB
:10EE0000074840F2C45203F077FD012344F8283C40
:10EE1000284638BD302D00205879030804240020EE
:10EE2000401E002070B52E4B8AB0054693F8DD00D9
:10EE30008DF8090093F8DC008DF80A0029489A6AD9
:10EE400090F81804039200268DF80B0004960C46E7
:10EE5000002940D00692D3F8882007921A8F93F8A1
:10EE60001A118DF8151052BAADF8202093F87C20B5
:10EE700093F848308DF8243003AB8DF822008DF8DC
:10EE8000232000930DF10A020DF10B030DF109018E
:10EE900005A88DF8146000F0D7FE9DF90900FEF773
:10EEA0004FF9607004A801F01BF8B0B9049A0F2A5A
:10EEB0000DD863789A420AD81544AB42A3EB0201FD
:10EEC0002CBF002001202170C0000AB070BD0023BB
:10EED00023700820F9E70320F7E71320F5E700BFC8
:10EEE00004240020C82900201FB50446002800F093
:10EEF00010810378412B00F20781DFE813F0420014
:10EF000049004D005100550059005E000501050102
:10EF100005010501050105010501050165006900FF
:10EF20006D0078007F00820085008A0088008C00D8
:10EF300090009300960099009C009F00AE00B200E4
:10EF4000BA00B600BE00C100C500CE00CA00CC00A9
:10EF50000501D200050105010501050105010501B5
:10EF60000501050105010501050105010501050171
:10EF70000501DA00DE00E200E700EB00EF00F3003D
:10EF8000FC00664B93F818312371002004B010BDCB
:10EF9000624B93F83031F7E7406803F08FFBF4E7FA
:10EFA000406803F0D1FBF0E75C4B93F81A31EBE7D4
:10EFB0005A4BD3F8E0306360E7E7584B011D93F8F4
:10EFC000300103F0D9FBE0E7544B93F81931DBE74C
:10EFD000524B93F88C30D7E71C238DF808304F4BF9
:10EFE00002A993F8480001F021FD6060CDE74C4B89
:10EFF000043493E8030084E80300C6E7494B043473
:10F00000F7E7494B0434F4E7484B0434F1E71A239B
:10F01000E3E71923E1E7414B93F86830B4E73F4B4E
:10F020005B6DC8E73D4B9B6DC5E73C4BDB6DC2E7B5
:10F030003A4B1B6EBFE7394B5B6EBCE702238DF882
:10F040000830364B02A993F87C2093F848008DF8DD
:10F050000A2001F0EBFC207197E7304B93F8DD308C
:10F0600092E72E4B93F839308EE72C4B93F8DC3037
:10F070008AE72A4B93F8383086E7284BDB6C9AE70F
:10F08000264B93F850307FE7244BD3F884306360ED
:10F090007BE7224B8FE7264B8DE7204BD3F8CC3014
:10F0A000F5E71E4BD3F82C31436001F04DFDA06015
:10F0B0006BE71A4BD3F890307DE7184B93F81F316C
:10F0C00062E7164BB3F88830A3805EE7134BB3F8C2
:10F0D0008A30F9E7114BB3F8D030F5E70F4BB3F8AE
:10F0E000D230F1E70D4B93F848200AB1062A12D12D
:10F0F000B3F8A035E8E7094B93F848200AB1062A8F
:10F1000009D1D3F8A43556E704B0BDE8104000F0AB
:10F1100021BE03203AE7182038E700BF042400206E
:10F1200070240020B824002078240020C02400206F
:10F13000401E00207FB5044610B9032004B070BD06
:10F14000A34DD5F840339A0700F16F820278412A27
:10F1500000F26882DFE812F04200470055005B00D1
:10F160005F00640069007600810087008D009300D5
:10F1700099009F00A500AB00B5006602BA00DC0054
:10F18000EF0016013801290142014B014F015301E3
:10F1900057015B0166025F01710199018701AB01B3
:10F1A000B101B801BD01C201660228026602660211
:10F1B000660266026602660266026602660266020F
:10F1C000660266026602660266026602340239025E
:10F1D0003E02430248024D0252025C020079FEF7F1
:10F1E00073FA30B1AAE70379022BA6D0794A82F8E4
:10F1F000303195F8913443F0200385F891340020A4
:10F200009CE7406803F04CFA0028F2D095E740688C
:10F2100003F08AFAF8E76F4B027983F81A21E8E7DE
:10F220006C4B4268C3F8E020E3E76A4E416896F809
:10F23000300103F097FA00287FF47FAF6368C6F8C7
:10F24000E430D6E7416800293FF477AF002001F0B1
:10F25000DDF90028CDD0112070E7416800293FF486
:10F260006CAF0120F3E7416800293FF466AF082046
:10F27000EDE7416800293FF460AF0920E7E7416806
:10F2800000293FF45AAF0C20E1E7416800293FF420
:10F2900054AF0D20DBE7416800293FF44EAF0E204C
:10F2A000D5E7416800293FF448AF0F20CFE74A4C2B
:10F2B000484B007983F81901A36D9847E36A984792
:10F2C00097E7444B027983F88C2092E7414E037A0A
:10F2D0008DF8043096F8480096F87D308DF80530AA
:10F2E000072201A901F0B5FB00283FF426AF6368AF
:10F2F00096F848000193002201A901F0AAFB00281A
:10F300003FF41BAF6C36D4E9010186E8030070E7D7
:10F31000304E037A8DF8043096F8480096F87D3028
:10F320008DF80530072201A901F093FB00283FF476
:10F3300004AFB436E7E7274E037A8DF8043096F829
:10F34000480096F87D308DF80530072201A901F0BC
:10F3500080FB00283FF4F1AED4E9010106F174030B
:10F3600083E8030096F81831022B7FF442AF96F839
:10F370003031002B3FF43DAF174BDB6A9847FEF767
:10F3800075F936E7134E037A8DF8043096F8480085
:10F3900096F87D308DF80530072201A901F059FB60
:10F3A00000283FF4CAAEBC36ADE7436802930123A0
:10F3B0008DF80C30074B02A993F8480001F056FB7A
:10F3C00000287FF416AFB8E6436802930023EFE706
:10F3D000C8290020042400205879030803795A1E04
:10F3E0000E2A3FF6AAAE934A82F8683001E7914BA5
:10F3F00042685A65FDE68F4B42689A65F9E68D4B87
:10F400004268DA65F5E68B4B42681A66F1E6894B8D
:10F4100042685A66EDE6874C037994F848008DF807
:10F420000430062201A901F014FB00283FF485AE48
:10F430009DF8043084F8DD30DBE67E4C03798DF8EE
:10F44000043094F8480094F87C308DF8063005229A
:10F4500001A901F0FEFA00283FF46FAE9DF80430D8
:10F4600084F83930C5E6734C037994F848008DF878
:10F4700004300A2201A901F0ECFA00283FF45DAE45
:10F480009DF8043084F8DC30B3E66A4C037994F8D4
:10F4900048008DF80430092201A901F0DAFA0028A9
:10F4A0003FF44BAE9DF8043084F83830A1E6614B50
:10F4B0004268C3F89420DA649BE65E4B027983F8D5
:10F4C000982083F8502094E65A4B4268C3F8842071
:10F4D0008FE6584B4268C3F8CC208AE6012B40F0F7
:10F4E000A480554C2421204603F01CFA636A9842FC
:10F4F00001D0172022E61C2104F1280003F012FAA3
:10F50000636C9842F5D14FF4807104F1480003F028
:10F5100009FAD4F848319842EBD1D42104F5A67009
:10F5200003F000FAD4F820329842E2D1002104F529
:10F53000097003F0F7F9D4F824329842D9D14FF486
:10F54000607104F50A7003F0EDF9D4F8A83598421B
:10F55000CFD1142104F2AC5003F0E4F9D4F8C03553
:10F560009842C6D1334E2146304640F2C45203F091
:10F57000C3F9204640F2C452002103F0D1F995F8B6
:10F580001B3485F8E833736FC5F8EC3396F87D309B
:10F5900085F8F83340F20123A5F8FA33274B96F8A3
:10F5A00019019B6D984724E68379012B3FF6C5AD81
:10F5B000204B42684068C3F82C2100F0BDFE48E6AD
:10F5C0001C4B4268C3F8902013E61A4B027983F86B
:10F5D0001F210EE6174B8288A3F8882009E6154BF9
:10F5E0008288A3F88A2004E6124B8288A3F8D020F0
:10F5F000FFE5104B8288A3F8D220FAE50D4B93F873
:10F6000048200AB1062A12D1A288A3F8A025F0E565
:10F61000084B93F848200AB1062A08D16268C3F85B
:10F62000A425E6E500F098FBDBE5012086E518203F
:10F6300084E500BF04240020401E00205879030800
:10F640002DE9F04387B00023ADF8003006460028CE
:10F6500000F0EE800361FEF747FD20B10124204653
:10F6600007B0BDE8F08300F065FD0028F6D100F09A
:10F670005BFD014618B96F48142203F051F96E4D35
:10F6800095F89134012243F0040385F8552485F858
:10F69000913433788DF804300021013B8DF805203A
:10F6A000ADF806100C2B00F2BB80DFE803F007B9C1
:10F6B000B9B97982B9B990B9AD9AA900D5F84073B2
:10F6C00017F02007CAD196F80480B8F1020F46D18E
:10F6D000DFF868815A4CFEF763F896F9051098F840
:10F6E00048003A4601F00FFA88F83900B37988F8F3
:10F6F0003830384607238DF80530FDF7E5FFFF2346
:10F7000004F58670A5F80C31C5F8084185F8047138
:10F7100003F01AF804F58A7002F0D0FF3846FDF7BE
:10F720002DFE0446002839D096F9051098F84800B7
:10F73000012201F0E8F988F83900D5F894343361F2
:10F74000002C71D000F0F0FC002888D195F891349D
:10F7500085F81A0460F3820385F891347FE7B8F1E5
:10F76000010F4FF00204E8D1DFF8D0908DF814407B
:10F7700099F8480089F81D7102A901F065F93379FB
:10F7800089F830318DF805708DF80680FDF7C4FCDE
:10F7900095F8913443F0100385F891340024CCE7B8
:10F7A00000226946022000F0F3FA0028F6D0132464
:10F7B000C3E7244BB288DB6B96F90C10B06898470E
:10F7C000D5F8403343F00203C5F84033E6E702A919
:10F7D0000D2000F053FB0028E0D0002269460D20E8
:10F7E000E1E7164B93F81831D3B9347904F00700E8
:10F7F00000F0ABFA8DF80040012269461020D2E7F4
:10F80000002269461220CEE78DF8072000F08EFA1C
:10F81000044638B900F087FA204600F089FABDE7BF
:10F8200002248AE7012488E701A800F0D1FB16E74B
:10F83000032414E71C2E0020C829002004240020E3
:10F84000CA290020587903082DE9F04F99B0804665
:10F85000059118B9032019B0BDE8F08F00230361AA
:10F86000FEF742FC0446002840F0A58046460FCE35
:10F870000EAD0FC51422524898F800A0B8F80C70CD
:10F8800098F90EB04F4E214603F04AF84E4B012234
:10F8900083F8412496F83021022A25460BD196F8A8
:10F8A0001821022A07D196F81E2122B9BAF1010FB8
:10F8B00038BF4FF0010ABAF1010F2BD0BAF1030F94
:10F8C0002AD0BAF1000F33D102229DF83C30DDF886
:10F8D0004090029362F34715012496F87C108DF84E
:10F8E000321002220CA996F848008DF8302001F061
:10F8F0009DF896F81A3196F830C196F81D1140B26D
:10F90000002B63D0BCF1010F57D1002955D1002C39
:10F9100061D153E00422D8E70023DDF83C90BDF824
:10F9200040709DF942B0029365F01F050124D4E7B1
:10F930004FF0000BD946CDF808B0CEE74FF00100EC
:10F9400084F81A04D2E005F29A420BA900F0D4FA26
:10F95000002800F015811320049B33871A4B0022E6
:10F9600083F81A2423E105F29A452A460BA900F0F0
:10F97000C3FA0028EFD10B9B84F82801C4F82C515E
:10F9800084F83031FCE0B9F1000F00F0F980002A72
:10F9900000F0F6804946E01C02F0AEFF94F83732E2
:10F9A00001332380ECE01220D6E70220D4E70720C1
:10F9B000D4E71320D2E701204DE7FCB90220F6E09E
:10F9C000082E002004240020C8290020002CF5D097
:10F9D0005845B8BF584696F87C308DF8200005226F
:10F9E00096F848008DF8223008A901F032F8002876
:10F9F0003FF430AF9DF8203086F839306F4A704BB5
:10FA0000D2F89804D3F8904038B105F053FA6C4B13
:10FA100084423CBF002283F83A20198F1A8F93F852
:10FA200030010491996A099152BA0028BFD093F825
:10FA30001B0100B9186393F81801ADF8582001387C
:10FA400093F87C2093F81A411491D0F1000BD3F86D
:10FA500088108DF85B204BEB000B93F8482093F84F
:10FA60003A0093F868308DF85A3009AB0093554B43
:10FA700003904FF001008DF84C0015918DF85C203B
:10FA8000A3F12F01A3F1300213A88DF84D4000F02F
:10FA9000DBF8039B4FEA0B1B4BEA431B00264BEAA8
:10FAA000801B4BEAC413B145444C039308BF37464F
:10FAB0003A46494604F59C70CDE90A669B46268085
:10FAC00084F81A6402F018FFE9B2A570C5F3421574
:10FAD000FAB2042D3A4E039B84F837223FF42EAF3E
:10FAE000072D3FF450AF022D7FF45FAF364D84F801
:10FAF0000D110420029984F80401FF2084F80C0100
:10FB000084F8281184F81431D6F8E410C4F80851A8
:10FB100005F59B730AA8C4F8101184F83021C4F8C5
:10FB20002C3100F011FC00287FF43DAF0A9BA4F8B3
:10FB300044040BA8A4F81631C4F84C3400F0D0F9F2
:10FB400000287FF408AF0B9BD3B196F93900FDF77D
:10FB5000F7FA94F83732002B3FF405AF0B9B0F2BCD
:10FB60003FF6F1AE05F58B720BA90F2000F0C4F93A
:10FB700000287FF4F0AE0B9B63F3030B84F814B101
:10FB80000598FDF7FBFB00287FF4E6AE099B86F89D
:10FB90003A00B36200F080F900287FF40AAF94F8CD
:10FBA000913484F840A443F0010384F89134034B6A
:10FBB000D3F89434C8F810304DE600BFC8290020AF
:10FBC000042400206C240020CA29002037B50B4DE6
:10FBD0008DF8040004460F2295F8480001A900F0B2
:10FBE00038FF40B1064A85F81C4192F8913443F041
:10FBF000200382F8913403B030BD00BF04240020FC
:10FC0000C829002010B5FFF7C1F8044688B90A4892
:10FC100005F08AF9094805F087F9094805F084F9E3
:10FC200000F094F8FDF7BCFD064BDB6A98472046D0
:10FC300010BD0124FBE700BF302D0020482D00201F
:10FC4000602D0020587903082DE9F04F8BB04778DC
:10FC50000093149B90F90C8090F90D6090F80EB011
:10FC60008A464168196004469146002F58D0022305
:10FC70008DF8103004A9C37B007C8DF8123000F0A1
:10FC8000D5FEB4F808C0618943B26068984545461E
:10FC90006144B8BF1D46604534BF00270127884234
:10FCA00009D30A218DF81010207C019304A900F0DB
:10FCB000BDFE019B46B2B4F808C0608961680CEBD8
:10FCC000400E714519D3A1EB0C01B1FBF0FC00FB18
:10FCD0001C1191B9984503DC2378CBB94FF0010B87
:10FCE00021238DF81030207CE37B8DF8115004A97E
:10FCF0008DF8123000F09AFE45B2009B8AF8005051
:10FD0000384689F8006083F800B00BB0BDE8F08F8A
:10FD10000223207C8DF8243006A900F095FEDDE753
:10FD20004546EAE7704770477047704700207047C4
:10FD300070477047704700207047002070470020D0
:10FD40007047002070470020704770477047704729
:10FD50000220704702207047022070477047002041
:10FD60007047704770470020704700207047704709
:10FD70007047704710B5054C4FF4037220460021C0
:10FD800002F0CEFD0020C4E9000010BDE42E0020EA
:10FD90002DE9F8438146904600293CD01F4C202392
:10FDA000224604F1100012F8017F6FBB8242FAD1A3
:10FDB0001B4E3368013403B93460736803B11C60AF
:10FDC00000252560C4F8088074601FFA88F284F862
:10FDD0000490601D02F090FDB9F1110F4FF0000387
:10FDE00098BF104D6373D6F8083298BF25FA09F50D
:10FDF00003F1010398BF05F0010543442573C6F8DC
:10FE000008323846BDE8F883013B13F0FF0304468F
:10FE1000C6D10227F5E70127F3E700BFEB2E00204C
:10FE2000E42E00202007020010B518B3124A136810
:10FE3000984204D103681360002305E00B46002BB1
:10FE4000FAD019688842F9D15168884208BF5360D6
:10FE50000BB101681960D2F808328168013B0024B7
:10FE60005B1A04602146C2F80832102202F058FDE5
:10FE7000204610BD0120FCE7E42E0020054B1B6846
:10FE800013B11A798242FAD1002B0B600CBF032008
:10FE900000207047E42E002010B5054B186800B90B
:10FEA00010BD037B04680BB9FFF7BEFF2046F6E7E1
:10FEB000E42E002038B5084B084C186800B938BD4E
:10FEC00003790568112B05D824FA03F3DB0701D564
:10FED000FFF7AAFF2846F1E7E42E002020070200E2
:10FEE00028B1044BD3F8083203600020704701208A
:10FEF000704700BFE42E00202DE9F04107460E4672
:10FF0000154642B339B3154B1C6800232CB9304653
:10FF1000FFF7E6FF0020BDE8F081A268F91A013280
:10FF2000914215D32279EA54581C22895FFA80F84D
:10FF3000611D55FA80F002F0DFFCA3682468984444
:10FF40005FFA88F3E2E720462568FFF76DFF2C464D
:10FF5000002CF8D1DBE70120DDE700BFE42E002014
:10FF60000238C0B211289ABF014B185C00207047BC
:10FF70007372030830B50B4B93F8202004460846F3
:10FF800072B100211C330578A54208D00131984296
:10FF9000CDB214BF04301038AA42F4D8002030BDCE
:10FFA0001046FCE7F030002010B5084C002320601C
:10FFB000142204F10C00FF2184F82030C4E9010070
:10FFC00002F0AEFC012384F8213010BDF030002097
:10FFD00010B50E4A92F82010042915D893680478B9
:10FFE0001C7044785C70C478807898700131DC7043
:10FFF00082F8201002F11C018B4214BF043302F17D
:020000040801F1
:100000000C039360012010BD0020FCE7F0300020BD
:10001000094B93F8200068B15A6803F11C018A4229
:1000200000F1FF3014BF043203F10C0283F820000A
:100030005A600120704700BFF030002010B5074B18
:1000400093F820200446084632B15968FFF792FF22
:1000500010B101234470837010BD00BFF030002048
:1000600008B5064B93F820202AB15968FFF782FFA4
:1000700008B1407808BD0120FCE700BFF030002047
:1000800030B50A4A92F82010536882F8210061B115
:10009000916801241C32DD78587005B99C70934238
:1000A00014BF0433103B9942F5D130BDF03000202D
:1000B00008B5044B5968FFF75DFF003818BF0120F1
:1000C00008BD00BFF0300020F7B50422154E0446ED
:1000D00000210DEB020096F8207002F021FC0025B3
:1000E000EBB29F4201D803B0F0BD7368197821705C
:1000F0005A786270987838B1336820469B68984780
:10010000FFF786FF0135EBE7DB788DF804108DF8FB
:1001100005208DF80730FFF77BFF01A8FFF758FF98
:10012000F0E700BFF0300020014B93F8200070474B
:10013000F0300020034B93F82000042894BF0020E7
:1001400001207047F03000201FB50024CDE90244A3
:10015000C41F8DF800408DF801100C0AADF8042082
:10016000090C120C8DF803108DF806208DF807305D
:1001700002461B0A012168468DF802408DF80830BE
:1001800002F029FA002818BF0E2004B010BD2DE996
:10019000F04188B090460D460F9A0746002847D098
:1001A00000240121CDE904448DF810109DF8381089
:1001B0008DF81510ADF81630190CCDE900441B0E62
:1001C000CDE902448DF81930ADF81A20130C120E47
:1001D00007948DF818108DF81C308DF81D20E3B2AF
:1001E0001E01002DF6B203DC002008B0BDE8F0814E
:1001F000013310218DF81F3042466B460DEB010094
:1002000002F07FF90346A8B9102D28463E44A8BF46
:1002100010206946327811F801CB013382EA0C02D2
:10022000984206F8012BF5DC103D2DB20134D6E7DB
:100230000920DAE70E20D8E70138032815D8DFE8CF
:1002400000F002080C100A4B1B681B690B600020B1
:100250007047074B1B685B69F8E7054B1B689B6998
:10026000F4E7034B1B68DB69F0E70520704700BF2C
:10027000143100202DE9F041C4B00C464A9E1746C7
:100280001D468046B8B3B1F5807F36D84FF48872EA
:100290000021684602F044FB492300934FF4807329
:1002A000ADF804302B0C8DF80830330CADF8065047
:1002B000ADF80A608DF80C3022460023414604A8B0
:1002C0002D0E360E8DF80E308DF809508DF80D601C
:1002D0008DF80F4002F010FB04F110014B9A3B46E1
:1002E00089B2684602F0F7F810B1012818BF0E2055
:1002F00044B0BDE8F0810920FAE70D20F8E70000DE
:1003000010B590B10A4C28220021206002F008FBB1
:100310002368084A1A6000204FF0FF32C3E9030245
:10032000C3E90522C3E9072210BD0820FCE700BF8E
:100330001431002000010101024B1B6818600020ED
:10034000704700BF1431002030B1044B1B68DB68DC
:1003500001330360002070470920704714310020EA
:1003600013B500230C460193CAB101A9FFF764FF3E
:1003700018B9019B591C02D1146002B010BD99B28A
:10038000611A002901DD5C18F6E702D1136007202D
:10039000F3E71B0C1B0403F580331C44ECE7092036
:1003A000EBE7000028B1044B1B681C3343620020BC
:1003B00070470920704700BF143100201FB5044664
:1003C00000B3002303A8039302F05CF9104ABDF8C0
:1003D0000C30126820469380E38200F05EFA98B9F0
:1003E00004F11803009321680123132202F068F836
:1003F00060B9204600F051FA003818BF0120000112
:1004000004B010BD0920FBE71020F9E70E20F7E744
:1004100014310020F0B5054687B01C4613B90920F9
:1004200007B0F0BD2E4E3368DB68834255D894F890
:100430002020002A0CBF08220922834205D320462F
:1004400000F05FFA68B11020EAE700230190009302
:10045000A36894F82810606AFFF799FE0028EED090
:10046000DEE723792168B4F808C0A768043B9AB294
:100470000029D4D0B2F5807F2DD8ADF80EC08DF80C
:1004800017304FEA174C04F12C033F0E8DF8117012
:1004900000932F0C08234FF0490EADF80C008DF897
:1004A00014708DF816002F0E0DEB0300CDF808E048
:1004B0008DF810C0ADF812508DF8157002F000F8EC
:1004C00008B10E20ACE7204600F01BFA0028BAD194
:1004D0003368DD60A4E70D20A2E70620A0E700BF97
:1004E000143100202DE9FF410A9D80460F46164633
:1004F0001C46002D5AD0002303A910460393FFF792
:100500009BFE18B1062004B0BDE8F081039B9C421D
:1005100001D80133F6D1284600F064F9002847D10C
:10052000264B1A78424503D01A79424542D1012020
:10053000AA68BA4240D103EB8002EB6A92F80180CC
:100540002979CDE900430439927828683B4689B27D
:10055000FFF790FE0028D6D195F820300194002BAB
:100560004FF00103009314BF4246082295F828106B
:10057000686A3B46FFF70BFE0028C4D1013E032EFC
:10058000C1D8DFE806F002070B0F0D4B1B681C619A
:100590001C62B8E70A4B1B685C61F9E7084B1B68F3
:1005A0009C61F5E7064B1B68DC61ACE70920AAE714
:1005B0000F20A8E70B20A6E70220A4E724040020D0
:1005C000143100201FB50B294FF00003CDE9003393
:1005D000CDE902330A4607D00C2914D00A2910D0DD
:1005E0000A2005B05DF804FB012802D120238DF814
:1005F00000300021684601F0EEFF002818BF0E20F1
:10060000EFE73023F3E70B21F4E7000038B50546A8
:1006100001F0DCFF044610B10E24204638BD002D49
:10062000FBD1094B1B680B219878FFF7CBFF002803
:10063000F2D10C21FFF7C6FF0028EDD10A21FFF708
:10064000C1FF0028E9D0E7E7143100202DE9F0438D
:1006500080468FB00C461746002A6BD0002969D01F
:10066000002529461D2206A805951DF091FF8DF84D
:100670001350344D2B680DF114099E88CDF8049069
:100680000DF1130302933B7900933B6832462146F8
:10069000404601F0BCFF00284ED138683A794946FF
:1006A00002F02AF9384600F04FF8002846D13C7A8B
:1006B000FA79BB79240444EA02241C432B689A6823
:1006C00094423DD99C609DF813000B21FFF77AFFFF
:1006D000034658BB0C21FFF775FF034630BB0A21C8
:1006E000FFF770FF034608BB7B7ABA7AFF7A3F04B4
:1006F00047EA02271F433A46334621460920FFF7BF
:1007000023FD034690B933463A4621460820FFF7B9
:100710001BFD034650B92A689DF813109170002103
:10072000D1604FF0FF31C2E90411916118460FB05A
:10073000BDE8F0830923F9E70E23F7E70F23F5E778
:100740000323F3E71431002010B50446002845D0F8
:100750000168002942D011F8013B437103220630A1
:1007600002F0CAF82046032250F8091B043102F0B7
:10077000C3F82168CB79E3600A7A43EA0223E36095
:100780004A7A43EA0243E3608A7A43EA0263E36017
:10079000CB7A23740B7B63742379212B1AD110221B
:1007A0000D3104F1120002F0A7F81D222168501C3F
:1007B0008B5C6362085C43EA0023901C6362085C04
:1007C000033243EA004363628A5C43EA0263636282
:1007D000002010BD112B03DC0D22E7E70220F8E713
:1007E0000120F6E710B50446002854D0016800291E
:1007F00051D00B7843714B7883608A7843EA0223A7
:100800008360CA7843EA024383600A7943EA026359
:1008100083604B7903738B79C381CA7943EA0223DE
:10082000027BC38102F00F020831103002F064F83D
:10083000237B002203F00F0384F8202084F8282073
:10084000227903F10800111A04290DDD216809330A
:10085000043AD21A085C84F82000D2B2606A84F8A4
:100860002820194402F048F8237922681A4400200D
:1008700012F8043CE36212F8031C43EA0123E3622A
:1008800012F8021C43EA0143E36212F8012C43EA26
:100890000263E36210BD0220FCE710B5044660B3BA
:1008A000036853B30279162A29D942791A7001468E
:1008B000082251F8060B013002F028F821460822E0
:1008C00051F80E0B093002F021F82368E28A5A74BD
:1008D000E38A22681B0A93742368A269DA74A36905
:1008E00022681B0A13752368628B5A752368E27E9F
:1008F0009A7517232371002010BD0120FCE7022008
:10090000FAE738B50446002863D00168002960D0B2
:10091000037B90F8282003F00F03002A57D10833F7
:10092000207904321344984255D363790B702368BD
:10093000A2685A70A36822681B0A937023686289B0
:10094000DA702368E27A1A712368227B5A7123686D
:10095000E2899A71E38922681B0A2146D371227BBE
:1009600051F8100B02F00F02083001F0C5FF237B95
:1009700094F8282003F00F0303F108052AB1226838
:1009800094F82010515503F10905206894F82820A7
:10099000616A284401F0B0FF94F828302268E16AC7
:1009A0002B44D1545A1CE16A206892B2090A81543E
:1009B0009A1C2168E08D92B28854DA1C216894F860
:1009C0002F0092B2043388542371002038BD0933BC
:1009D000A6E70120FAE70220F8E70000024B1A8898
:1009E00010431880704700BF1831002008B5074B2E
:1009F0001B883BB1FEF7CAF9002814BF6FF0020054
:100A0000002008BD6FF00100FBE700BF1831002097
:100A100010B5034B00241C80FEF7AEF9204610BD34
:100A200018310020B0FA80F04009704782B018B940
:100A3000084602B000F0CAB8002002B0704710B9F2
:100A4000084600F079B9704710B9084600F090B92F
:100A500070470346084611460BB900F0DDB9002087
:100A6000704710B9084600F039BD704710B9084604
:100A700000F0FEB90020704710B404460846114645
:100A80001A46019B14B910BC00F00CBA10BC704798
:100A90000346084611460BB900F036BA00207047ED
:100AA00010B40446084611461A4614B910BC00F0AA
:100AB000A3BA002010BC704730B405460846114662
:100AC0001A46DDE902341DB9029430BC00F022BBA5
:100AD000002030BC704710B9084600F0D3BB00209E
:100AE000704710B9084600F037BD0020704710B9B4
:100AF000084600F0E2BB0020704710B9084600F03D
:100B0000DFBB002070470346084611460BB900F0D2
:100B1000F9BB0020704710B40446084611461A4637
:100B2000019B14B910BC00F0EFBB092010BC70474A
:100B300010B40446084611461A4614B910BC00F019
:100B40002DBDC8B210BC70470048704701000102BB
:100B5000064B10B51B6A0446984730B10448054B54
:100B6000204498428CBF0020012010BD5879030812
:100B7000403576C9405DC600F0B5114B85B00C46D6
:100B800010491F56054601F017F80F4BE4B25E6A94
:100B9000072D4FF00103CDE9024301460AD105229A
:100BA0000023CDE900234FF47A727A431846B04708
:100BB00005B0F0BD08220020CDE900203A46F5E757
:100BC0004073030820730308587903081FB50023F6
:100BD00000930378013B372B21D8DFE803F01C2476
:100BE0002020201E202020204143454E2055585BC8
:100BF0005E6164206C1E6E73787A7D207F83262070
:100C000020202020202020202020202085878C20AC
:100C100020858C208E92C3780BB10223009300981C
:100C200005B05DF804FB8378F6E743788DF804306F
:100C300007238DF805308378003B18BF01235B0044
:100C40008DF8063010238DF80730314B1B6801A852
:100C500003F55872CDE9022300F08EFF0090DEE725
:100C60004023DBE72023D9E7827890F9013012B9DD
:100C7000284AD35CD2E7284AFBE7827890F9013012
:100C8000002AF8D1254AF4E740F6B833C6E74FF416
:100C90007A73C3E74FF4FA63C0E741F28833BDE7E4
:100CA00041F27073BAE71E484FF47A7101F008FE02
:100CB00000F5FA60D2E71B4BB0E7154B1B6803F554
:100CC0005873ABE7124B1B6803F55B73A6E7102361
:100CD000A4E70F4B1B68A1E701239FE74FF0834375
:100CE00000939CE7104BFBE7104B97E740F2111382
:100CF000ADF8003093E7032390E790F901300C4AF8
:100D0000B7E70C4990F9010000F056FFA6E700BFD5
:100D10002031002015730308057303080D730308C1
:100D200018FCFFFF00EA06379A99094040F7093797
:100D3000407303082073030837B50B4B02781B6818
:100D40000C2101FB02335B7A03EB4304074B1D6864
:100D500003690093C3684278816805EBC40000F022
:100D6000A7FC03B030BD00BF203100201C310020A3
:100D700030B587B0027B6423ADF80030012A4FF014
:100D80000003CDE90133CDE903338DF802308DF84E
:100D9000143028D0022A2FD01ABB03680BB3436843
:100DA000FBB11A4C80682360194B18226946186001
:100DB00001F0A2FD174B246893E807000C3384E888
:100DC000070093E8070004F10C05032385E80700FA
:100DD000A4F86C33012204F55B7104F5587000F03F
:100DE00058FC07B030BD094908684360036100F54D
:100DF0005B7100F55870F2E7044B1B68B3F8602391
:100E0000B3F86C130A43A3F86023EAE7203100200B
:100E10001C310020B01B030808B503460A2924D85A
:100E2000DFE801F006232323230B161B23212100D7
:100E3000BDE808400068FFF78BBE90F90000997884
:100E4000072271B900F0E5FB003818BF012008BD8A
:100E5000052293F900000021F4E790F90000597889
:100E6000EEE70221EEE70722F3E70020EFE70000BC
:100E700008B502791AB1012A0BD0002008BD084B31
:100E800001681B68012203F5587000F002FC012084
:100E9000F4E7034B01681B6803F55B70F5E700BFDF
:100EA00020310020F7B50728144D1C46A8BF0720A5
:100EB00058700E462946174600F07EFE94F9013020
:100EC000A070072B13D1322000F076FD0C4BDB6DA8
:100ED0000546984704F10C02083403460192009439
:100EE0003A463146284600F06CFD03B0F0BD054A95
:100EF00055F82310D05C00F057FDE7E72073030896
:100F000058790308407303082DE9F04F344F90F9E6
:100F100001607B68D0F804908BB0044688469847FF
:100F20000546002859D1E37C73B92E4A237812680C
:100F300003EB4303990002EB8303D3F80490B9F168
:100F4000000F01D152F80190274B484613F906B023
:100F5000FB689847A37C2289D7F818A00993072E2D
:100F600028D100230121CDE90223204A0693CDE9AF
:100F70000431CDE907330521CDE900214FF47A7220
:100F800002FB0BF24CF250311846D047637C13B38E
:100F9000174B995D7B6D0D31C9B228469847E07CAF
:100FA0003246494600F01AFE88F8006001200BB076
:100FB000BDE8F08F002101250823CDE90013CDE91C
:100FC0000715CDE90511CDE903110292A1782B4651
:100FD0005A462846D9E7074BDBE70020E7E700BF82
:100FE000587903082031002040730308854501002B
:100FF0000D730308157303082DE9F04F8DB090F9B8
:101000000130DFF8FCA0DFF8FC90CDE90A123E4A7F
:1010100012F903B00278DAF800300C2505FB023330
:101020003A4A5B7A126803EB430302EBC3030446BC
:1010300093F9021090F9020000F0B9FD3449064618
:1010400094F9010000F0B8FDA2686168804630465E
:1010500000F0DFFC2178DAF80020D9F80C30694381
:10106000074650589847D9F81C309C4694F90130EF
:101070000025072B4FF47A63CDE90753CDE90555D9
:101080002DD10123CDE903530523CDE901534FF4BD
:101090007A7303FB0BF300933946434646F2A812DA
:1010A00028466746B8472378DAF800200C214B43DE
:1010B00094F90110D05800F0B3FDA18994F9010012
:1010C000FFF75AFD0B9B217B1860D9F85430284656
:1010D00098470A9B01201E700DB0BDE8F08F0120DB
:1010E0000823CDE90350CDE901032A46CDF800B02D
:1010F000654643463946A84701200546D3E700BF69
:101100002031002058790308407303081C31002067
:10111000207303082DE9F04F8FB0002405468A465E
:10112000914698460494ADF81440ADF80240072665
:101130004FF0010B2B7AA34206D9686804A920441A
:1011400000F0CAFB00285DD102238DF8083002A808
:101150006B7A8DF80A30FFF739FDAB7A8DF81D30C8
:101160009DF811308DF81E309DF812308DF81F302B
:101170009DF810308DF82030EB7A8DF821302B7BE4
:101180008DF822306B7B8DF8233010238DF81C6096
:101190008DF824303A4E8DF82C000DF102030A939D
:1011A000072332688DF82D30ADF834302B680C925F
:1011B00006930DF1120204AB0DF1110106A800F027
:1011C000A5FB072805460BD130680C22002100F54D
:1011D000587001F0A5FB3368BDF80220A3F8602326
:1011E0009DF811308AF800309DF8123089F80030EF
:1011F0009DF8103088F80030189B28461C700FB0FE
:10120000BDE8F08F9DF81330BDF81470ADF8027092
:101210002044C4B2F3B917B3194A00201168072655
:1012200002464FF00C0C062B1BD10CFB00FE51F8B4
:101230000EE0BEF1000F04D00BFA00F23A4397B271
:10124000012201301028EED1002A3FF473AFADF82F
:1012500002706FE75A1E042A01D9062BDCD006263D
:1012600068E747FA00FE1EF0010FEAD00CFB00FE13
:1012700051F80EE0BEF1000F08BF0626E1E700BFFF
:101280002031002038B505464068FFF761FC072291
:10129000841D002195F90000E4B200F0BAF908B904
:1012A00004F0FD0495F901000722002100F0B1F9D6
:1012B00008B904F0FB04204638BD00207047000048
:1012C00010B503780F2B044618D84068FFF740FC90
:1012D00022780B4902EB42020968831C01EB820071
:1012E00051F82220DBB21AB903F0FD0358B210BD49
:1012F000032B06BF626842600223F7E70020F6E78F
:1013000020310020022070472DE9F0413A4D04467B
:10131000286896B00E46904600211F4601220323FE
:1013200000F55870CDE90411CDE906118DF80C10C7
:101330008DF80D10ADF80E3000F08DF930B92A6837
:10134000B2F8603343F00303A2F860332A68637A8B
:101350008DF8203002F55871CDE90912274A94F929
:10136000083012680B921022ADF830200DF10E02F9
:101370000D9222680E9262680F92D4E90301A27A5C
:101380008DF8402001228DF8412011AA82E8030047
:10139000227DE18A8DF8213018468DF84C20FFF728
:1013A000EBFB08AB15930DF10D0314900093CDF8F2
:1013B000048003AB04AA39460EA800F099FB04464A
:1013C00078B99DF80C10013901F07AFA00F1580350
:1013D0000DEB030010F8483C3370204616B0BDE812
:1013E000F0810C2801BF2A68B2F8603343F0030390
:1013F000A2F86033F1E700BF203100201C3100204B
:10140000F8B50679012E054648D90F2E48D803684D
:10141000187A40F303000722002140B200F0F9F8E7
:101420002B680446187A40F303100722002140B2CB
:1014300000F0EFF8B8B1B4FA84F4640929680B7AC3
:10144000086843F3030243F303135BB252B29A42B8
:10145000C8BF0124FFF77CFB80F00103DBB224B19D
:101460000533D8B2F8BD0124E8E7DBB90E4F29688F
:101470003B6806EB460003EB80000C2201F03CFACF
:101480003A680C2303FB062320465C72B2F8601313
:101490000123B3400B43A2F86033E3E70620E1E702
:1014A0000320DFE70420DDE72031002010B40178BD
:1014B00001290ED9084B18680C234B43C41800228D
:1014C000C250C4E9012200F5587010BC102200F08F
:1014D000A9B8002010BC7047203100202DE9F04150
:1014E00086B050238DF81430037A102B074630D184
:1014F0004368DD7B6DBB0224A8466426062C14D805
:101500007A68535D03932A44517843EA0123039395
:10151000927843EA02437343CDE9033863B96846DE
:101520008DF80040FFF7C2FF0DE0CDF80C808DF87C
:101530001480CDF81080F2E703AB01A801938DF879
:101540000840FFF75DFF0134E4B2102C05F10305FC
:10155000D4D106B0BDE8F0811FB5026803791168E7
:1015600049B901A88DF80430FFF7A0FF78B1032036
:1015700005B05DF804FB02A802928DF80C30FFF76D
:101580003FFF042805D0052805D00028EFD0002013
:10159000EEE70220ECE70120EAE70000C90020B9ED
:1015A000034B0B449856C0B27047024BF9E700BF9B
:1015B000C572030885720308F0B59A42069D03DBE5
:1015C0009DF914309A4220DD0020F0BD03EB430367
:1015D00031F814C005EB830300264CFA06F7FF0729
:1015E00007D51F7A07F00F0E964502DCB2EB171FE6
:1015F0000DDD0136102E03F10C03EED10134E4B2FF
:101600002301DBB29842E1D8DEE70024F8E70120AD
:10161000DBE7884204DB9042CCBF0020012070470A
:101620000020704710B51409B4EB111F03464FEAB0
:1016300011100ED391420CD202B201F00F0133F817
:101640001240012000FA01F124EA010123F81210EE
:1016500010BD0020FCE7F0B528B100EB41050127E3
:101660000020914200D3F0BD002435F802CB234680
:1016700007FA04F636EA0C0608BF013304F1010448
:1016800008BFDBB2102CF3D118440131C0B2C9B28B
:10169000E7E710B500B149B910BD31F8134020F8A3
:1016A00013400133DCB2A242F7D8F5E70023F9E793
:1016B00082B030B504880493D2B9B3F5616F15D305
:1016C00049F6AF2542F21072AB4298BF4FF47A72DE
:1016D000944238BF14466143BDE83040C3688B4232
:1016E0008CBF5B1A0023C36002B070476422EFE72F
:1016F000012C38BF0124EEE72DE9F04F8FB01546DD
:10170000199F03939DF8603007930C46804603F0C1
:10171000C7FB6A4A0590A7F5F633303BB3FBF2F3FB
:10172000534303F5F63B0493182313FB05430BF1D6
:10173000300B069300254FF0FF3A069B9C4207D1E1
:10174000002D14BF50464FF0FF300FB0BDE8F08FB2
:10175000BDF96830ADF824300999199738460897D3
:1017600003F02EFB2688B8F1000F5FD1B7F5616F4B
:101770005AD349F6AF2242F21073974298BF4FF402
:101780007A739E4238BF1E46642E59D1DFF83091DD
:10179000A060A1680CA803F035FB0D9B0093DDE968
:1017A00008120C9B0AA803F08CFA039A0A9B0AB948
:1017B000079A2AB122694A4502D1424A93420ED978
:1017C000414BC4F80C909F4209D90023ADF82C304E
:1017D0000B99CDF828B0584603F0F2FAA060606883
:1017E00008B9C4F80C90C4F81090B8F1000F04D0F8
:1017F00003F060FBE3680344E360D4E903329342FF
:10180000059B88BFE26063601B9BE168734399425C
:1018100004D20398E8B9B8F1000F1AD001231D448F
:101820002375EDB2183488E76423AAE7039B0BB94C
:10183000234BE360012EDFF8889038BF0126CEE706
:10184000B6F57A7F0ABFDFF88490DFF88490A06055
:101850009FE700209342207506D85B1A9A4505F150
:10186000010528BF9A46EDB2B8F1000FDAD1642E17
:10187000184AADF82C801DD049F6B023B6F57A7F12
:1018800018BF1346974281BF049A02F5A83202F5A9
:10189000C0729B180A931A9B00930AAE96E8060042
:1018A000199B304603F00DFA96E8030003F088FA1E
:1018B0008246B7E74FF46163E4E700BF805101005F
:1018C00040771B007F5101002FEC010080A812011E
:1018D000002E930230EC01000378032B14D14378DF
:1018E00003F00F021B098A704B7083788B80C278DB
:1018F00043EA02238B800379C3F3021203F00F0340
:10190000CA700B7005207047002070472DE9F3471F
:101910009A464379057990F907609146044690F913
:1019200006208846D3B190F90870002D37D00F2AD1
:101930001BD194F909200F2E27D194F90A00072D05
:1019400002D1002F08BF012788F8002089F8000085
:1019500028468AF8007002B0BDE8F08790F90B7055
:1019600090F9092090F90A60DFE7A369019394F9DF
:101970001530009394F914302169207BFFF71CFE89
:101980000028D8D105F0FD05D5E794F91D00B04237
:10199000D5DC94F91C30B34203DA05F0FB05304680
:1019A000D2E73046CBE70000024B03FA00F0B0FB71
:1019B000F1F0704740420F004FF4FA53B3FBF0F0E0
:1019C000704730B54FF47A750C1F6A4300FB042250
:1019D00052001EBF00F1FF341219B2FBF0F2914227
:1019E00038BF1146039A1160820048431CBF013082
:1019F00040084FF47A71121A01FB1323002BCABF5F
:101A000003F2E73393FBF1F1B3FBF1F1049B1960AF
:101A100030BD38B5400014460D46F0F7CBFA01460C
:101A20002846F0F715FA2146F0F712FAEFF78CFE88
:101A30001EF0BAFEF0F790F940B238BD2DE9F74F2D
:101A4000019300239C469E46048A1E01F6B2B442CE
:101A500046D906EB46054FEA4309AD000024476826
:101A600037F809702741FF0729D5876807EB050A72
:101A70007F5927B3077837B9476927B137F8097015
:101A80002741FF071BD59AF8087090F901B047F37A
:101A900003084FFA88F8D84511DC47F303177FB2E3
:101AA0005F450CDB9AF8097007EB4708C76807EB3E
:101AB000C8073F7D5FB90CF1010C5FFA8CFC013463
:101AC000102C05F10C05CAD10133DBB2BCE70EF1D5
:101AD000010706EB040801F80E805FFA87FEEEE7C7
:101AE000019B82F800E083F800C003B0BDE8F08FEE
:101AF0002DE9FF4704464068DDE90C671D468A462C
:101B0000914603F0D7F923681B1A3B604FF0000899
:101B10000123337085F80080636813B12368834222
:101B200024D8D4F81CC0CAF80080A3699CF800E04F
:101B30000393D4E9030101AB83E80300237D009301
:101B4000DCF80C10237A627A7046FFF7D5FD334635
:101B500038602A46E0694946FFF770FF2B782BB1C1
:101B6000C7F80080002004B0BDE8F0873378002B70
:101B70000CBF0C200B20F6E737B590F9002090F948
:101B80000250954204460FD0013A52B295420BD012
:101B9000A368019394F9013000936168E0782B46C3
:101BA000FFF70AFD0028EFD0104603B030BD884291
:101BB000B8BF08467047000051F82000054B984216
:101BC00005D0054BC31A58425841400070470120C8
:101BD000704700BF90D0030020A1070005281FB563
:101BE0000ED80C4B53F820300093CDE901120A4B6C
:101BF00001220021022002F06BFE05B05DF804FB1B
:101C0000CDE90012054B01220021022002F060FE06
